:020000040000FA
:040000006FD00400B9
:101000006F00907D00000000000000009020002094
:10101000AA220020A9BDF9F56C23002000000000E1
:10102000000000006C230020902000200000000041
:101030000000000090200020000000009020002010
:101040000000000090200020902000209020002030
:101050009020002090200020482F00208224002093
:101060000000000090200020902000200C24002090
:1010700090200020D22300209020002090200020EB
:101080009020002090200020902000209020002020
:101090009020002001A04111B7170040985F3AC688
:1010A000945F3247E39CE6FE3245410182800111A4
:1010B00013078008F337078093F787083EC20100C3
:1010C0000100B7170040930570052380B70413068D
:1010D00080FA2380C7040100010083C6B70493F699
:1010E000F60DA385D704238007049246F3A6068055
:1010F0000100010093760502D5CEF336078093F602
:10110000860836C4010001002380B7042380C70489
:1011100001000100B70614007D89558D88C70100C4
:1011200001000100010023800704A246F3A6068007
:101130000100010073370780137787083AC6010062
:1011400001002380B7042380C704010001000100CF
:1011500001003727004093061005A303D7802380A2
:101160000704B247F3A70780010001009307800836
:10117000F3B7078093F787083ECE01000100B71749
:101180000040130770052380E704130780FA2380CB
:10119000E7040100010003C7B70413670708A3852C
:1011A000E70423800704F247F3A70780010001004A
:1011B0000561828093760504BDC6F336078093F6F9
:1011C000860836C8010001002380B7042380C704C5
:1011D00001000100B7061400938606047D89558D31
:1011E00088C7010001000100010023800704C246F6
:1011F000F3A6068001000100733707801377870884
:101200003ACA010001002380B7042380C70401000B
:1012100001003727004093062005A303D7802380D1
:101220000704D24781B773370780137787083ACC12
:10123000010001002380B7042380C70401000100DE
:1012400098471367070C98C723800704E24719BF24
:101250000111814601468145114506CE97000000E7
:10126000E780405793078008F3B7078093F7870814
:101270003EC601000100B717004013077005238028
:10128000E704130780FA2380E7040100010003C785
:101290006704136717002383E70423800704B2471A
:1012A000F3A7078001000100F2400561828041112F
:1012B000814601468145114597000000E780805135
:1012C00013078008F337078093F787083EC40100AF
:1012D0000100B7170040130670052380C70493066A
:1012E00080FA2380D70401000100FD552396B70240
:1012F00023800704A245F3A5058001000100733790
:101300000780137787083AC6010001002380C704CD
:101310002380D7040100010003C767041367170087
:101320002383E70423800704B247F3A70780010063
:10133000010001A0B1473305F50201007D1575FDDF
:101340008280411122C426C206C6AA8401446317C2
:101350009400B24022449244410182800504130566
:10136000803E420497000000E78000FD4180C5B741
:101370009305000273A04580824573901534924016
:101380002242B2424243D2436244F2440255925551
:101390002256B2564257D2576258F25806499649D9
:1013A000264AB64A464BD64B664CF64C065D965DD1
:1013B000265EB65E465FD65F09617300203041113C
:1013C000B7170040985F3AC6945F3247E39CE6FE49
:1013D000324541018280B71700401307000323887C
:1013E000E7028547171700002322F74673002030D5
:1013F000411122C406C637040020976000E0E78050
:10140000C02C1C408297976000E0E780002CF5B765
:1014100037370040834747009146BD8B639ED70214
:10142000B73600401306F00F973500009385051F6F
:101430009737000083D7872E03C7A6001377F70FCF
:101440001DE3B7E70400BC4F0946894517150000A6
:10145000034585F7829731A099466394D700834767
:1014600057007300203003C786001377F70FE3653A
:10147000F6FC13851700AE97173800002310A82A32
:101480002380E70075B7B787004003C76700098B63
:101490006309071003C77700930600031377070358
:1014A000630DD70817380000034818771736000077
:1014B000130686730547B30606012380E60083C53D
:1014C00077001737000013072774429793F5F50F3D
:1014D0002300B70003C58700973500009385C571C9
:1014E000C2951375F50F2380A500034707008945B2
:1014F0001377F703630CB70C63E7E50A6306071A73
:101500008545630CB7129737000083C7F770330720
:10151000F600034707001377F70F19CB850793F7FA
:10152000F70F3D476363F71A17370000A306F76EFE
:10153000B787004009472383E700B787004083C788
:101540007700E207E18763DE07049737000083C76F
:10155000B76C17370000130727693E9785462300AD
:10156000D700173700001307276A3E97930600033A
:101570002300D70017370000130707683E97A146DE
:1015800085072300D70093F7F70F3D476364F714EF
:1015900017370000A302F768B78700400947238385
:1015A000E70073002030930610026300D70E930605
:1015B00020026305D70693060002E316D7F403C79B
:1015C00027021377C70F13672700D5A803C7670043
:1015D0001377070465CB03C7A70217380000130869
:1015E000284217350000130565391347070823857E
:1015F000E70203C7A7021377370F13678700238516
:10160000E702814713070004B305F5008C41B306D8
:10161000F80091078CC2E399E7FEF5B503C7A7026E
:10162000134707042385E70203C7A7021377C70FF1
:10163000136727002385E702F9B503C7670013770F
:10164000070449C303C76702173800001308082FAF
:101650001735000013054526134707082383E702C3
:1016600003C767021377370F136787002383E702E7
:10167000814713070004B305F5008C41B306F80059
:1016800091078CC2E399E7FEBDBD03C7670213470C
:1016900007042383E70203C767021377C70F1367A3
:1016A00027002383E70285B503C767001377070484
:1016B00011CB03C727021377370F136787002381E6
:1016C000E70291B5238006003DBD97370000A38552
:1016D0000754B9BD97370000A380075475BD230395
:1016E000048015472303E48001002302A480828044
:1016F00083076480E3CE07FE230304808280830790
:101700006480E3CE07FE03454480828083076480C3
:10171000E3CE07FE2302A4808280411126C44AC280
:101720004EC006C61377F50BAD47AA892E8995449E
:10173000630CF700194597000000E78080FA9700D6
:101740000000E78020FB8D444E8597000000E78075
:1017500040F9FD59FD1463983401B240A244124986
:10176000824941018280135509011375F50F9700D5
:101770000000E780E0F92209F1BF011126CC06CE76
:10178000B704080097000000E780C0F615459700F1
:101790000000E78000F597000000E78080F69700E2
:1017A0000000E78000F62AC697000000E78080F47A
:1017B00032459377150089EB136515001375F50F06
:1017C000F240E24405618280FD14E9F00145CDBF9D
:1017D000397126DC4ADA4ED852D656D45AD25ED067
:1017E00006DE62CE66CCB7E700E07D5783AA07002D
:1017F00022C603AA470023A0E71823A2E718B717B9
:101800000040130770052380E704130780FA238044
:10181000E70483C74704930B75FFB684E20793FB85
:10182000FB0F8546AA892E8B328937240040E18739
:10183000015763FA76016308D50089461307000251
:101840006313D5000157D98F93F7F70FB71C0040EA
:101850002382FC0411472303E4801305F00F970053
:101860000000E78000E8094C97000000E78080E86E
:1018700063657C15B7050700DA953787070079554A
:1018800063FEE504B3879500636AF704370B08002D
:10189000A94733EB65016395F90881E88144970016
:1018A0000000E78020E5268515A8DA850945970020
:1018B0000000E780C0E605090345F9FFFD14050BAC
:1018C00097000000E780C0E481C49377FB0FE5F741
:1018D00097000000E780A0EA69F17D55B717004046
:1018E000130770052380E704130780FA2380E704B9
:1018F00003C74704418B2382E704F250B7E700E0B7
:1019000023A0571123A24711E25432445259C2591D
:10191000325AA25A125B825B724CE24C2161828085
:10192000A547639BF90685691309F00FB306990073
:10193000B3742B01B6941349F9FFB3749900856B06
:1019400033796901416B9387F9FFB3F7270199E375
:1019500063FC340193D94900C147E3E637FF3DBF3B
:101960000569C1697D19D9B71305800D63886901BF
:10197000130500026384790113051008CA859700D6
:101980000000E780C0D997000000E78040DF31D534
:101990004E99B38434416DBFDA852D459700000020
:1019A000E780E0D7CA94E30B99EE050997000000A1
:1019B000E78020D5A30FA9FEFDB79387F9FF93F722
:1019C000F70F636DFC0C83C71C0413073008631505
:1019D000F706370708006361EB06B3079B00B706FD
:1019E000100063FBD704334BEB0089476399F9067A
:1019F0008980D549E38404EADA8509459700000027
:101A0000E780E0D111090327C9FF91472320E48033
:101A100003076480E34E07FE23033481FD17EDFBCB
:101A2000FD14110B81C49377FB0FE9FF97000000B1
:101A3000E780E0D461F155B5B717004003C75704FC
:101A4000B70708001377070219E3B787070079552E
:101A5000E376FBE833079B00E3F9E7F841B58547F8
:101A6000E380F9F0DA852D4597000000E78020CB70
:101A70009389F4FFE38404E297000000E78060C8E4
:101A800093F7390091EB832604800327090093071D
:101A90004900E396E6E03E89CE84D9BFB547639915
:101AA000F9001305900B97000000E78080C3FDB399
:101AB000B1471305B00AE388F9FE99476397F90423
:101AC000B7050800B365BB002D4597000000E7800F
:101AD00000C581448D4BA14997000000E78060C29A
:101AE00063967401832704802320F9008504E3951D
:101AF00034FF8327048013172B016355070023123B
:101B0000F90069BB2322F90051BB9D47639FF9028D
:101B100081451305B00497000000E78040C0BD4434
:101B20002320090023220900FD5997000000E780C7
:101B300040BD93F77400CA9703C70700FD14398DA1
:101B40002380A700E39334FF91BBA1476397F90675
:101B500097000000E780A0C28144630D0B008D4711
:101B60009304C0036308FB009304000563048B0126
:101B7000930440041375C507E30295D219459700F5
:101B80000000E78000B697000000E780A0B605459A
:101B900097000000E780E0B4268597000000E7800A
:101BA00020B7094597000000E78080B69700000045
:101BB000E780E0BCE31405CE0DB39147639FF900C5
:101BC0001305600697000000E780A0B197000000B1
:101BD000E78040B213059009F9B5E38109CCF154CF
:101BE0007DB9BD660147173600001306662093864F
:101BF00006A685458347060093F7F70F91C38280B9
:101C00000507E3F9E6FE973700002383B71EDDB72B
:101C10007D166206618693178601E18763D407000B
:101C200001458280931726003307F500AE971843CD
:101C30009C4363E7E7007D16E37FF7FC7D558280D8
:101C400005458280FD15E205E185139785016187D1
:101C500093F7F50F63480700FD15139725002A97A2
:101C6000584365D713851700620561858280330864
:101C7000B5021C4283A80600B335B502C29733B53E
:101C80000701AE98469585486367B5006394A50043
:101C900063E3070181480C43C6950CC388C21CC28C
:101CA000828081471397870161876343B7008280F1
:101CB000139727002A97232007008507E5B7814758
:101CC000014793968701E18663C5B6001335170077
:101CD000828093962700AA9694428507558FD5B7A0
:101CE00093D755408A07AA979C4305453315B500FD
:101CF0007D8D828017F3FFDFE702A33D2A849700E2
:101D00000000E78060F405C5931725003E94032783
:101D1000C4FF814711EB7D1516053E9542054185AF
:101D200017F3FFDF6700233D05838507E5B701450E
:101D3000C5BF81471397870161876343C7008280CE
:101D400013972700B386E50094422A97850714C3AA
:101D5000D5B77D1662066186014793178601E18734
:101D600063D5070013351700828093172600B3064A
:101D7000F500AE9794429C437D16B58F5D8FF1BF01
:101D80008A05AA9501476363B500828083A6C5FFD3
:101D9000F11593D71600D98F9CC11397F601E5B7BB
:101DA0002A830148014701456343D7008280B387F6
:101DB000050183A80700B30706019C43C697AA97AD
:101DC0006384F80033B517010507B3080301620700
:101DD00023A0F80061871108C1BF2A83014781470A
:101DE000014563C3D70082803388E500832808005B
:101DF000330EE600032E0E003388A8403308C84196
:101E00006384080133B508018507B308E300E207DE
:101E100023A00801E1871107E9B717F3FFDFE70205
:101E2000432B0111B286B2842E86AA850A859700BB
:101E30000000E780C0FA2A84A6850A859700000082
:101E4000E78020E833348000060413351500018D47
:101E5000056117F3FFDF6700032A17F3FFDFE702CF
:101E6000C3244111AA89AE8A328BB68402C202C44D
:101E700002C60144131C8401135C8C4163499C021B
:101E8000939B1400FD1B0549138CF4FFF15C330494
:101E90008901620461846340740792478E04CE9482
:101EA00023AEF4FE410117F3FFDF6700832313190C
:101EB0002400B30B2B01014A93172A00D69783A560
:101EC0000B00884378003400500097000000E78042
:101ED00040DA050A93178A01E187F11BE35EFCFCF7
:101EE00092474E9905042320F900A2473EC2B2470B
:101EF00002C63EC441B7131A8901135A8A41131D01
:101F0000240093178A01E18763CF970092470A0460
:101F10004E941CC0A24705091379F90F3EC2B2477F
:101F200002C63EC4ADB7B3079A0313152A005695EF
:101F30000841780034005000050AEA97DA978C438C
:101F400097000000E780E0D26DBF0000197106C263
:101F500012C416C61AC81ECA22CC26CE2AD02ED229
:101F600032D436D63AD83EDA42DC46DECAC0CEC2D9
:101F7000D2C4D6C6DAC8DECAE2CCE6CEEAD0EED209
:101F8000F2D4F6D6FAD8FEDA971500009385858B41
:101F90008841E700050092402242B2424243D243C8
:101FA0006244F244025592552256B2564257D257D5
:101FB0006258F25806499649264AB64A464BD64BCD
:101FC000664CF64C065D965D265EB65E465FD65F55
:101FD0000961730020300000972100209381810265
:101FE000175100201301018217F5FFFF1305C501EA
:101FF0009705002093850501171600201306C6FDDE
:1020000063FAC5008322050023A055001105910540
:10201000E3EAC5FE170502001305053097150020F9
:102020009385C5FB171600201306466563FAC500A5
:102030008322050023A0550011059105E3EAC5FEA2
:102040001715002013058563974500209385052605
:102050006377B500232005001105E36DB5FEFD4251
:10206000739002BC8D4273904280B722000093822D
:10207000828873900230970200209382A2F893E244
:10208000320073905230975200009382C29F739037
:1020900012346FB0F47673002030397101436EC68C
:1020A00019A0397141536AC866CA62CC5ECE19A0C4
:1020B000397101535AD056D252D44ED64AD826DA64
:1020C00022DC06DE33016140828241114AC026C211
:1020D00022C406C68282B24D4101024D924C224C6E
:1020E000B24B4101024B924A224AB2494101024994
:1020F00092442244B240410182803D432A87637367
:10210000C3029377F700BDEFADE5937606FF3D8AF6
:10211000BA960CC34CC30CC74CC74107E36BD7FE40
:1021200011E28280B306C3408A06970200009696A9
:102130006780A6002307B700A306B7002306B700F1
:10214000A305B7002305B700A304B7002304B70015
:10215000A303B7002303B700A302B7002302B7000D
:10216000A301B7002301B700A300B7002300B70005
:10217000828093F5F50F93968500D58D9396050192
:10218000D58D61B7939627009702000096968682B8
:10219000E78086FA9680C1171D8F3E96E374C3F8D8
:1021A000A5B73367B500FD530D8B79E7B7877F7F00
:1021B0009387F7F710419441B372F6003363F6004A
:1021C000BE92B3E262006397720C6318D606504168
:1021D000D441B372F6003363F600BE92B3E26200FC
:1021E0006398720A631BD60410459445B372F600D7
:1021F0003363F600BE92B3E262006391720A631E1B
:10220000D6025045D445B372F6003363F600BE9251
:10221000B3E26200639A72086311D60210499449CE
:10222000B372F6003363F600BE92B3E262006393CA
:1022300072085105D105E30FD6F6131706019397DF
:102240000601631CF7001357060193D706013305F7
:10225000F7409375F50F91E982804183C18333057F
:10226000F7409375F50F91E182801377F70F93F79D
:10227000F70F3305F74082800346050083C605004B
:10228000050585056313D60065FA3305D6408280BF
:1022900011059105E312D6FE014582802105A105B5
:1022A000E31CD6FC014582803105B105E316D6FC5E
:1022B000014582804105C105E310D6FC01458280BD
:1022C000B717004003C777051377E70FA38BE70421
:1022D000130700F8A38DE7043D47238CE704130799
:1022E0005003A38CE70403C7A7051377D70F238DEB
:1022F000E7048280B717004003C7E7020D89411148
:102300001377C70F498F93068008F3B6068093F6BC
:10231000860836C601000100930670052380D704A5
:10232000930680FA2380D704010001002387E70287
:1023300023800704B247F3A7078001000100410191
:10234000828041112A83014E930E407E130F0019A3
:10235000930F400663E56E129308001913034006BD
:10236000B3781503854E0D4FA14F337365020D8968
:102370001335150063EFBE121308F6FF7946729805
:102380004208135808013307C70213D61700BE07C7
:1023900032976146B3F6C60213068070B386C60252
:1023A0003697A166F58F42075D8FB716004083C749
:1023B000F60293F70708A303F1000346710083C7F1
:1023C000F60293F70708E394C7FE83477100B71638
:1023D000004093F7F70F6388071293078008F3B75D
:1023E000078093F787083EC401000100B71700403B
:1023F000930670052380D704930680FA2380D704C0
:102400000100010023AA070383C6170393E6060809
:10241000A388D70223800704A247F3A707800100FF
:1024200001001166B71700407D16D45BC85F938525
:102430004703A98EF18EF5FA93068008F3B606805D
:1024400093F6860836C601000100930670052380C6
:10245000D704930680FA2380D7040100010098C1B5
:1024600003C7170313670704A388E7022380070441
:10247000B247F3A7078001000100410182807D136C
:102480003368E3039308E016630E08003368F30330
:102490009308D016630808009378330093B81800A7
:1024A0009388D81633081E01131E0801135E0E010F
:1024B00055B56393E5030548638608000148630347
:1024C00003002A8871087298FD15131E0801C205C1
:1024D000135E0E01C18179BD13F8150063F4BF00CE
:1024E0007908D5B713381800E5BF83C7F60293F70C
:1024F0000708A303F1000346710083C7F60293F7B0
:102500000708E394C7FE8347710093F7F70FF1DFE5
:10251000E9B531714AD966CB06DF22DD26DB4ED71D
:1025200052D556D35AD15ECF62CD6AC96EC7AA8C36
:1025300002D897100000E78020B12A89930780080D
:10254000F3B7078093F787083EDA01000100B71759
:102550000040130770052380E704130780FA2380E7
:10256000E7040100010003C7F7021377770FA38781
:10257000E70203C7F70213678700A387E7022380F8
:102580000704D257F3A70780010001000545970013
:102590000000E78060D6130780C13347E902116A63
:1025A00093070AE893065002BD69930BA004814A81
:1025B000014B13048008930470057D1AB347F90298
:1025C0003307D7023EC0FD873ECC938709A6930907
:1025D000803E3347F7023AC27D873AC43347390316
:1025E0008549B399990193D93940B306D702B30B02
:1025F0007703B3C6F602B3CBFB0236C6FD8636C8F8
:1026000093D6FB4136CEB7460F0093860624334956
:10261000D9028566938606FAB3969601B389E902D4
:10262000130760553309D90293060010B389E902F4
:102630003349D902B3C9F9029316390036CA37199A
:102640000040FD8636D0930D090493D7F9413ED260
:10265000F336048093F6860836DC01000100930708
:1026600070052380FD00930680FA2380DD000100C1
:1026700001008346390593F6860FA309D9048346E2
:10268000390593E61600A309D90423800D00E2560C
:10269000F3A6068001000100130C80FA116DF336D9
:1026A000048093F6860836DE01000100930770056A
:1026B0002380FD0023808D01010001008346390540
:1026C000216693E60602A309D90483560905B3E6F9
:1026D000A6012318D90483560905D18E2318D904DD
:1026E00023800D00F256F3A6068001000100834608
:1026F000390593F606026381061A03463905218AD5
:102700006DDE081897100000E7800098733604808B
:1027100013768608B2C20100010023809D00238049
:102720008D0101000100B717004003C6370513767D
:10273000F60DA389C70403C6370513660602A389ED
:10274000C704835609052166B3E6A6012318D904F8
:1027500083560905D18E2318D90423800D0096468F
:10276000F3A60680010001008346390593F60602B0
:10277000638B061483463905A18AEDFE970000207D
:10278000E7806091AA8636D497000020E780A09069
:10279000A256E30AD5FE835609054255B3E6A601C3
:1027A0002318D90497100000E780C08F83463905AD
:1027B000A18AEDDE03560905834629058247337653
:1027C000CA00B306DA0293D5F641B296B388F64052
:1027D000E24733B8C6002E983308F840A247B3B694
:1027E00016013308D84063C70701631DF8009247FC
:1027F00063FA1701C247634FF80E63950701B247AA
:1028000063EAF80E894663E9660FF24693151800ED
:1028100013D3F8015E8613951800B365B30042D652
:1028200046D497C00100E78060CC3258050B137B7B
:10283000FB0F63470001631A0838A2586387083802
:1028400013081500B336A800B69513D6F5013298D3
:10285000B336C800AE9613581800FE06B3E606015C
:102860007336048013768608B2C601000100238007
:102870009D0023808D01010001000356C902B2961C
:10288000C206C1822316D90223800D00B646F3A6E4
:1028900006800100010021B5F336048093F6860816
:1028A000B6C00100010023809D0023808D0101003E
:1028B00001008346390593E60602A309D904238063
:1028C0000D0086460DB5F336048093F68608B6C42F
:1028D0000100010023809D0023808D010100010083
:1028E0008346390593E60602A309D90423800D0027
:1028F000A646BDB5E30B0BF0F336048093F68608CD
:10290000B6C801000100930680FA23809D00238051
:10291000DD00010001008346390593F5FC0F93F6B5
:10292000860FA309D90483463905CD8EA309D9049E
:1029300023800D00C646F3A60680010001001305A2
:1029400080FA03463905930639051D8A631C9629CA
:102950007336048013768608B2CC0100010013069A
:1029600080FA23809D002380CD000100010003C672
:1029700006001376F60D2380C60003C60600136614
:1029800006022380C600835609051166D18E2318DE
:10299000D904835609052166D18E2318D9042380D2
:1029A0000D00E646F3A6068001000100130680FA3A
:1029B0008346390593F60602638006268346390569
:1029C000130C3905A18AFDDA081897000000E7808A
:1029D000A06BF336048093F68608B6D001000100A0
:1029E000930680FA23809D002380DD000100010012
:1029F00083460C00116693F6F60D2300DC00834637
:102A00000C0093E606022300DC0083560905D18EF4
:102A10002318D904835609052166D18E2318D904B9
:102A200023800D008656F3A60680010001001306E0
:102A300080FA8346390593F60602638A06208346A8
:102A40003905A18AEDFE97F0FF1FE780C0642A8C4C
:102A500097F0FF1FE7802064E30C85FF835609058C
:102A600011664255D18E2318D90497000000E780E3
:102A700060638346390513063905A18AFDDAF3360A
:102A8000048093F68608B6D401000100930680FA0C
:102A900023809D002380DD000100010083460600A5
:102AA00093F6F60D2300D60023800D00A656F3A65C
:102AB0000680010001008356090503462905D24717
:102AC000B376DA003306CA021305800C9355F6413B
:102AD0003696330DF6408257333CD6002E9C333663
:102AE000A601330CFC40330CCC40330885039256CE
:102AF0004E86B335A5033305A503C29597C00100E3
:102B0000E780C09E63468001631E0C16630C0D16A1
:102B1000130615003335A6002E959356F50136960B
:102B2000B335D600AA959396F50105828585D18E99
:102B30006346B000639D051A638B061A0356C902EB
:102B400015823305D6003336C500B2956348B00010
:102B5000639105241306F00F637DA622894663F373
:102B6000561593078008F3B7078093F78708BED6FA
:102B70000100010037170040930770052300F70498
:102B8000930780FA2300F704010001008356C7026F
:102B900089678117D58FC207C1832316F7022300E7
:102BA0000704B657F3A7078001000100FA506A54E2
:102BB000DA544A59BA592A5A9A5A0A5BFA4B6A4C59
:102BC000DA4C4A4DBA4D296182801308F5FF33353E
:102BD000A800FD152E951356F5013298B336C8009E
:102BE000AA9695B9F336048093F68608B6CA010012
:102BF000010023809D002380AD0001000100834679
:102C00003905CD8EA309D90423800D00D646F3A63D
:102C100006800100010035B3F336048093F6860880
:102C2000B6CE0100010023809D002380CD0001006D
:102C300001008346390593E60602A309D9042380DF
:102C40000D00F646F3A606800100010095B3F336A9
:102C5000048093F68608B6D20100010023809D000F
:102C60002380CD00010001008346390593E606026A
:102C7000A309D90423800D009656F3A6068001000F
:102C8000010045BB9306F5FF33B5A600FD152E9553
:102C90009355F501AE96B3B5B600AA951396F50116
:102CA000858269B5F336048093F68608B6D80100AC
:102CB0000100930680FA23809D002380DD0001003F
:102CC00001008356C9020566011693F6F60FD18EF0
:102CD000C206C1822316D90223800D00C656F3A670
:102CE000068001000100850A93FAFA0F95B233E6D7
:102CF000B60045C20356C9023305D0403338A000A0
:102D0000B305B040B385054115826345B000D1E1FC
:102D10006371A608894663F0560593078008F3B7E8
:102D2000078093F78708BEDA01000100B71700405B
:102D3000130770052380E704130780FA2380E70454
:102D40000100010003D7C7027D8B2396E702238091
:102D50000704D65781BDF336048093F68608B6DCA7
:102D600001000100930680FA23809D002380DD008E
:102D7000010001008356C9020566011693F6F60F9D
:102D8000D18EC206C1822316D90223800D00E656D9
:102D9000B9B793078008F3B7078093F78708BEDEBB
:102DA0000100010037170040930770052300F70466
:102DB000930780FA2300F704010001000356C702BD
:102DC00093975600B297C207C1832316F7022300D8
:102DD0000704F657C1BB914763EEB70217D701004E
:102DE0001307475C8A05BA959C41BA978287B71743
:102DF000004003A7470B1345F5FF698F23AAE70A95
:102E000003A7070B698F23A8E70A03A7070A798D91
:102E100023A0A70A8280B717004083A6470B134759
:102E2000F5FFF98E23AAD70A83A6070B558D23A891
:102E3000A70A83A6070A758F23A0E70A8280B7171F
:102E4000004003A7470B498F23AAE70A03A7070BF4
:102E50001345F5FF45BFB717004083A6470B13473F
:102E6000F5FF758F23AAE70A03A7070A598D4DB707
:102E7000B717004003A7470B498FEDB7914763EEA3
:102E8000B70217D70100130727538A05BA959C414B
:102E9000BA978287B717004003A7470D1345F5FF80
:102EA000698F23AAE70C03A7070D698F23A8E70CF6
:102EB00003A7070C798D23A0A70C8280B7170040C9
:102EC00083A6470D1347F5FFF98E23AAD70C83A6D7
:102ED000070D558D23A8A70C83A6070C758F23A07B
:102EE000E70C8280B717004003A7470D498F23AA3C
:102EF000E70C03A7070D1345F5FF45BFB7170040C3
:102F000083A6470D1347F5FF758F23AAE70C03A788
:102F1000070C598D4DB7B717004003A7470D498FD0
:102F2000EDB7797122D43714004026D24AD0035924
:102F300024028354040206D64209C2044ECE52CC67
:102F400056CA13590901C1802DE11379F9F793F499
:102F5000F49F4209C20413590901C18093078008F4
:102F6000F3B7078093F787083EC401000100930779
:102F700070052300F404930780FA2300F404010091
:102F80000100231124032310940223000404A24708
:102F9000F3A7078001000100B25022549254025955
:102FA000F249624AD24A45618280B7F507008146FC
:102FB0003000B105194597000020E7806081A247E5
:102FC00013972701E34A07FC1369090893E40440B7
:102FD00093098008F3B7098093F787083EC0010082
:102FE0000100930A700523005405130A80FA230098
:102FF000440501000100231124032310940223003F
:1030000004048247F3A7078001000100294597F0D7
:10301000FF1FE7802032F3B9098093F989084EC277
:1030200001000100230054052300440501000100B4
:103030008357040293E707202310F40223000404BB
:103040009247B9B7B7170040884742054181937747
:10305000050491EB9377F5013755E80113050580D9
:103060003345F50282809377050C130700046397BC
:10307000E7009377F50137459C1CCDB72165130513
:1030800005D0828037E700E01C435443A183E20669
:10309000D58F1CC1FD572320F7182322F7188280F3
:1030A00013178500B7E700E023A0E710618123A292
:1030B000A7108280B7F700E08847CC47828081471D
:1030C00037370040A14663C4C7003285828003457C
:1030D000B740E38EA6FE3385F5000345050085075E
:1030E0002304A740CDB797070020938727EF9C4381
:1030F000173700201307871B3E95636EE5001737CF
:103100000020130727506368A70017070020232714
:10311000A7EC3E858280FD57EDBF8280411122C41D
:1031200006C62A8497000000E78000F22947B3070B
:10313000E502B2408D83B3D7870222449507B3D707
:10314000E70237370040C207C1832316F700410169
:103150008280411137150E0006C697000000E780F7
:1031600020FCB7370040130770F82381E7000D47B4
:10317000A381E70013070004A380E7000547238726
:10318000E700B24041018280373700408347270083
:103190001A0593F7F703C98F93F7F70F2301F70089
:1031A0008280B737004003C7170019C9D98DA380A3
:1031B000B70003C70700136787002380E7008280FA
:1031C00093C5F5FFF98DA380B7008280AE872A876B
:1031D000B736004021463738004089E71703000022
:1031E0006700E3F383C8B600E30916FF05078348C9
:1031F000F7FFFD17C20723041801C183F9BF41116E
:1032000022C406C62A8497000000E780E0E329472D
:10321000B307E502B2408D83B3D7870222449507F6
:10322000B3D7E70237370040C207C1832316F74000
:1032300041018280716541111305052006C6970082
:103240000000E78000FCB7370040130770F82381C7
:10325000E7400D47A381E74013070004A380E74040
:1032600005472387E740B24041018280CC414111AC
:1032700006C6328503C6150083C5050022064D8E9D
:1032800042068D654186138875A2630C0611634B57
:10329000C804138845A26300060D634AC8009385DD
:1032A00035A26301B6082390060029464DA0138875
:1032B00055A26305060D938565A2E316B6FE8D45FE
:1032C0001D4663E6E5081146198E63F3C7003E8686
:1032D000B7E704002390C600FC4797D5010093850B
:1032E000E50F9DA0138895A263030611634E060D9A
:1032F0001388A5A263000613938505A5E315B6FA06
:1033000099451D4663E5E504198E63F3C7003E86C3
:10331000B7E704002390C600FC479705002093857B
:1033200025D61DA09D451D4663E3E5022146198E65
:1033300063F3C7003E86B7E70400FC472390C6004E
:103340009705002093850534BA9582970146B240CF
:10335000328541018280AD451D46E3EAE5FE3146F6
:10336000198E63F3C7003E86B7E704002390C600BA
:10337000FC4797D501009385E508F9B7B1451D468F
:10338000E3E7E5FC3546198E63F3C7003E86B7E7F1
:1033900004002390C600FC4797D50100938585075C
:1033A00065B78D451D46E3E4E5FA1146198E63F3D2
:1033B000C7003E86B7E704002390C600FC4797D5B8
:1033C00001009385650249B78D451D46E3E1E5F8A7
:1033D0001146198E63F3C7003E86B7E704002390B9
:1033E000C600FC4797D5010093858504B1BFA5456C
:1033F0001D46E3EEE5F42946198E63F3C7003E86C9
:10340000B7E704002390C600FC4797D501009385D9
:1034100065FE1DBFB5451D46E3EBE5F23946198E45
:1034200063F3C7003E86B7E704002390C600FC475D
:1034300097D50100938585F901BFB7E7040003A381
:103440000713970600209386A6C24146A545170597
:1034500000201305E5B802832D455DE703C505008F
:103460000947631FE50803A84500411106C6034745
:10347000180032850346080022074168518F9308DF
:1034800028FE6307170563E9E800051863030703CF
:1034900023900600294591A8130648FE630AC70435
:1034A0001518E31707FF15463E87637BF60015479F
:1034B00001A8130600023E876374F600130700029A
:1034C000B7E704002390E600FC471316070111A894
:1034D0003E8691C30546B7E70400FC472390C6002B
:1034E0004206CC45418282970145B240410182802B
:1034F000130600083E87E375F6FC13070008C9B7FA
:103500002390060005458280828041677917630415
:10351000E504411122C406C685472A84639FF5004D
:10352000B7E7040022852244B24003A3871397051E
:1035300000209385652F4101028389476399F50037
:10354000B7E7040083A7070B8545829771D9B2407E
:103550002244410182808280797126D252CCAE848D
:103560002A8A97D501009385A5EE17D5010013058A
:10357000A5F006D63AC622D44AD0368432894ECE39
:1035800097B00100E780C041A28517D5010013055F
:10359000A5EF97B00100E780A040294597B0010052
:1035A000E780E04483C7840093F70702F9E383C907
:1035B00004008947054532476396F908D44083C71C
:1035C000160083C60600A207D58FC166138616FEB5
:1035D000638CC7028D16638FD7068D6693862690FF
:1035E00029456391D706B7E70400A286225403A3B6
:1035F0004714B250F2494A86A68502599254528520
:10360000624A8547456102832D450DEF930700020D
:10361000354563E98702B7E70400FC47C844130651
:103620000002CA85829781499707002093878720E7
:103630009C43014581CB9C4391C74E852286CA8518
:1036400082970145B250225492540259F249624A7B
:10365000456182802D457DF79307700F3545E3E383
:1036600087FEB7E70400FC47C8442286CA858297D4
:1036700065BF2145C1BF411122C437E4040083273F
:10368000841326C2AA84416506C697050020938547
:10369000A5197D1582978327C40A17050000130515
:1036A00005E78588829795C0032304132244B2401E
:1036B000924497060020938626AE4146C5451705DD
:1036C00000201305659C41010283B24022449244CC
:1036D00001454101828019C59707002023ACA7143A
:1036E00001458280454582801147636AA70A97D6C3
:1036F00001009386A6D40A0536951841411106C6E5
:103700003697AE87B2850287130700026145639D35
:10371000E700B7E70400FC47130600021705002086
:103720001305C5F682970145B240410182800547E5
:103730006145E39BE7FEB7E70400FC470546170534
:1037400000201305A5F6F9BF1307700F6145E39D2F
:10375000E7FCB7E70400FC471306700F17050020CD
:10376000130505F5C1B7130700086145E39EE7FAA5
:10377000B7E70400FC4713060008170500201305EF
:10378000A5024DB715476145E390E7FAB7E7040096
:10379000FC471546170500201305450961B7094583
:1037A0008280411126C2B7E4040083A7C41322C457
:1037B0004AC006C62E84970500209385E5062A890F
:1037C0008297058905C5970700209387E78B83D7E4
:1037D000A70BA28503A3440D2310F4002244B2409A
:1037E00092444A850249014641010283B240224483
:1037F0009244024949454101828097070020238D68
:1038000007029707002023AB0702B717004003A762
:10381000070CB706C0FFFD16758F23A0E70C03A7A2
:10382000070DB7064000558F23A8E70C03A7070C28
:103830003D9B23A0E70C03A7070D1367070123A8EF
:10384000E70C8280B717004003A5470C83A7470CFD
:10385000598113451500C18B058999E3136525002E
:103860009707002083C747FD6380A70297070020C2
:103870002384A7FC11C997070020938727FC03A383
:1038800007006303030002838280114517F3FFFFE3
:10389000670063C8411193962500AA852D4506C689
:1038A00097F0FF1FE780C0F2B240014541018280DE
:1038B000011122CC06CE3714004026CA4AC84EC693
:1038C00052C483447405034AB405834984050349FB
:1038D000940597F0FFFFE780E09E8347A40593F4EB
:1038E000F40F137AFA0F93E71700230DF40493F9FA
:1038F000F90F1379F90FB717004003C7A705058B18
:103900006DFF03D5C705A38D4705238C3705A38C11
:103910002705A38B9704F2406244D2444249B2493E
:10392000224A0561828041119397050122C406C68F
:1039300026C2C1872E8463DC0700B7E40400FC5470
:10394000829719C1BC5482972165218D15A893F7E0
:10395000150013C515008DE793F725009DC7970047
:103960000000E78060EEB7E70400BC4F1306000AD2
:103970008945170500200345E5EC8297134524008F
:10398000B24022449244410182809397250163D83A
:103990000702B7E4040083A7C41E829797000000C3
:1039A000E780E0EEBC4C3756070013060630896509
:1039B00017050020034505E98297096579B79397B4
:1039C00015010145E3DE07FA17D501001305C5B35C
:1039D00097B00100E780A014B7E70400BC4F1306BE
:1039E00000649165170500200345C5E582971165C0
:1039F000A9BF2D71232A9110FD74E98C232C81100D
:103A000023282111232631112A84AE893289930675
:103A100000100A86A6852D45232E111097F0FF1F52
:103A2000E78000DB13154401B7E70400FC47518130
:103A30000A0513962900CA850A958297A685856688
:103A40000146254597F0FF1FE78080D80A86A685A6
:103A500093060010294597F0FF1FE78060D7832069
:103A6000C1110324811183244111032901118329E8
:103A7000C11015618280B7F7070003C70701411124
:103A800006C622C426C24AC0A547631DF700970098
:103A90000000E78040F6B2402244924402490145CA
:103AA0004101828013942500AA843289A286AA85C6
:103AB0000146254597F0FF1FE78080D1A2864A8600
:103AC000A685294597F0FF1FE78080D0E9B71D71D3
:103AD000A2CC37E404005C5C485886CE494697D5B2
:103AE00001009385E59D829711E917D50100130523
:103AF000659E97B00100E780800201A0B7F600E064
:103B0000795798CAFD57DCCA0567B7E700E023A0DC
:103B1000E7101306F00290C223A0E718010001008D
:103B20003707002018471306000481459706002038
:103B300023A8E6D04157A38AE7403C44080882976F
:103B4000970700209387076D3EC885671387074056
:103B5000231AE1001D673ACC370701051307071048
:103B60003ACE938757D11307B00F2310E1022312E7
:103B7000F102054797F7FFFF938707542301E102FE
:103B80003ED817070000130727D197070000938737
:103B900067D2B7F50700BAC23EDC1707000013076B
:103BA000C7ED97070000938787CE81463000E10577
:103BB0001945BAC43EDE97F0FF1FE78060C11808C0
:103BC0008147994630003E96034606008507050763
:103BD000A30BC700E398D7FEC24791C70357410123
:103BE00085676373F70001A0B7E7040083A7470A5E
:103BF00008088297AA8511C917D501001305C58E3B
:103C000097B00100E780C0D901A0F6406644256165
:103C10008280411126C2B7E4040083A7040806C6C7
:103C200022C417050000130545D082971704002011
:103C3000130444C12300A40097000000E780800221
:103C400097000000E780A0BB03450400224403A3C3
:103C50008405B24092441306003289654101028313
:103C6000797106D622D413078008F337078093F7BB
:103C700087083EC201000100B71700409305700598
:103C80002380B704130680FA2380C70401000100D3
:103C900083C6F70293F6A60FA387D70223800704F3
:103CA0009246F3A606800100010073370780137760
:103CB00087083AC4010001002380B7042380C704A9
:103CC0000100010003C7F70213672700A387E7027B
:103CD00023800704A247F3A70780010001000545E0
:103CE00097E0FFFFE780406197000000E78020BA7F
:103CF000014781468147054685451305407E97E08B
:103D0000FFFFE780406437E404003C44680051460C
:103D100081458297B707C0A83EC8B787E803938755
:103D200007D03ECA97E7FF1F938767693EC67C5856
:103D300068008297B250225445618280411197D524
:103D400001009385A5E217C501001305E57206C6BB
:103D500097B00100E780C0C417D501001305C5F96D
:103D600097B00100E780C0C3B2402945410117B3B5
:103D700001006700C3C7411197D50100938545E055
:103D800017C501001305456F06C697B00100E7800F
:103D900020C117D501001305E5F497B00100E780B5
:103DA00020C0B2402945410117B30100670023C478
:103DB000411122C406C6834705002A849DC797D5B2
:103DC00001009385A5E117C501001305E56A97B0C9
:103DD0000100E780E0BC4C4017D501001305050049
:103DE00097B00100E780C0BB3DA058410DEF97D5CB
:103DF00001009385A5DE17C501001305E56797B09F
:103E00000100E780E0B917D501001305A5FE97B0C2
:103E10000100E780E0B82244B2402945410117B3D0
:103E200001006700C3BCA1679386D7036313D70261
:103E300097D50100938585DA17C501001305C56381
:103E400097B00100E780C0B517D50100130585FBC9
:103E50007DBFED0797D50100938545D817C50100B3
:103E600013058561631BF70097B00100E78040B33D
:103E700017D50100130545FA59BF97B00100E78037
:103E800020B24C4017D50100130505FB91BF41112D
:103E900097D50100938505D017C501001305C55DB1
:103EA00006C697B00100E780A0AFB24029454101A6
:103EB00017B301006700A3B3797122D426D24AD088
:103EC0002E842A898145B2844800714606D697E03F
:103ED000FFFFE780C02297F7FF1F9387A74CDC47BF
:103EE00083D70700231421012313F100975000000A
:103EF000E78060CB9547A305F1009307401F3EC6BE
:103F0000FD572305A100230AF10097500000E78028
:103F1000C0DD2686A285480097500000E78080CB50
:103F2000B250225492540259456182809717002062
:103F30002395077E97170020238E076CB7E70400B0
:103F4000BC47411106C641468145170500201305AF
:103F5000A51A829797200000E780606297200000F2
:103F6000E780E040014597500000E780A058170720
:103F700000200347671A9307F00A6315F7029307B7
:103F8000F0F88945170500201305051917070020CB
:103F90002304F71897070020A38007189750000004
:103FA000E780E07F97600000E78040AC81453705FF
:103FB00004009707002023AF0712970700202399DA
:103FC00007129707002023860712970700202397E0
:103FD000070A9707002023950708970700202398D2
:103FE0000710970700202391071297300000E78001
:103FF000C00E014597600000E780608397D50100FF
:104000009385C5BB17C501001305054797B001008F
:10401000E780009917D50100130545E897B0010026
:10402000E7800098B2402945410117B301006700BD
:10403000039C411122C406C626C293F715002E84A4
:10404000638F0710814617F6FF1F1306E63285457A
:10405000170500200355850097C00000E780000683
:1040600015C997D50100938525B617C5010013051D
:10407000A54097B00100E780A09217C50100130585
:10408000655797B00100E780A091294597B00100DE
:10409000E780E09597D50100938505B317C501002A
:1040A0001305853D97B00100E780808F17C501009B
:1040B0001305855597B00100E780808E294597B09C
:1040C0000100E780C09217F5FF1F1305A52D5C4581
:1040D00005472390E70097400100E78080B697D519
:1040E0000100938565AE17C501001305E53897B04B
:1040F0000100E780E08A17C501001305255297B03B
:104100000100E780E089294597B00100E780208E13
:10411000930710F8170700202300F70097070020E7
:1041200083D787F317070020A308F7FE17050020A1
:10413000130585FEA183914517070020230FF7FC87
:1041400097070020A38B07FC97500000E7802065AD
:1041500013451400B240224492444101828093F7F7
:104160002500E1C317070020035787F845CB9706C2
:104170000020938626F8944297D70100938707D4AE
:10418000170600200346E6F68145170500201305B3
:10419000A5F697700000E780C011AA8441C197D5A9
:1041A0000100938525A917C501001305E52C97A0EB
:1041B0000100E780E07EA68517C50100130585474D
:1041C00097A00100E780C07D294597B00100E780F6
:1041D000008297070020239D07F0930710F8170728
:1041E0000020230BF7F29707002083D7E7E6170795
:1041F0000020A303F7F2A18317070020230FF7F095
:1042000091458D4717050020130505F1170700207C
:10421000A305F7F097500000E7806058134524008D
:1042200015BF93F74500D1C397D50100938585A0AD
:1042300017C501001305452497A00100E7804076CB
:1042400017C501001305C54097A00100E780407520
:10425000294597A00100E7808079930720F8170788
:104260000020230BF7EA9707002083D727E11707E1
:104270000020A303F7EAA18317070020230FF7E824
:10428000854717070020A30AF7E897500000E7804A
:10429000C0A517050020130525E89145975000009B
:1042A000E780E04F1345440075B593F78500A9C733
:1042B00097D501009385059817C501001305C51B07
:1042C00097A00100E780C06D17C50100130585396F
:1042D00097A00100E780C06C294597A00100E78006
:1042E000007197070020239507E097700000E78092
:1042F000200C13458400B9BD93F70501D1C3854552
:1043000017050020035585D797600100E78040BE60
:1043100097D501009385059217C501001305C515B2
:1043200097A00100E780C06717C501001305C534D9
:1043300097A00100E780C066294597A00100E780AB
:10434000006B930730F8170700202307F7DC970767
:10435000002083D7A7D217070020A30FF7DA17058D
:104360000020130565DBA1838D4517070020230678
:10437000F7DA97500000E780804213450401D9BB6B
:1043800093F70502D1C797D501009385A58A17C574
:1043900001001305650E97A00100E780606017C556
:1043A00001001305A52F97A00100E780605F294554
:1043B00097A00100E780A063930740F8170700204B
:1043C000230CF7D49707002083D787C9170700204D
:1043D000A304F7D4A183170700202300F7D485474F
:1043E00017070020A30BF7D297070020239A07C6D0
:1043F00097500000E780608F170500201305C5D196
:10440000914597500000E78080391345040299B325
:1044100093F70504FDC397D501009385A58117C5C2
:1044200001001305650597A00100E780605717C5D7
:1044300001001305252897A00100E7806056294553
:1044400097A00100E780A05A9707002083C7C7CC38
:104450001307700A6386E7061307800A638CE70870
:104460001307600A6393E704930760F817070020B7
:104470002304F7CA9707002083D767C717070020D0
:10448000A30CF7C8A183170700202308F7C88547A6
:1044900017070020A307F7C8B1451705002013052B
:1044A000A5C797500000E780802F97500000E78055
:1044B000C0831345040497070020239A07C259B903
:1044C000930770F8170700202308F7C49707002008
:1044D00083D7E7C117070020A300F7C4A1831707FC
:1044E0000020230CF7C2854717070020A308F7C256
:1044F000994565B7930780F8F1B793F7050801452B
:10450000E38A07C497C501009385C57217C50100EA
:10451000130585F697A00100E780804817C50100C4
:104520001305C51A97A00100E7808047294597A089
:104530000100E780C04B9307A0F817070020230D68
:10454000F7BC9707002083D727BC17070020A305D7
:10455000F7BCA183170700202301F7BC8547170785
:104560000020A30CF7BA97070020239F07B89740B5
:104570000000E7808077170500201305E5B9914515
:1045800097500000E780A02113450408E1B64111CF
:1045900022C497C501009385A5652A8417C501002B
:1045A000130585ED06C697A00100E780603F4C40EB
:1045B00017D501001305058097A00100E780403E54
:1045C000294597A00100E780804203470400930734
:1045D000F00F631FF70297C501009385656117C54A
:1045E0000100130565E997A00100E780603B4C409E
:1045F00017C501001305057D97A00100E780403A2B
:104600002244B2402945410117A301006700233E1F
:10461000B240224441018280B1C1411122C417C578
:104620000100130565E52E8497C501009385455764
:1046300006C697A00100E780A036A28517D5010025
:104640001305858397A00100E78080352244B2409E
:104650002945410117A30100670063398280411198
:1046600022C426C22E84AA8497C5010093850554CE
:1046700017C50100130545E006C697A00100E780B5
:10468000203217C501001305E57F97A00100E780E0
:104690002031294597A00100E780603597C50100CA
:1046A0009385C55097070020239A979A17C5010054
:1046B000130585DC854497070020239F879897077B
:1046C0000020239C9798971700202398870497A091
:1046D0000100E780E02C9715002083D5050417C55D
:1046E00001001305A57A97A00100E780602B2945FA
:1046F00097A00100E780A02F97170020238C97F048
:1047000097200000E780A0C6228597500000E78030
:1047100060DE054597500000E780601197F7FF1FA6
:10472000938747C8DC4703D70700C167FD176312AB
:10473000F7022244B7E70400B240924403A387057E
:1047400017F5FF1F034585101306000A8545410133
:104750000283B2402244924441018280011122CC62
:1047600037E404005C5C06CE354697C501009385AE
:10477000E55917D501001305E51F829711E917C503
:104780000100130525D597A00100E780403901A05D
:1047900097F7FF1F9387470C3EC4B7F5070085675F
:1047A00093870780814617F6FF1F1306660AE10507
:1047B00019453EC697E0FF1FE78080017C441946FB
:1047C00097F5FF1F9385C508170500201305458B36
:1047D0008297340017F6FF1F1306860797D501004E
:1047E000938505A417D50100130505A59770000052
:1047F000E78020812A841DCD97C5010093858542DD
:1048000017C50100130545C797A00100E7804019AF
:10481000A28517C501001305655097A00100E78028
:104820002018294597A00100E780601CF2406244EF
:104830000561828097E00000E78080E317C50100F2
:104840001305C54497500000E780607597A00000ED
:10485000E780C03797600100E780409C17F5FF1F95
:104860001305C5B097600100E780E08417C501001B
:104870001305C54297600100E780C09C2A849760B9
:104880000000E780A0DB97000100E780207497809C
:104890000100E780400D97700000E780E0339760EB
:1048A0000000E780A05197300100E780803597C570
:1048B00001009385253717C501001305E5BB19C80D
:1048C00097A00100E780C00DA28517C50100130560
:1048D0002547A1B797A00100E780800C17C501000C
:1048E0001305454897A00100E780800B294597A054
:1048F0000100E780C00F97300100E780601197F05A
:104900000000E780203055C9854537050400972011
:104910000000E780807C97C501009385A53017C50E
:104920000100130565B597A00100E780600717C572
:1049300001001305A54497A00100E7806006294502
:1049400097A00100E780A00A97F7FF1F938747957C
:1049500083D70700171700202311F7DC85471717A7
:1049600000202309F7CA97200000E780E0B79720CE
:104970000000E780C09F17150020035505DA975007
:104980000000E78020B7054597500000E78020EA47
:1049900097C501009385052917C501001305C5AD0D
:1049A00097A00100E780C0FF17C501001305453F30
:1049B00097A00100E780C0FEADB597C501009385C3
:1049C000652617C50100130525AB97A00100E780F8
:1049D00020FD17C501001305654C97A00100E78075
:1049E00020FC294597A00100E7806000014569BFD0
:1049F000411122C437E404008327041A06C68297B3
:104A000097500000E780C0B28327040817F5FFFF26
:104A100013056562829797F7FF1F2389A7E217F5B1
:104A2000FF1F1305259897400000E780A05E2244F1
:104A3000B240410117030000670083D2B7E70400CA
:104A4000FC471171A2DDCAD986DFA6DBCED72E8442
:104A500032892E86AA8517F5FF1F1305E56B82970D
:104A600017F7FF1F1307476B834707009306800262
:104A70009387E70793F7F70FE3ECF610BA898A07F5
:104A800017C70100130787A8BA979C43BA97828774
:104A90008D4797C501009385251B17C50100130598
:104AA000A59D630FF40097A00100E78060EF17C594
:104AB0000100130525D897A00100E78060EEBDA492
:104AC00097A00100E780C0ED17C50100130505D8C8
:104AD00097A00100E780C0EC294597A00100E7807E
:104AE00000F1930720F8114697F5FF1F9385C562E3
:104AF0004A8517F7FF1F2301F76297F7FF1FA38E61
:104B0000076097F0FFFFE780603B2A841DC997C5C7
:104B100001009385651317C501001305E59597A05E
:104B20000100E780E0E7A28517C501001305C5D5A0
:104B300097A00100E780C0E6294597A00100E78023
:104B400000EB97C501009385251017C501001305DB
:104B5000A59297A00100E780A0E417C50100130506
:104B6000E5D397A00100E780A0E3294597A00100C5
:104B7000E780E0E74165930730FA054697F5FF1FA8
:104B8000938585597D1517F7FF1F2307F75897F071
:104B9000FFFFE780A0322A841DC997C501009385D5
:104BA000A50A17C501001305258D97A00100E78010
:104BB00020DFA28517C50100130505CD97A00100D0
:104BC000E78000DE294597A00100E78040E2B7E7D3
:104BD0000400BC4F0566130606C8A14517F5FF1F64
:104BE0000345C5C68297FE506E54DE544E59BE59D9
:104BF0001161828091476303F40297C50100938598
:104C0000A50417C501001305258797A00100E780BB
:104C100020D917C501001305A5CB71BDB7E7040066
:104C2000FC4F914517F5FF1F034545C2829797C575
:104C300001009385650117C501001305E58397A061
:104C40000100E780E0D517C50100130525CA97A02C
:104C50000100E780E0D4294597A00100E78020D932
:104C600097400000E7806008914535A485476303BD
:104C7000F40297C50100938525FD17B501001305C2
:104C8000A57F97A00100E780A0D117C501001305FB
:104C900065C715B597F7FF1F2392273FB7E70400B5
:104CA0000566BC4F130606C8C1450DBF8D4763039B
:104CB000F40297C50100938525F917B50100130586
:104CC000A57B97A00100E780A0CD17C501001305C3
:104CD00025C5D5B3930740F8114697F5FF1F938577
:104CE000A5434A8517F7FF1F2308F74297F7FF1FD1
:104CF000A385074297F0FFFFE780401C2A84E30466
:104D000005EE97C50100938525F417B5010013053D
:104D1000A57697A00100E780A0C8A28517C501006D
:104D2000130585B697A00100E78080C7294597A0A5
:104D30000100E780C0CB45BD9147E31CF4F6B7E71F
:104D40000400FC4F9305000217F5FF1F034505B053
:104D5000829797C50100938525EF17B501001305CC
:104D6000A57197A00100E780A0C317C50100130536
:104D7000A5BCF1BD894763E3870297C50100938510
:104D8000A5EC17B501001305256F97A00100E7807A
:104D900020C117C50100130565BB31BB97F4FF1F88
:104DA00083C4A43797F7FF1F83C7173797C5010040
:104DB000938585E9A20417B501001305E56BDD8C29
:104DC00097A00100E780C0BDA28517C501001305AB
:104DD00025B997A00100E780A0BCC204294597A08F
:104DE0000100E780C0C0C1849305D4FF93960401FD
:104DF000C1824A8693F5F50F17F5FF1F1305F531AC
:104E000097200000E7802031E35F90DC930750F8A3
:104E100017F7FF1F2302F73083C73900228697F563
:104E2000FF1F9385652F85074A8517F7FF1FA30688
:104E3000F72E97F0FFFFE78060082A84E30505DA84
:104E400097C50100938545E017B501001305C562BC
:104E500097A00100E780C0B4A28517C50100130523
:104E6000A500C9B5894763E3870297C5010093850B
:104E7000A5DD17B501001305256097A00100E780A7
:104E800020B217C50100130565AF35B1974000008A
:104E9000E780A0E5A28517F5FF1F1305E5279750CA
:104EA0000000E780C08F81B38D476303F40297C58C
:104EB0000100938565D917B501001305E55B97A03F
:104EC0000100E780E0AD17C501001305E5ACE5B6CC
:104ED000B76602000146B7750200054597E0FF1F5F
:104EE000E780008F930760F817F7FF1F2306F7226C
:104EF00097F7FF1FA38307229307000617F7FF1FEB
:104F0000230EF720894717F7FF1FA309F72097F70C
:104F1000FF1F2386072097F7FF1FA3820720C147A3
:104F200017F7FF1F230EF71E930720F917F7FF1F30
:104F3000A308F71E314697F7FF1FA384A71E97F516
:104F4000FF1F9385651D4A8597F7FF1F238B071C5D
:104F500097F0FFFFE78080F62A84E30605C897C52F
:104F60000100938565CE17B501001305E55097A0A4
:104F70000100E780E0A2A28517C50100130545A343
:104F800055B3B1476303F40297C501009385C5CBC0
:104F900017B501001305454E97A00100E78040A01A
:104FA00017C50100130585A239B6B7E70400FC4F09
:104FB0009305000417F5FF1F034545898297974025
:104FC0000000E78080D2B145F9B5914763E38702DD
:104FD00097C50100938545C717B501001305C5495D
:104FE00097A00100E780C09B17C501001305C59F6E
:104FF000D9B497F4FF1F83C4641297F7FF1F83C7C8
:10500000D711A204DD8C8E04B77702006D14BE9414
:105010002286A68517C501001305459E97A00100AD
:10502000E7800098B7E70400FC47228697F5FF1F4A
:105030009385D50E2800829793160401C182300013
:10504000A685094597D0FF1FE78080782A8409C983
:1050500017C501001305459C97A00100E78020AC0F
:10506000930770F8194697F5FF1F9385E50A4A855F
:1050700017F7FF1F2302F70A97F7FF1FA380870A7E
:1050800097F0FFFFE78080E32A84E30E05B497C51D
:105090000100938565BB17B501001305E53D97A099
:1050A0000100E780E08FA28517C501001305C597B1
:1050B00095B99947630BF41297C501009385C5B85C
:1050C00017B501001305453B97A00100E780408D0F
:1050D00017C501001305C596F9BA914763E3870226
:1050E00097C50100938545B617B501001305C5386E
:1050F00097A00100E780C08A17C501001305C59578
:105100005DBA97F4FF1F83C4640197F7FF1F83C73D
:10511000D700A204DD8C8E04B77702006D14BE9414
:105120002286A68517C501001305459497A00100A6
:10513000E7800087B7E70400FC47228697F5FF1F4A
:105140009385D5FD2800829793160401C182300013
:10515000A6850D4597D0FF1FE78080672A8409C97F
:1051600017C501001305459297A00100E780209B19
:10517000930780F8194697F5FF1F9385E5F94A854F
:1051800017F7FF1F230AF7F897F7FF1FA38887F881
:1051900097F0FFFFE78080D22A84E30605A497C535
:1051A0000100938565AA17B501001305E52C9790BA
:1051B0000100E780E07EA28517C501001305058E7A
:1051C00095B699476303F40297C501009385C5A777
:1051D00017B501001305452A97900100E780407C30
:1051E00017C501001305058DF9B0B7E70400FC4FA2
:1051F0009305000417E5FF1F034545658297974017
:105200000000E78080AE994579B18D476303F402D1
:1052100097C50100938545A317B501001305C52562
:1052200097900100E780C07717C501001305058A34
:1052300059B017C501001305658A97A00100E780E2
:10524000008E1305C01297D0FF1FE780800F014525
:1052500097E0FFFFE78040E30D4597100000E780EF
:10526000009F294597D0FF1FE780A00D97D0FF1F13
:10527000E78000FE8DBA99476303F40297C50100E9
:105280009385859C17B501001305051F97900100B4
:10529000E780007117C501001305058529B817F7C8
:1052A000FF1F0347B7E797F7FF1F83C727E72207CB
:1052B0005D8F9166BA96C2061166C1821306F6EF3B
:1052C0008D476365D60297E7FF1F9387A70D9C4B19
:1052D00017F6FF1F034676E49386C7002DC203D658
:1052E000070069CA8907E39CD7FE89471307A0F81E
:1052F000114697F5FF1F938525E24A8597F6FF1F14
:10530000238CE6E017F7FF1FA309F7E097F0FFFFF4
:10531000E780C0BA2A84E308058C97C5010093850D
:10532000A59217B501001305251597900100E78098
:105330002067A28517B501001305457CE5B203D6A9
:105340000700630EE60A8907E39BF6FE8D4779BFE7
:1053500091476304F40297C501009385E58E17B564
:1053600001001305651197900100E780606317B590
:1053700001001305257A6FF00FF4B7E70400FC4F26
:105380009305000817E5FF1F0345454C8297C9B8F0
:1053900097C501009385458B17B501001305C50D11
:1053A00097900100E780C05F17B5010013050578ED
:1053B0006FF06FF02390E70017E5FF1F130585FEE0
:1053C00097300100E780408A97C501009385C58723
:1053D00017B501001305450A97900100E780405C6E
:1053E00017B501001305857597900100E780405BB4
:1053F000294597900100E780805F8147C5BD2390D4
:10540000070017E5FF1F1305E5F997300100E78056
:10541000A08597C501009385258317B50100130565
:10542000A50597900100E780A05717B50100130567
:1054300065725DBF411122C406C6834705002A84F8
:105440009DC797B501009385E57B17B5010013054E
:10545000A50297900100E780A0544C4017C50100B9
:105460001305C5A697900100E7808053E1A058413D
:10547000B707CF009387777D631DF70697B50100C7
:105480009385457817B50100130505FF9790010036
:10549000E78000511C448356E4008355C40003C6D2
:1054A000070017C501001305E5A397900100E780E9
:1054B000204F294597900100E78060530357E4008F
:1054C0009707002083D767256309F7008355C40039
:1054D000084497E0FFFFE780A0CF0356E400835520
:1054E000C40008442244B240410117F3FFFF6700A3
:1054F0002355B707CC009387777D6315F70497B5DD
:1055000001009385257017B501001305E5F6979006
:105510000100E780E0481C448356E4008355C40042
:1055200003C6070017C501001305C59B979001002E
:10553000E78000472244B24029454101179301000A
:105540006700E34AB707CE009387777D6304F702CD
:1055500097B501009385056B17B501001305C5F1DB
:1055600097900100E780C0434C4017C50100130528
:10557000A58CCDBDB240224441018280B7E7040032
:10558000FC4741112E8606C622C426C24AC02E847C
:105590002A89AA8517F5FF1F130505B8829797B5C5
:1055A00001009385256C17B501001305E5EC979074
:1055B0000100E780E03E97F5FF1F83C5E5B517B50D
:1055C00001001305251297900100E780603D2945F1
:1055D00097900100E780A04197F4FF1F9384C4B324
:1055E00083C7040041479387070693F7F70F636A61
:1055F000F75C17B701001307A7FB8A07BA979C430C
:10560000BA9782879D476307F40297B50100938597
:10561000656517B50100130525E697900100E78041
:10562000203817B501001305650C97900100E7803D
:105630002037ADAC97F7FF1F83C717AEDDCB17F749
:10564000FF1F034797AD97F7FF1F83C707AD2207DB
:105650005D8F97F7FF1F83C767ACC2075D8F97F712
:10566000FF1F83C7B7ABE207D98F17F7FF1F2323AD
:10567000F7A883C7640097B501009385A55E17B5A9
:105680000100130565DF17F7FF1F2304F7A69790A6
:105690000100E780E03097F7FF1F9387A7A58C43B1
:1056A00017F6FF1F0346E6A417B501001305C5054D
:1056B00097900100E780C02E294597900100E78070
:1056C000003397F7FF1FA38907A42244B2409244F6
:1056D0000249930700F817F7FF1F230FF7A29D4514
:1056E00017F5FF1F130545A341011743000067008D
:1056F000030B97600000E78020DB97F7FF1F238EE6
:10570000A7A09357850017F7FF1FA308F7A093578B
:1057100005012A8417F7FF1F2302F7A0935785017D
:10572000014517F7FF1FA30BF79E97600000E78066
:1057300060D897F7FF1F2384A79E97B50100938534
:10574000655217B50100130525D397900100E78036
:10575000202517F6FF1F0346869CA28517B501007A
:10576000130505FCB1B7CD476303F40297B50100FB
:105770009385454F17B50100130505D0979001009B
:10578000E780002217B50100130505FB79BD37E45A
:1057900004007C44414697F5FF1F9385F59717F564
:1057A000FF1F13056595829717F5FF1F1305C59415
:1057B00097100000E78080CE97100000E78020BBA4
:1057C00097F7FF1F83C7679617F7FF1F0347D79504
:1057D000A20703238405D98F17F7FF1F231AF79019
:1057E0001306000A89452244B2409244024917E553
:1057F000FF1F0345A505410102838D476303F402A2
:1058000097B501009385054617B501001305C5C678
:1058100097900100E780C01817B5010013058501B6
:1058200029B517F4FF1F0344448F97F7FF1F83C761
:10583000B78E97B501009385E542220417B50100A4
:10584000130585C35D8C97900100E7806015A285E4
:1058500017B501001305C5EF97900100E7804014CC
:10586000294597900100E78080180D4697F5FF1FA6
:105870009385858A228597E0FFFFE7802064AA84CC
:1058800021C197B501009385E53D17B501001305CA
:10589000A5BE97900100E780A010A68517B501006E
:1058A000130545EC97900100E780800F2244B24039
:1058B00092440249294541011793010067002313CF
:1058C00097E7FF1F239C877AB7E70400116603A3BD
:1058D0008705130606E8914539B78D476303F4023F
:1058E00097B501009385053817B501001305C5B8B4
:1058F00097900100E780C00A17B501001305450223
:105900002DB317F4FF1F0344448197F7FF1F83C78C
:10591000B78097B501009385E534220417B50100DF
:10592000130585B55D8C97900100E7806007A2851F
:1059300017B50100130545E497900100E780400684
:10594000294597900100E780800A0D4697E5FF1FE3
:105950009385857C228597E0FFFFE7802056AA8407
:105960001DC197B501009385E52F17B501001305FB
:10597000A5B097900100E780A002A68517B50100A9
:105980001305C5E005B797E7FF1F239B876CB7E7B3
:105990000400116603A38705130606E893050002B9
:1059A00099B5894763E3870297B501009385852BF5
:1059B00017B50100130545AC97900100E78040FE44
:1059C00017B50100130585F88DB197E4FF1F83C457
:1059D000C47497E7FF1F83C7377497B50100938599
:1059E0006528A20417B50100130505A9DD8C979061
:1059F0000100E780E0FAA68517B50100130585DAF6
:105A000097900100E780C0F9294597900100E78051
:105A100000FE228697E5FF1F93850570268597E097
:105A2000FFFFE780A0492A84630E051A97B501009D
:105A30009385452317B50100130505A49790010030
:105A4000E78000F6A28517B501001305E5D699BDDC
:105A5000854763F98718834519002244B240924470
:105A60000249B335B00097E7FF1F2383B76217B52C
:105A700001001305A5D5410117930100670043F20A
:105A8000A2852244B24092444A850249410117034B
:105A900000006700032299476303F40297B50100F1
:105AA0009385451C17B501001305059D97900100CE
:105AB000E78000EF17B5010013050503BDB617E435
:105AC000FF1F0344846597E7FF1F83C7F76497B5FB
:105AD000010093852519220417B501001305C59906
:105AE0005D8C97900100E780A0EBA28517B50100BF
:105AF000130545CF97900100E78080EA29459790EC
:105B00000100E780C0EE194697E5FF1F9385C56049
:105B1000228597E0FFFFE780603AAA841DC197B510
:105B200001009385251417B501001305E59497909E
:105B30000100E780E0E6A68517B50100130585CBD7
:105B400095B397E7FF1F2391875CB7E704001166C1
:105B500003A38705130606E89305000869B1854786
:105B600097B501009385051017B501001305C59081
:105B7000630BF40097900100E78080E217B5010005
:105B8000130585C85DB497900100E78060E117B503
:105B900001001305E5C897900100E78060E0294502
:105BA00097900100E780A0E42244B2409244024969
:105BB00097E7FF1F239E075241011753000067001C
:105BC000237F97B501009385E50917B501001305FB
:105BD000A58A97900100E780A0DC17B501001305A6
:105BE000E5F4A1B4B24022449244024941018280CA
:105BF000411106C622C497E0FFFFE780202C93776F
:105C0000F50FA1C32A8497B501009385250717B521
:105C100001001305658697900100E78060D89375B1
:105C2000F40F17B501001305252497900100E780B4
:105C300020D72244B2402945410117930100670053
:105C400003DBB240224441018280411122C49146CB
:105C50002A8417E6FF1F1306665A9D652D4506C662
:105C600097D0FF1FE780C0B6B7F7070003C707014B
:105C7000A5476313F70001A09306001001469D6538
:105C8000254597D0FF1FE780A0B497E7FF1F238724
:105C900087562244B240914617E6FF1F1306065668
:105CA0009D652945410117D3FF1F670063B211713C
:105CB000CED7B7E9040083A7C904CAD917E9FF1FE3
:105CC00013098945A2DD2E8686DFA6DB2E84AA85F0
:105CD0004A85829797E7FF1F83C707441307700A17
:105CE0006385E710636DF7001307600A6385E704B7
:105CF000FE506E54DE544E59BE5911618280130716
:105D0000800A6385E7161307900AE393E7FE8D4741
:105D10006306F41C97B501009385452817A501007B
:105D20001305857597900100E78080C717B50100BE
:105D30001305052425A08D47630CF40297B50100D7
:105D40009385C52517A501001305057397900100DC
:105D5000E78000C517B501001305C51A979001002B
:105D6000E78000C4294597900100E78040C849B703
:105D7000854717B501001305A51A17E7FF1F23096B
:105D8000F73097900100E78080D9B7750200B766B9
:105D900002000146054597D0FF1FE78060A39307E7
:105DA00060F817E7FF1F2309F73697E7FF1FA38661
:105DB00007369307002617E7FF1F2321F736E577FD
:105DC0009387072117E7FF1F231CF734B14597E797
:105DD000FF1F2388073497E7FF1FA384A7344A8552
:105DE00097000000E780E01621B7914763E3870240
:105DF00097B501009385851A17A501001305C5679E
:105E000097900100E780C0B917B50100130545134D
:105E1000B1B797E4FF1F83C4643097E7FF1F83C7C0
:105E2000D72FA204DD8C83A7C9046D14228697E5C1
:105E3000FF1F9385B52E280082978E0493160401C8
:105E4000B7750200C1823000A695094597D0FF1FA3
:105E5000E7800098930770F817E7FF1F230EF72AD3
:105E6000994597E7FF1FA38BA72A95BF914763E347
:105E7000870297B501009385651217A501001305E8
:105E8000A55F97900100E780A0B117B50100130549
:105E9000A50CE9B597E4FF1F83C4442897E7FF1FCB
:105EA00083C7B727A204DD8C83A7C9046D1422869B
:105EB00097E5FF1F93859526280082978E049316F9
:105EC0000401B7750200C1823000A6950D4597D038
:105ED000FF1FE780E08F930780F8BDBF17B5010073
:105EE0001305450A97900100E78060C3930790F877
:105EF0002304F100834719008D452800A304F10015
:105F0000834729002305F10097000000E780600423
:105F10001305C01297C0FF1FE780A042014597D02C
:105F2000FFFFE78060160D4597000000E78020D254
:105F3000294597C0FF1FE780C04097C0FF1FE7803B
:105F400020317DB397E7FF1F23A2A72C828097E71C
:105F5000FF1F9387A72B03A307006303030002839C
:105F6000174300006700A38341114AC097F6FF1F43
:105F700083D6A67A328917D6FF1F0356C64422C499
:105F800026C206C62A84AE8497000000E7804065DA
:105F900035C12DC0994763FF970483471400034719
:105FA0000400A207D98F13978700A183D98FC20756
:105FB0003167C1831307C755639EE70297D7FF1F59
:105FC00083D76740A301F400A1832302F40097F76D
:105FD000FF1F83D7877491C7A302F400A183230313
:105FE000F400A68517B50100130545FF9790010041
:105FF000E780009B97F7FF1F83C7C761B9CF97D58D
:10600000FF1F83D5453C17B501001305E5FE9790AA
:106010000100E780E0982686A28517D5FF1F03556B
:10602000853A97000000E780E0BC6301090497E728
:10603000FF1F83C7E71D9DCB95C897E7FF1F83C749
:1060400027058DE722852244B2400249A685924465
:106050004101173300006700837417B50100130571
:10606000A5FA97900100E78080ABC1B7B240224407
:10607000924402494101828083475500834545008F
:1060800017B50100130545F4A207DD8D1793010034
:106090006700039117B50100130505F2179301007E
:1060A0006700E3A78D4763FBB70A011126CA06CE36
:1060B00022CC0344350097E4FF1F83C4741597B5C1
:1060C0000100938525F5B337800017E7FF1FA30173
:1060D000F71409C497B50100938585F417B501003D
:1060E000130585F497900100E780808B97E7FF1FE9
:1060F00083C717126386970097000000E780402C43
:1061000097E7FF1F83C7D7108DC785472306F10088
:10611000B7E7040083A74717700085451305503083
:10612000829717B50100130525F197900100E780CC
:10613000009F9967938757EE2316F1006800854703
:106140009145A30781002307F10097000000E78035
:1061500040E0F2406244D2440561828082808947F7
:1061600063F7B708011122CC06CE26CA8344250066
:1061700085472A84639DF404914763F5B70403457A
:1061800045008347340022055D8D97D7FF1F239C70
:10619000A72297000000E780804D9967938767EEFC
:1061A0002314F1008347340023059100A305F10077
:1061B00083474400954528002306F100970000001E
:1061C000E78020D9F2406244D24405618280FDF824
:1061D0009967938767EE2314F10097D7FF1F83D742
:1061E000871EA305F10023050100A183E1B782808A
:1061F0000111996722CCD51717F4FF1F13048441AE
:106200002314F1008347040026CA97F4FF1F9384E8
:10621000C4502305F10083D7040028009545A30549
:10622000F100A18306CE2306F10097000000E7806D
:1062300040D203D604008345040017B501001305BE
:1062400025E197800100E780A075F2406244D244C6
:10625000056182809D677971D9172316F10097F740
:10626000FF1F83C7273B06D62307F100A9C3B7E763
:106270000400FC47414697E5FF1F9385E5E71305BA
:10628000F10082976800CD4597000000E78060CC60
:1062900097F5FF1F83C5053817B50100130545DEC7
:1062A00097800100E780C06FB25045618280B7E7F8
:1062B0000400BC47414681451305F1008297D9B7D8
:1062C00045C5411106C622C4930750FA2300F500C4
:1062D0009307A005A300F50089472301F500914726
:1062E000A301F50093076002A302F50097F7FF1FD3
:1062F0009387473283C70700230205002A842303BC
:10630000F50097E7FF1F9387B7F083C70700414663
:1063100097E5FF1F938545DEA303F50097F7FF1F61
:1063200083D7A73F2304F500A183A304F50097D7E3
:10633000FF1F83D747092305F500A183A305F500B7
:10634000B7E70400FC47310582972285F1459700A5
:106350000000E780E024230EA4002181A30EA40006
:10636000B24022444101828082805D710A8586C6E6
:10637000A2C497000000E780E0F437E404007C4406
:106380008A850810794682973C441305E103094643
:1063900081458297101093050002014597D0FFFFB9
:1063A000E780C034B640264461618280AA85856654
:1063B0000146254517C3FF1F670083410111B7C779
:1063C000A55A22CC9387C73317E4FF1F130454E464
:1063D0003EC483470400196506CE3EC69700000000
:1063E000E78000FD3000A1469965294597C0FF1F51
:1063F000E780003E8345040017B50100130505D969
:1064000097800100E780C059F240624405618280B4
:106410000111A146300099652D4522CC06CE97C0CA
:10642000FF1FE780E03AA24737C4A55A1304C433DC
:1064300063958702B24517B50100130565C8B335EA
:10644000B00097E7FF1FA385B7DC97800100E780C6
:106450002055F2406244056182809165A14630007A
:10646000938505F02D4597C0FF1FE7806036A24752
:10647000E38287FC814517B501001305A5C697E7A0
:10648000FF1FA38707D897800100E780605197001E
:106490000000E780E0F275BFB7C7A55A797193870E
:1064A000F7353EC6B7E70400FC4706D6AA85414645
:1064B00008088297116597000000E78060EF700080
:1064C000D1469165294597C0FF1FE780603017B519
:1064D0000100130565CF97800100E7804064B2504A
:1064E000456182807971D146700091652D4522D435
:1064F00026D206D697C0FF1FE780802DB24737C44B
:10650000A55A1304F4358144638987029165D14605
:106510007000938505E82D4597C0FF1FE780402B4D
:10652000B2478544638B870017B50100130585C307
:1065300097800100E780A05E25A8B7E70400FC472C
:1065400017E5FF1F130545BB41460C08829717B599
:106550000100130525BF97800100E780405C89C8D2
:1065600017E5FF1F130545B997000000E78000F30A
:10657000B25022549254456182804111116506C681
:1065800097000000E780C0E2B24017B50100130594
:1065900065B141011783010067006358C1676976DF
:1065A0008146FD1705061397060141836364B70012
:1065B0003E8582803307D50003470700B98F214706
:1065C00013F81700858363050800B18FC207C183E4
:1065D0007D171377F70F6DF78506F1B741C5A5470E
:1065E000054763F2B7088347150003470500316884
:1065F000A207D98F13978700A183D98FC207C183C0
:106600001308C855054763900707411106C622C401
:1066100026C203442500914763F087049307540082
:1066200063ECF502A301C50021822302C500930497
:10663000340091C6A302D500A1822303D5002A8489
:10664000A68597000000E780A0F526942300A4000B
:106650002181A300A4000147B240224492443A851C
:106660004101828005473A8582800111B7C7A55A4A
:1066700022CC9387E7342A842AC6156506CE3EC409
:1066800097000000E780C0D23000A14695652945FB
:1066900097C0FF1FE780C013A28517B5010013053F
:1066A000E5B097800100E780A02F97000000E78009
:1066B00000CCF2406244056182800111A1463000A5
:1066C00095652D4522CC06CE97C0FF1FE780401070
:1066D000A24737C4A55A1304E43463808706916542
:1066E000A1463000938505EE2D4597C0FF1FE7803A
:1066F000200EA247639087020355C10097D7FF1F62
:106700002393A7CC97000000E78060F6F240624434
:1067100005618280D147D14517B501001305859EDB
:1067200017D7FF1F2311F7CA97800100E780402782
:1067300017D5FF1F035525C9F1B7B24517B501009D
:106740001305459E97D7FF1F239FB7C6C205C1817A
:1067500097800100E780C02497000000E78020C1F7
:1067600075B721C1411126C206C622C4AE848DC5AB
:106770002A8497000000E780A05E97E7FF1F83C789
:1067800027A999CB22852244B240A6859244410193
:10679000173300006700A300B24022449244410135
:1067A0008280828001114AC806CE22CC26CA4EC6FB
:1067B00093F715002E899DCBAD673717004093875F
:1067C000A7AA1CC3B7E70400BC4F130600198545F0
:1067D00017D5FF1F034505BF829713451900F240E7
:1067E0006244D2444249B2490561828093F7250050
:1067F000638A071C17F7FF1F035707F2954763F9D2
:10680000E70C014417F6FF1F130606E19306300557
:1068100013055004130810049308B00413039005E3
:10682000930764006374F7043A84FD5997F4FF1FDB
:1068300083C484DE97F7FF1F83C717DEA204DD8CB5
:10684000AD679387B755638BF41463E3970AA96721
:106850009387A755638EF414A28517F5FF1F1305C0
:10686000A5DB97000000E78000F031A2B3078600A7
:1068700083C50700639AD50483C517006396A504F2
:1068800083C527006392050583C53700639ED50243
:1068900083C54700639A150383C757006396670251
:1068A000A2890DE897F5FF1F83D505E7B38535412C
:1068B000C20517F5FF1F130525D6C1814E95970018
:1068C0000000E78040EAE1A005044204418089BF5E
:1068D0003A84FD598547E3EB87F45DC4854517F598
:1068E000FF1F130565D397000000E780C0E769A884
:1068F000B1679387C7556380F404B5679387D7550D
:10690000E39CF4F4A28517F5FF1F1305E5D097303B
:106910000000E780C0E88947630FF4049305E4FFB3
:10692000C205C18117F5FF1F130525CF9700000091
:10693000E780004389A097200000E780C0D8970037
:106940000000E780404111C9A28517F5FF1F13051C
:10695000A5CC97000000E780A0400546A28517F56A
:10696000FF1F130565CB97F0FFFFE780206097209E
:106970000000E78040D5A68517B501001305C58640
:1069800097800100E780C001FD57E39DF9F097F77C
:10699000FF1F239307D81345290091B5A28517F54A
:1069A000FF1F130565C797F0FFFFE780206DE1B774
:1069B000A28517F5FF1F130525C697F0FFFFE78097
:1069C000A06D55BF93F745000145E38A07E017B571
:1069D00001001305A58297800100E78040149730DD
:1069E0000000E780600A13454900D5BB411122C46D
:1069F00037E404005C5C06C6354697A50100938524
:106A0000E53017B501001305E5F6829711E917A5E2
:106A100001001305657F97800100E780401001A009
:106A20008327041C82972A84054597C00000E780CD
:106A300080C397600100E780A04897600100E7806D
:106A4000A01D97B00000E78000D52285B240224407
:106A5000410182801567B71700401307575598C347
:106A6000D8439D66558FD8C3D843FD76758FD8C35C
:106A7000D8431367F70FD8C335671307C7CC98C33C
:106A800082804111054506C622C426C297C0FFFF79
:106A9000E78060491305A00497B0FF1FE7802061DD
:106AA000757585457D1597C0FFFFE78000337D75BF
:106AB00085451305F53697C0FFFFE780603C371426
:106AC00000408327840A8D451305002093E70720A3
:106AD0002324F40A97C0FFFFE7802030B7E40400C6
:106AE00097C0FFFFE7804075C85897800100E78096
:106AF000000317B501001305E5E797800100E78063
:106B000000028327840C8545414593E70708232429
:106B1000F40C97C0FFFFE780A0368D4513050008F1
:106B200097C0FFFFE780C03597C0FFFFE780A062F6
:106B300037A507001305051297C0FFFFE780405EE9
:106B4000014597C0FFFFE78060649545054589478B
:106B500017F7FF1F2304F7BC97C0FFFFE780A0646F
:106B6000B7E700E013070006238DE740370700046E
:106B700023A0E71097D0FFFFE780A0F597D0FFFF95
:106B8000E780600997000000E78080E6970000003A
:106B9000E780408897000000E78060B297E0FFFF41
:106BA000E78040E597000000E780C01C97000000E8
:106BB000E780600B83A70408170500001305C5BE16
:106BC000829797C7FF1F238FA77EBC4C13060064D4
:106BD0008545829797000000E78000E897C0FF1F77
:106BE000E780008101458280B7F7070003C70701EE
:106BF000A547AE866316F7009397450191C301A0A0
:106C0000AA850146254517C3FF1F670063BC4111D4
:106C1000B2862E86AA852D4506C697C0FF1FE7803F
:106C200020BBB2400145410182809307000463E824
:106C3000C7021D71A2CC2A84080886CE32C697806E
:106C40000100E78080CAB2461008A285294597C096
:106C5000FF1FE780E0B7F640664425618280395522
:106C6000828041110D658D4506C697C0FFFFE78004
:106C7000C016B71700408D6623A6D70A17F5FF1F69
:106C8000130505AA1387C70A9387870A1CC15CC529
:106C9000856689675CC958C114C518C9B7E704007F
:106CA000B24003A3871E410102838145B307B500AB
:106CB0008387070089E717230000670063A785051E
:106CC000C205C181E5B7411126C2E97797F4FF1FDC
:106CD000938484B522C49387A7552E842381B4005E
:106CE0002E86AA8517F5FF1F130545B406C6239007
:106CF000F400A381040097800100E78000BF9305A2
:106D00002400C205C18117F5FF1F130505B29700C6
:106D10000000E780E088B38784002382A7002181F8
:106D2000A382A700930564002244B24026859244C2
:106D3000C205C1814101172300006700639F09C993
:106D40009307800263E6B700170300006700E3F7CC
:106D5000828017F5FF1F0345259E828097F7FF1F4E
:106D600083C747AC89E7172300006700639C8280D4
:106D700097F7FF1F83C727AE99EF411106C69720EB
:106D80000000E780C092B240854717F7FF1F230439
:106D9000F7AC410182808280630E0532638C05323C
:106DA0005D71CAC04EDE86C6A2C4A6C252DC56DAE7
:106DB0005AD85ED662D466D26AD0B9472A89AE89DB
:106DC00063F9B706394697A501009385A54A9780D0
:106DD0000100E78020AF31ED8347E900130710037E
:106DE0006394E702854717F7FF1F230DF7A217A546
:106DF00001001305254997F7FF1F239407A2970069
:106E00000000E780C0EA71A01307000317A5010086
:106E10001305454AE395E7FE97F7FF1F238407A074
:106E200097F7FF1F239F079E17A50100130505472E
:106E3000F9B797F7FF1F83C7E79E63870722BD6AED
:106E4000B96B938CFA55014A17FBFF1F130B0B8F7D
:106E5000138CEB65938AFA6605A8B307490183C6CC
:106E6000070097F7FF1F83D7C79BB1E39307A005E0
:106E7000639BF600854717F7FF1F2314F79A97F7D0
:106E8000FF1F238DD78A050A93170A01C183E3E602
:106E900037FDB640264496440649F259625AD25A02
:106EA000425BB25B225C925C025D61618280054D57
:106EB000639BA7039307500A639EF600894717F761
:106EC000FF1F2310F796930750FA17F7FF1FA3072A
:106ED000F78655BF9307A005E387F6FA97F7FF1FDC
:106EE000239107944DB7138717004207DA97418320
:106EF0002380D70017F6FF1F2315E6928D47E3F492
:106F0000E7F817F4FF1F0344948397F7FF1F83C725
:106F1000078322045D8C9307F4FFC207C1839306A5
:106F2000F00DE3EDF6FA93076400C207C183E31C9A
:106F3000F7F493052400C205C18117F5FF1F13055F
:106F4000058097F0FFFFE780A06533078B0083473C
:106F5000570003474700A207D98F17F7FF1F2312D7
:106F6000078C6318F50E8144630CA40197E4FF1F9E
:106F700083C4047DA20497E7FF1F83C7777CDD8C61
:106F8000170500001305E5DB97F0FFFFE780C0FB66
:106F900063878407636D9C029387EB556382F404D7
:106FA00097E7FF1F83C7C77905476389E70681CB4A
:106FB0001387A7051377F70F8D4663F2E6081307CB
:106FC000F0072300E100A300F10089459DA0638242
:106FD0009405E39754FD97F0FFFFE780E02711A8A1
:106FE000A28517E5FF1F1305A57597F0FFFFE78042
:106FF000A00B014597F0FFFFE78000F569B5A2857A
:1070000017E5FF1F1305C57397F0FFFFE7806015B5
:10701000CDB797F0FFFFE780E01DE1BF930710F8C1
:10702000130511002300F10097F0FFFFE78080298E
:10703000FD450A8597000000E78020C95DBFA28555
:1070400017E5FF1F1305C56F97F0FFFFE78060C6C8
:107050004DB79307F00789450A852310F100970083
:107060000000E78080C605B5C14763FE370541468D
:1070700097A50100938545264A8597800100E78002
:10708000608431E18347090113071003639CE70023
:10709000854717E7FF1F2301F76A17A501001305AE
:1070A000E524B1BB1307000317A50100130505274D
:1070B000E397E7D497E7FF1F2380076817A5010030
:1070C000130545242DBBCE854A8597C0FFFFE78079
:1070D0002010C1B38280411126C2AE848D4522C4E6
:1070E00006C62A8497C0FFFFE78080D9B717004003
:1070F00099C803A5C70C418D23A6A70CB240224412
:1071000092444101828003A5870C418D23A4A70CE2
:10711000F5B78347050003471500A207D98FC207BB
:107120006177C18713072720639AE700834525000D
:107130003705040017030000670023FA828017E672
:10714000FF1F1306A6718147B2861303F00FA948EB
:107150003308F6000348080013F7F70F6307A80C7D
:10716000630668008507E39517FF2947B387E600A4
:107170002380A70097E7FF1F9387076F5DA8411142
:1071800013D765001347170006C693F63500058B25
:10719000954791CA054699476387C60009469D47AA
:1071A0006383C600A14713F645003336C00093F64B
:1071B0008503050685C2A145638BB604E145638A54
:1071C000B604930580026388B60493058003639335
:1071D000B600914697F5FF1F238DF58E97F5FF1F9B
:1071E0002388C58E97F5FF1FA384D58EBE8517A56E
:1071F00001001305A51797700100E780607AB2407F
:10720000854717F7FF1FA306F78C4101828085464B
:10721000D1B78946C1B78D4675BF17A501001305C3
:107220006517177301006700A37717E7FF1F1307A0
:10723000A763BA972380B700E147E302F5F4930709
:107240007002E30CF5FC82802A87238005008147C9
:1072500017E5FF1F130585601308F00F2946B306D5
:10726000F50083C606006396E60297E6FF1F938645
:10727000A65FB69783C7070005452380F5009947A9
:10728000636EF7029D4763FDE700E147630DF7007A
:107290008280638506018507E393C7FC0145C5B776
:1072A000238005008280B737004003C7370083C7BB
:1072B000050093F70704D98F2380F50082805D7164
:1072C00052DC56DA5ED6716A97FBFF1F938B8B9167
:1072D0008D6AA6C24EDE62D486C6A2C4CAC05AD87F
:1072E00066D26AD06ECEC1495E8C97E4FF1F93844C
:1072F0006458130A0A20938A7ADC17F9FF1F03499E
:107300006991B3872B0183C7070093F7F70FC9EF84
:10731000B787004003C76700058BE310077C03C7EE
:107320006700118BE30D077E83C75700918B99E3AC
:107330006F10200317F7FF1F0347E78D854763048E
:10734000F7006F10400197E7FF1FA384E77897E7E6
:10735000FF1F2381075E97E7FF1F238F076897E7CB
:10736000FF1F238D077497E7FF1F238A077497E792
:10737000FF1FA381075C97E7FF1FA38F076697E7AF
:10738000FF1FA38D077297E7FF1FA38A077297E776
:10739000FF1FA381077497F7FF1FA38E0786B78788
:1073A000004011476F0070779307190093F7F70FAC
:1073B0003D476364F70617F7FF1F230DF78497F720
:1073C000FF1F93872784CA9783C7070013071002FC
:1073D00093F7F703638EE71E6366F704054463853E
:1073E000871CE38C07620947638EE71013070002CE
:1073F000E384E74EB7E700E03707400023A0E71833
:1074000001000100629923000900FD1923A0E71083
:1074100093F9F90FE39309EEE5BD97E7FF1F238B7F
:10742000077E71BF130730026388E70C63E8E71635
:1074300013074002638CE70A13070003E39CE7FA93
:1074400097E7FF1F9387077BCA9703C70700A147EA
:107450001377F70FE31BF71483C7640097E6FF1F4A
:107460002380F66697E7FF1F83C7374191C7FD5713
:1074700097E6FF1F2386F66497E5FF1F83C5953FB8
:1074800097E7FF1FA38EB76297E7FF1F83C7873E6B
:1074900013FB07089306000493F70706639FD74C76
:1074A0009307A009638DF51663EAB7129307F005F9
:1074B0006386F54A930750096384F52A014497E7E8
:1074C000FF1F83C7F75F1547E392E736B7E700E092
:1074D0003707400023A0E71801000100B7860040ED
:1074E00023808602130680FC6F00500EFD5717E7BD
:1074F000FF1F2306F75CFDBDFD5717E7FF1F230F96
:10750000F75ACDBD17A50100130545FA9770010084
:10751000E780E06097E7FF1F9387C76DCA9703C4B2
:107520000700014B97ECFF1F938C4C4D1374F40F25
:1075300017AD0100130D0DF863478B0429459770B3
:107540000100E780C04A854717E7FF1FA306F74AF7
:1075500017E7FF1F2303874A17E7FF1F230CF75680
:1075600037E700E0B70640002320D71801000100EC
:10757000378600408347A60293F7370F2305F602AC
:107580002320D71085BDB3876C0183C507006A85AA
:10759000050B97700100E780A04079BF854717E78A
:1075A000FF1F230BF744B9B517E7FF1F13078764C5
:1075B0004A970347070097E6FF1FA38DF63697E625
:1075C000FF1F238AE63617E7FF1F2305F7501DB577
:1075D000854717E7FF1F230FF73429BD9307400A9C
:1075E0006389F5349307200B6384F5369307100AFB
:1075F000E396F5EC838724000144E3D207EC97E798
:10760000FF1F83C7572793F63700638A061A05467C
:10761000638AC62209466395C61A1D4755A217E517
:10762000FF1F03454525C94797ECFF1F83CCBC24AA
:1076300097E5FF1F83C5452417E4FF1F0344D423A8
:107640006315F510CD476392FC1093077008639C97
:10765000F5021307300FB7170E006308E400130795
:10766000900DB7B704006314E40817E7FF1F232F3A
:10767000F744BE8517A50100130545E49770010086
:10768000E780003225BD93078008639DF500B307AE
:10769000804013F4F70FB7774600938787CDB3D7B1
:1076A0008702E1B793079008639AF500B30780401B
:1076B00013F4F70F91679387C766D5B79307A008B0
:1076C000639BF500B307804013F4F70FB7173D0035
:1076D00093870790E9B79307B008639AF500B3075B
:1076E000804013F4F70F9167938797D04DBF93F5C0
:1076F000F5078D47639BF500B307804013F4F70F40
:10770000B7975B00938707D859BF8947639BF500FC
:10771000B307804013F4F70FB7770B009387071B6D
:10772000BDBF8547639AF500B307804013F4F70F98
:10773000DD67938767E3A5B7D28785F9B3078040F4
:1077400093F7F70FB3D7FA020DB797000000E78061
:10775000409FA285668597000000E780809EB9BBA8
:107760009305610017E5FF1F0345E51017E4FF1FB0
:107770000344741097000000E78040AD930571004A
:10778000228597000000E78060AC3C0017E7FF1FF0
:107790002328F744834761002304F10083477100E5
:1077A000A304F100894717E7FF1F230BF730835726
:1077B000810017E7FF1F231FF70A094409B3154784
:1077C00093F64700B336D00093F78703850685C349
:1077D0002146638BC7066146638AC706130680028B
:1077E0006388C706130680036393C700914717E6B3
:1077F000FF1F230FD62C97E6FF1FA38BF62C97E7CE
:10780000FF1F2388E72C17E7FF1F0347E706937640
:10781000070497E7FF1F83C737068DEE1377770CB2
:1078200093067008630CD7021377F7078D4663122F
:10783000D70CB307F040B7955B0093F7F70F93852C
:1078400005D849A81947ADBF854755B7894745B7FA
:107850008D4771BF930670086311D7021307300F6D
:10786000B7150E006389E7021307900DB7B5040042
:107870006383E7021307700845BF9306800C63110A
:10788000D702B307F040B775460013F7F70F938799
:1078900085CDB3D5E70297E7FF1F23A9B722D9BB50
:1078A0009306900C631CD700B307F04093F5F70FD5
:1078B00091679387C766B3D5B702F1BF9306A00C53
:1078C000631DD700B307F040B7153D0093F7F70FDE
:1078D00093850590B3D5F5027DBF9306B00CE315F3
:1078E000D7F4B307F04093F5F70F9167938797D0DC
:1078F000D9B78946631BD700B307F040B7750B00B3
:1079000093F7F70F9385051BF1B78546631AD700E8
:10791000B307F040DD6593F7F70F938565E35DBF2F
:10792000D28535FBB305F04093F5F50FB3D5BA0218
:107930009DB783C72400C18B99C7854717E7FF1FF1
:107940002303F718A5BE97E7FF1F238E0716BDB6C2
:10795000854717E7FF1FA30EF7168DB63C0017E704
:10796000FF1F232FF7260947930700032314F10075
:1079700097E6FF1F2386E6142DBD63940756A9479B
:1079800063E5B74217A701001307879B8A05BA95DD
:107990009C41BA97828717E4FF1F0344D4ED894CBA
:1079A0006306940D63E68C0685476303F40893072A
:1079B000F00F17E7FF1F0347A71063F6E70017E76D
:1079C000FF1F230FF70E97ECFF1F83CC6C0F93075D
:1079D000000413F4FC0F63F497011304000497E709
:1079E000FF1F9387E71F03AD070022862685EA85E0
:1079F000B38C8C40229D97700100E78000EF97E7E1
:107A0000FF1F238F970B97E7FF1F23ABA71D45BCD5
:107A10008D47630CF40A9947E31BF4F897A701001C
:107A20009387879817E7FF1F232CF71AA94751B7A9
:107A300017E7FF1F0347271E97E7FF1F9387470A94
:107A4000494697A501009385259F6306870097A562
:107A500001009385659A3E8597700100E780E0E814
:107A600017E7FF1F232EA716C947A1B797E6FF1FE9
:107A700083C6661A054797E7FF1F938767066394D7
:107A8000E6023E851306700297A50100938545988E
:107A900097700100E78060E517E7FF1F2322A71416
:107AA0009307700239B73E851306300497A501008D
:107AB0009385459097700100E78020E317E7FF1F4B
:107AC0002320A71293073004EDB597E5FF1F83C568
:107AD00085DA17A501001305A59F97700100E780BF
:107AE00020EC054D97EDFF1F83CDED1297E5FF1FAD
:107AF00083C565D817A501001305859D6398AD0B57
:107B000097700100E780C0E997E7FF1F83C7A7D6FA
:107B1000B5CBE36EF4E817A4010013042496638C3C
:107B2000B70117A401001304E4956386970117A415
:107B300001001304A496228597700100E780E006F7
:107B40001375F50F93071500860717E7FF1F230925
:107B5000F7F88D4717E7FF1FA304F7F897E7FF1F14
:107B6000938707F80147BE861376F70F8907636589
:107B7000A60297E7FF1F23A5D70697E7FF1F83C736
:107B800027F605BD97A701009387478817E7FF1FD2
:107B90002328F704914731BD3306E400034606006D
:107BA000A380070005072380C7007DBF97700100F1
:107BB000E78000DF97E7FF1F83C7E7CBE1D7E368E4
:107BC000F4DE17A4010013046488638CA70117A4D2
:107BD0000100130424886386970117A4010013048D
:107BE000E488228597700100E78020FC1375F50F6B
:107BF00093071500860717E7FF1F2303F7EE8D474E
:107C000017E7FF1FA30EF7EC97E7FF1F938747EDDA
:107C10000147BE861376F70F8907E37CA6F4330687
:107C2000E40003460600A380070005072380C70081
:107C3000D5B797E5FF1F83C505C417A50100130538
:107C4000E58997700100E780A0D597E7FF1F83C7FC
:107C5000F7E893E7470017E7FF1FA301F7E883C79B
:107C6000240017E7FF1FA309F7E689B817A501004D
:107C70001305058897700100E78060EA97E7FF1F0A
:107C8000938787E583C7070017E7FF1F2304F7BE25
:107C900017E4FF1F0344C4E2333480000DB017A57E
:107CA00001001305258697700100E78040E797E7FC
:107CB000FF1F83C7B7E293E7070117E7FF1FA30F73
:107CC000F7E083C7240017E7FF1F2307F7E06FF0F3
:107CD000EFFE17A501001305258497700100E780CA
:107CE00000E403C704007D8B51EFB787004003C752
:107CF00067021377C70B136727002383E70203C7C5
:107D0000A7021377C70B136727002385E70203C772
:107D1000E7021377C70B136727002387E70203C720
:107D200027031377C70B136727002389E7028547CB
:107D300017E7FF1F2300F7C017E7FF1F230EF7CA3F
:107D400017E7FF1F230CF7D617E7FF1F2309F7D606
:107D500097E7FF1FA38007BE97E7FF1FA38E07C803
:107D600097E7FF1FA38C07D497E7FF1FA38907D4CA
:107D700097E7FF1FA38007D697E7FF1FA38D07E8AC
:107D80006FF0CFF389476312F70297E7FF1F83C7AE
:107D9000A7AE9146638CD70863E0F604638EE70CC8
:107DA0006369F70A05476380E70EFD5717E7FF1F72
:107DB000A308F7D037074000B7E700E023A0E71893
:107DC00001000100B78600401306F0FC2381C602C3
:107DD00023A0E7106FF00FE2130720086382E70883
:107DE0006362F70213071008E391E7FC378700404E
:107DF0008347670293F7C70B93E727002303F70234
:107E00006FF0CFEB130730086389E70213074008D0
:107E1000E39DE7F8378700408347270393F7C70BB5
:107E200093E727002309F7026FF04FE937870040F7
:107E30008347270393F73707F5B737870040834712
:107E4000E70293F7C70B93E727002307F7026FF0CA
:107E5000EFE6378700408347E70293F73707F5B728
:107E6000378700408347A70293F7C70B93E72700A4
:107E70002305F7026FF08FE4378700408347A7029E
:107E800093F73707F5B7378700408347670293F7C3
:107E90003707ADB717950100130505699770010005
:107EA000E780E0C797E7FF1F2386079CD5B31795A8
:107EB00001001305656897700100E78040C697E7E9
:107EC000FF1F2399079A97E7FF1F938767BF03C494
:107ED0000700894763F3870009441374F40F6FF0B8
:107EE0000FDE13070002E392E7EC631B0B0A638FBC
:107EF000F500930720026383F50817950100130529
:107F0000256797700100E780A0A945B51795010086
:107F10001305456397700100E78060C00144179D19
:107F20000100130D6D63A14CB387840083C5070066
:107F30006A85050497700100E78080A6E31694FF28
:107F400017950100130505BA97700100E78020BD61
:107F500017E4FF1F0344449201E897E7FF1F238DB6
:107F6000078E014B6FF0AFD58947E310F4E48547E6
:107F700017E7FF1F2302F78E6FF04FD417E6FF1F9E
:107F80000346768F97E5FF1F83C5E58E17950100A1
:107F90001305055D97700100E78080A06FF00FD298
:107FA0006380F50693071002E399F5F497E5FF1F48
:107FB00083C5858C179501001305855C97700100BA
:107FC000E780009E97E7FF1F23AC97C097E7FF1F4E
:107FD0009387C7AF944383D7470017E7FF1F034733
:107FE00047AF17E6FF1F2327D6881D4497E6FF1FDC
:107FF0002394F68897E7FF1F2381E7886FF02FCC43
:1080000097E5FF1F83C54587179501001305C558E0
:1080100097700100E780C09897E7FF1F238E0782C3
:1080200097E7FF1F239807846FF02FF92547638F89
:10803000E7C89946378700406394D7022300870238
:10804000B7E700E0B706400023A0D7180100010001
:10805000130600FC2301C70223A0D7106FF08FB9CD
:108060009306100A639FD70023008702B7E700E05A
:10807000B706400023A0D71801000100130680FCBA
:10808000D1BF9306A009E381D7FE9306400AE38D92
:10809000D7FC93062002639DD700B7E700E0B70640
:1080A000400023A0D7180100010023008702F9B780
:1080B0008546E384D7FE93070008E300FBFEB7E79D
:1080C00000E0B706400023A0D71801000100130606
:1080D00020FC23008702BDBF17E7FF1F0347579E01
:1080E0006302F71E63E7E70295476300F7109947BD
:1080F000630AF704B786004023800602B7E700E072
:108100003707400023A0E718010001001306A0FC78
:1081100075B99307F005630AF700930750096306E2
:10812000F70093071002E317F7FCB7E700E0370703
:10813000400023A0E71801000100B78600401306A5
:1081400020FC69B117EBFF1F034B8B9793070004CB
:108150005A8D63F46701130D000497E7FF1F93879F
:1081600027A883AC07001374FD0F2286E6852685B9
:1081700097600100E7806077B3078B40669417E74C
:10818000FF1F230FF79297E7FF1F23AB87A4B78743
:108190000040630C0B022380A703B7E600E037061C
:1081A000400023A0C6180100010003C7270213479F
:1081B00007042381E70203C727021377C70F238130
:1081C000E70223A0C6106FF0EFA22380070237E773
:1081D00000E0B70640002320D71801000100130675
:1081E00020FC2381C7026FF0AFB937870040834777
:1081F000370097E6FF1F83C6368E93F70708D58FA3
:10820000A301F700B7064000B7E700E023A0D718A6
:10821000010001001306A0FC35BD97E7FF1F9387FF
:10822000679DCA9783C7070093F7F70FC1CF97E7FA
:10823000FF1F83C7479ED9E717E7FF1F03475788EC
:10824000930700026310F70883AD040017DDFF1FDA
:10825000034D8D6297DCFF1F83CC1C6217DBFF1F71
:10826000034BAB61E6876A87DA866E8697D5FF1F78
:1082700083C5855E1795010013058533976001005E
:10828000E780007297E7FF1F23A2B78597E7FF1FDC
:108290002380A78597E7FF1FA38C978397E7FF1F8E
:1082A0002389678397D7FF1FA387875AB7E700E023
:1082B0003707400023A0E71801000100B7860040FF
:1082C0006FF04FA2B7E700E03707400023A0E718A0
:1082D00001000100B786004015BD97E6FF1F83C669
:1082E00086930547639CE60429472381E7020947F3
:1082F0002383E7022385E70297D7FF1FA38C077C20
:1083000097E7FF1FA3890790B7870040A381070065
:1083100017D7FF1FA302077C05472383E700B6405A
:10832000264496440649F259625AD25A425BB25BDD
:10833000225C925C025DF24D61618280294723815B
:10834000E70209472383E7022385E7022387E70241
:108350002389E70255B717D7FF1FA30EF74E6FE02B
:108360001FFF854717D7FF1F2306F75C17D7FF1F8F
:108370002304F76817D7FF1F2302F77417D7FF1FCF
:10838000230FF7726FE0BFFE854717D7FF1F230348
:10839000F75A17D7FF1F2301F76617D7FF1F230FC1
:1083A000F77017D7FF1F230CF77017D7FF1FA30312
:1083B000075817D7FF1FA301076417D7FF1FA30F85
:1083C000076E97D7FF1FA38C076E8280411106C6E8
:1083D00097000000E78080FBB787004023800700FC
:1083E000130740FC2386E7001307C004A386E700B9
:1083F00017D7FF1F130707482398E70017D7FF1F5A
:108400001307474B239AE70017D7FF1F1307C756D9
:10841000239CE70017D7FF1F13074762239EE7003F
:1084200029472381E70209472383E7022385E702DF
:108430002387E7022389E702A3810700930600F858
:10844000A380D700930690022380D700FD56238394
:10845000D7002381E7009306000537E700E0230BF0
:10846000D740B70640002320D71003C71700136773
:108470001700A380E700B24097D7FF1F239E076431
:1084800041018280411106C697000000E78000F09C
:10849000B787004023800700130700FC2386E7000E
:1084A0003147A386E70017D7FF1F1307A73C239880
:1084B000E70017D7FF1F1307E73F239AE70017D7F7
:1084C000FF1F1307674B239CE70029472381E7021F
:1084D00009472383E7022385E702A3810700930668
:1084E00000F8A380D700930690022380D700FD56A2
:1084F0002383D7002381E7009306000537E700E0D8
:10850000230BD740B70640002320D71003C717001E
:1085100013671700A380E700B24097D7FF1F239D82
:10852000075A41018280F1679387072017D7FF1F01
:10853000232EF758854717D7FF1F231BF758A1474E
:1085400017D7FF1F2307F75897D7FF1FA383075895
:1085500097D7FF1F2380075897D7FF1F238E072E1B
:1085600097D7FF1FA389072E814717D5FF1F130534
:10857000E52EFD5517D6FF1F1306062F2947B30614
:10858000F5002380B600B306F600238006008507B9
:10859000E397E7FE97D7FF1FA385075297D7FF1FE3
:1085A000A383075297D7FF1F238E075097D7FF1F2C
:1085B0002389075097D7FF1F2388075097D7FF1F9E
:1085C000A382075097D7FF1F238F074E814717D6E7
:1085D000FF1F130626614147B306F60023800600FD
:1085E0008507E39BE7FE828017D7FF1F0347A7623B
:1085F00085476316F700170300006700E3E81703D9
:1086000000006700E3DC411122C406C617D7FF1F34
:108610000347676085472E8613F4F50FAA85631715
:10862000F70417D5FF1F1305253997600100E78070
:10863000C02B97D7FF1F2381073CB78700402384B7
:108640008702B7E600E03706400023A0C618010005
:10865000010003C7A7021377C70F2385E702B240C3
:10866000224423A0C61001454101828017D5FF1F77
:108670001305452897600100E780202797D7FF1F43
:10868000238A072AB787004023828702B7E600E0E3
:108690003706400023A0C6180100010003C7670287
:1086A0001377C70F2383E7025DBF411106C697000A
:1086B0000000E78080E7B240410117030000670037
:1086C000E3F2411106C697F0FFFFE78080BF97D71E
:1086D000FF1F83C73726A1CB97D5FF1F83C5A525CD
:1086E00089C917D5FF1F1305252597E0FFFFE780F0
:1086F000E06A97D7FF1FA38F072297D7FF1F238B0F
:10870000073C37E700E0B70640002320D7180100F8
:108710000100378600408347660293F7370F230333
:10872000F6022320D710B2404101828041C9D9C549
:1087300097D7FF1F83C7473AD1C3011122CC4AC83C
:108740004EC656C25AC006CE26CA52C42E89AA891F
:108750000144930A0004371B030063772403B30723
:108760008940C207C183BE8463F4FA009304000405
:10877000C204C180130A1BD497D7FF1F83C7871B6E
:108780009DE37D1A631C0A00F2406244D2444249D0
:10879000B249224A924A024B0561828097F0FFFF5C
:1087A000E78020B2D1BF338589002694A685420494
:1087B00097000000E78060E5418045B7828097D749
:1087C000FF1F9387E74818429C4383D64500034523
:1087D000070083C5C700035646006396A50083D5EE
:1087E000E700638DD502011106CE2386A7002397EB
:1087F000D700B705CF00DC4B9385757D05077D1647
:108800002EC2230001003AC42316C1002317D10051
:1088100099C30A858297F240056182808280DC4D8F
:10882000DC4B81CFB7E70400904503A38705914552
:1088300017D5FF1F03450542028382806D713C08F6
:108840003EC6B707E500232291103EC8AA843C0823
:108850003285232611103ECA2324811023202111A2
:108860002E8997300000E780005E2A8497950100EA
:10887000938585D717850100130505C09760010012
:10888000E7800012A28517950100130565E6976041
:108890000100E780E010294597600100E78020157E
:1088A000B705CB009385757D680097100000E780C1
:1088B0002067A285680097300000E780204B0147C1
:1088C00081467000CA85268597200000E780A08A2F
:1088D00005CD2A8497950100938505D11785010060
:1088E000130585B997600100E780800BA285179575
:1088F00001001305A5E097600100E780600A2945A3
:1089000097600100E780A00E8320C110032481102E
:1089100083244110032901105161828097D7FF1FE2
:108920009387073318429C43797122D406D60348B3
:10893000070083C807012A8483D6450003554600F3
:108940006396080183D82701638DD8022388070125
:1089500005072399D7003708CC00DC4B1308787D36
:108960003ACC1307F5FF42CA23080100231EE10099
:10897000231FD10099C7080832C62EC482973246F9
:10898000A245228597000000E78080EBB250225478
:10899000456182806D713C083EC0B707E5003EC26C
:1089A0003C083EC423261110232481102322911059
:1089B000231701002318010023190100231A0100C5
:1089C000231B010097B7FF1F83D747A299E3C16715
:1089D000FD172316F10097B7FF1F83D747A191EB2F
:1089E00097D7FF1F9387C7269C439C43DC4783D7B9
:1089F000070017B4FF1F1304649F584C2317F1009E
:108A000083574400484B2318F10031E1979501004A
:108A1000938585C417850100130505A6976001009D
:108A2000E78000F817950100130545C49760010021
:108A3000E78000F7294597600100E78040FB83202D
:108A4000C11003248110832441105161828097B7A3
:108A5000FF1F83C7179A89EBB7E70400BC578297BB
:108A60005C4C23AA0700E1BFFD1797B6FF1FA38246
:108A7000F69803560701834704014C470A85230BE8
:108A8000F10097300000E780802B97D7FF1F938776
:108A9000271C9C430147814688430A866C00971037
:108AA0000000E780406DAA8429C197950100938555
:108AB000A5BA178501001305259C97600100E78082
:108AC00020EEA68517950100130505BB97600100F0
:108AD000E78000ED294597600100E78040F1584CA0
:108AE000B7E70400BC57484B9DBF97B7FF1F83C72C
:108AF0005790F5D7B7E70400BC4F1044854517D50C
:108B0000FF1F0345251582971DBF5C4EDC4BB9CF77
:108B1000B1CD411122C4178501001305E5952E84BE
:108B200097950100938585B106C697600100E7809F
:108B300020E7A285179501001305C5B697600100CF
:108B4000E78000E6294597600100E78040EAB7E743
:108B500004002244B24003A3870517D5FF1F034535
:108B6000650F130640069145410102838280411141
:108B700022C417B4FF1F130424851C4C06C689C7E2
:108B8000DC4399C34C488297584CB7E70400BC5764
:108B9000484B82975C4CB240224423AA0700410113
:108BA000828017B7FF1F13072784834707009306A8
:108BB000F00B850793F7F70F63E9F60097B6FF1FF1
:108BC0002384F682034507008280930700F8FDB7EF
:108BD000835745006386071001114AC817B9FF1F64
:108BE0001309C98052C4032AC90106CE22CC032727
:108BF0004A0126CA4EC656C2F15735E31307D00DB7
:108C0000FD57636EC704B7E9040083A709072A84E8
:108C10001305860042054181B284AE8A8297232AD9
:108C2000AA000325C9015C49A9E79795010093852E
:108C3000E59E178501001305258497600100E780F4
:108C400020D617950100130525AE97600100E78037
:108C500020D5294597600100E78060D9DD57F240B3
:108C60006244D2444249B249224A924A3E85056151
:108C7000828093874400B705CF002319F5009385C0
:108C8000757D310597100000E78080290325C90113
:108C900083456400310597300000E780200D0325EF
:108CA000C9012686D685310597300000E780200966
:108CB0007146A2854A8597600100E78000C3504451
:108CC00019CA83A78905854517D5FF1F034585F870
:108CD0008297814769B797000000E780E0CBD5BF56
:108CE000FD573E858280411126C297A4FF1F9384C1
:108CF000E46FD84C22C437E404003C54484B06C609
:108D00008297DC4C0323C4052244B240924423AA38
:108D1000070017D5FF1F0345E5F385454101028391
:108D2000411126C297D4FF1F938484F29C4006C64B
:108D300022C44AC0D5C3DC43C5C35CC12300B5000F
:108D40002A84979501009385A5881775010013055E
:108D5000A57297600100E780A0C4294597600100D3
:108D6000E780E0C89C4023A4070023A2070097A740
:108D7000FF1F93876765DC4FDC4B91C72955970030
:108D80000000E78000DF97A7FF1F93872766DC4F6F
:108D9000DC4B89C797000000E78020F537E9040025
:108DA0008327C905894517D5FF1F0345A5EA829783
:108DB0008327C905914517D5FF1F0345A5E982976C
:108DC0009C4003A347016309030022852244B2406B
:108DD0009244024941010283B24022449244024932
:108DE000410182800111328506CE22CC26CA2E8412
:108DF00097300000E7802005AA84979501009385AD
:108E00006580177501001305256797600100E780ED
:108E100020B9030784000356640083554400A686E6
:108E2000179501001305058A97600100E78040B798
:108E3000294597600100E78080BB97A7FF1F83C784
:108E40000759639D9700014597000000E78060D2B5
:108E500081450A8597000000E780C0ECF24062443B
:108E6000D244056182806D71232481102326111064
:108E70002322911093F745002E84638707143C0842
:108E80003EC0B707E5003EC23C083EC423170100C0
:108E90002318010023190100231A0100231B0100DC
:108EA00097A7FF1F83D7475299E3C167FD17231682
:108EB000F10097A7FF1F83D7475191EB97D7FF1F6B
:108EC000938707D99C439C43DC4783D7070017A7A8
:108ED000FF1F1307674F2317F100544F83574700B5
:108EE0002318F100DC4AA1E7978501009385C57539
:108EF000177501001305455897600100E78040AAE7
:108F0000178501001305857697600100E78040A969
:108F1000294597600100E78080AD13454400832018
:108F2000C11003248110832441105161828097A7CE
:108F3000FF1F83C7D7492555D9C3FD1717A6FF1FA4
:108F4000A307F64803D6060183470701CC460A85E6
:108F5000230BF10097300000E78060DE97D7FF1FFA
:108F6000938707CF9C4317A7FF1F1307E7459786F3
:108F700001009386A67288430A866C009710000051
:108F8000E780601FAA8451D9978501009385C56B3E
:108F9000177501001305454E97600100E78040A05A
:108FA000A685178501001305256D97600100E780F0
:108FB000209F294597600100E78060A326859700E0
:108FC0000000E78000BB91BF93F725009DC7B7E77E
:108FD0000400BC47414681452808829725559700E3
:108FE0000000E78000B928089305F00F9700000003
:108FF000E78040D3134524001DB793F715000145C2
:1090000099DF97000000E78020991345140001BF05
:109010005C4D411106C688C317D7FF1F232AF7C22C
:10902000B7E7040083A70708170500001305E5E369
:109030008297B24097D7FF1F238EA7C001454101F9
:10904000828001113335A000A307A100B7E7040017
:1090500083A7471706CE1306F10085451305503048
:109060008297F240056182808280411122C406C647
:1090700097D7FF1F83C787BF014489EF97B7FF1FAB
:1090800083C71719054499E717C4FF1F0344845881
:1090900013441400228597000000E780C0FA17856A
:1090A00001001305257409E4178501001305857473
:1090B0002244B2404101176301006700638E797159
:1090C00022D4A30F010037E404008327841726D29B
:1090D0004AD006D6AA842E89130550309305F10193
:1090E00032C6829732468347F10193150601C1814A
:1090F00085CB01452EC697000000E780C0F483278A
:109100004417B2454A862685829705459700000098
:10911000E78060F3B2502254925402594561828034
:10912000832744174A8626858297EDB74111939786
:10913000050122C406C626C2C1872E8463D4070255
:10914000B7E40400FC5417A5FF1F0345252D8297A3
:1091500019C1BC5482972165218DB24022449244AA
:109160004101828093F715008DC7B7E7040083A7FC
:10917000471A17A6FF1F1306662997D5FF1F938569
:1091800025AE17A5FF1F03456529829713451400D7
:10919000E9B793F7250099CFB7E70400BC4F130652
:1091A0000064894517A5FF1F03454527829713458E
:1091B000240065B793F7850085CF97D7FF1F83C736
:1091C000A7AB85E7B7E7040003A8871A1307401F7A
:1091D00097A7FF1F83C7872481461306400699453A
:1091E00017D5FF1F0355C5A8029813458400B5B7CE
:1091F00093F745000145B5D3B7E4040083A70418ED
:1092000017D5FF1F0355C5A68297BC4C13060064F3
:10921000914517A5FF1F034565208297134544001C
:109220002DBF97D7FF1F83D7A7A46398A70217D78F
:10923000FF1F2310B7A417D7FF1F231DC7A217D7DF
:10924000FF1F231AD7A22E86178501001305C55FBD
:10925000BE85175301006700A3741785010013052D
:109260002560176301006700838B0357450097D77C
:10927000FF1F83D7E79F631EF704C1674111F917EA
:1092800022C417D7FF1F2325F79E37E4040097D782
:10929000FF1F23A1079E97D7FF1FA389079C97D77E
:1092A000FF1F238B079C7C4C06C6894517A5FF1F13
:1092B0000345C51682977C4C914517A5FF1F0345B2
:1092C000E51582972244B240410117030000670070
:1092D00003DA178501001305A5581763010067001D
:1092E00003847D15954763E2A71C178701001307C8
:1092F000274D0A053A951C41011122CC06CEBA979A
:109300002E8482871785010013050556976001009A
:10931000E780E080A1A203C7250099476311F70207
:109320002E8597000000E78080F483456400178550
:1093300001001305655497500100E780606697B7F8
:10934000FF1F238707EC178501001305A5547DBF78
:1093500003C7250095476319F702C16717D7FF1F99
:1093600003570791F91703D5A5006309F702B7E77B
:10937000040083A7C717829717850100130585523C
:1093800097500100E780A079854717B7FF1F230199
:10939000F7E817850100130565538DBF97D7FF1FA9
:1093A0002398A78C83D7E50097D6FF1F2393F68CCD
:1093B00083D7050197D6FF1F239EF68A83D7250101
:1093C00097D6FF1F2399F68A97D7FF1FA380078A96
:1093D000631BE502B7E70400BC4F0966130606905D
:1093E000A14517A5FF1F0345650382970356E400B7
:1093F0008355A400178501001305054C9750010003
:10940000E780005A51B79307700F2316F100B7E7B2
:10941000040083A7870D17A6FF1F034626006C00D4
:1094200082974DF9854717D7FF1FA301F7845DB7D2
:10943000178501001305454AD1BD83C52500914715
:109440006392F502178501001305854A97500100C4
:10945000E780E06C97000000E78060C1F240624462
:109460000561828099476392F5022285970000008A
:10947000E780E0DF83456400178501001305C53FE1
:1094800097500100E780C051D1BF9547639AF5001E
:1094900083471400E1F3178501001305A547BDB507
:1094A0001785010013058547E1BF8280411122C461
:1094B00017A4FF1F1304C4F7AA861786010013061A
:1094C000A6312285C14506C697500100E780606637
:1094D0000357440097A7FF1F938787F62393E7005E
:1094E000035764002394E700B24022444101828084
:1094F000411106C697000000E78080FBB7E7040033
:1095000083A7871417A6FF1F130686F2D5450145CA
:109510008297B2404D4697A5FF1F938565F21305CC
:1095200070304101170300006700A3B96171232463
:10953000811A37E40400832704082326111A232202
:10954000911A2320211B232E311917050000130522
:1095500025BE829717A9FF1F130949EC9947854437
:109560002300A900231CF100978501009385C52ADB
:109570009307400617750100130505F0231CF10839
:109580002308910097C9FF1F93892919975001005B
:10959000E780004183D50900178501001305C52622
:1095A00097500100E780C03F294597500100E780B0
:1095B000004403D50900896997000000E78040EF67
:1095C0008327441710088545130550308297832759
:1095D000441717A6FF1F1306A6E6CD4513057030E6
:1095E00082978327441717A6FF1F130666E3B54526
:1095F0001305603082978327441730088945130587
:10960000103182978327441730098945130520318B
:10961000829783274415938509900D458297832768
:1096200044159385099011458297A305910023065F
:1096300091002308910002CD230C0100832784169A
:1096400030099145130570408297832784161306CD
:10965000B10085451305004082978327841670006A
:109660008545130510408297832784163008854569
:10967000130520408297832784161008854513051B
:1096800050408297832704157D5582978327441382
:109690007D5582977D5597A0FFFFE78000FE8327C9
:1096A000440C829797A0FFFFE78060D9832784143A
:1096B00017A6FF1F1306C6D7D545014582978947D0
:1096C0001306700F814528092306F1009790FFFFCC
:1096D000E780E0A28D471306000881452808230C87
:1096E000F1089790FFFFE78080A19147230CF100DC
:1096F000977701009387C7C9984383C747003AC843
:10970000230AF10097D0FFFFE78060C6700085450F
:10971000054597A0FFFFE78060FD30099305700FB6
:10972000094597A0FFFFE78060FC3008930500081B
:109730000D4597A0FFFFE78060FB10089545114598
:1097400097A0FFFFE78080FAC16717C7FF1F1307C5
:109750002752F9171CC32322070017A5FF1F130563
:10976000A5CB97A0FFFFE78040F78327C41D17C54F
:10977000FF1F1305654E82973C4803450900854548
:1097800082978320C11A0324811A8324411A032952
:10979000011A8329C1195D618280C16717C8FF1F43
:1097A0000358084DF9176301F8083DCDB5CD0111F7
:1097B00026CAB7E4040083A7841222CC2E86231580
:1097C000B10006CE2A8401478146ED454285829745
:1097D0002AC611ED178501001305050597500100F4
:1097E000E780E033F2406244D24405618280FC4469
:1097F0000356A100A28582972C0017C5FF1F0355B1
:10980000254797A0FFFFE78000FA69DD1785010073
:109810001305C50297500100E780603083A7C4128A
:10982000ED45280082977DBF8280411106C61DC983
:10983000854717A7FF1FA30AF7BE354697A5FF1F49
:10984000938505BE1305603097A7FF1F238007BED1
:1098500097000000E780E086B24041011703000056
:109860006700E38097A7FF1FA38107BCF9B797C7DD
:10987000FF1F83C76740A9EFC16717C7FF1F0357C3
:10988000273FF9176306F7044111854722C417C71C
:10989000FF1F2303F73E37E404007C4C06C6A145B6
:1098A00017A5FF1F034585B782970323841A224417
:1098B000B24097A7FF1F83C767B617C5FF1F0355A1
:1098C000253B1307401F81463146994541010283DC
:1098D00082806D7123248110232611102322911080
:1098E000328401CD8947630AF5028320C110032425
:1098F0008110832441105161828017850100130576
:10990000A502AE8497500100E7806021A2852685DC
:1099100097C0FFFFE780C0C6C9BFB7E70400FC4798
:1099200028008297178501001305C5009750010094
:10993000E780E01E8347810039C41307000B638072
:10994000E7021387A7051377F70F8D4663EDE6024D
:10995000A285280097C0FFFFE780A03579B785472B
:10996000E3F587F88345910017750100130505E6B7
:10997000B335B00097A7FF1F238CB7709750010035
:10998000E78000029DB703479100A207D98F356792
:109990001307D7556385E7086368F7022D67130738
:1099A000B7556387E70631671307C755638AE7042E
:1099B00029671307A7556394E702A285280097C07B
:1099C000FFFFE780606D15B739679306E765638130
:1099D000D70863E9F6001307E7556384E706A28515
:1099E00028003DB73D679306F755638AD7061307EE
:1099F000F766E396E7FE97D0FFFFE780E085F5B5D1
:109A00000146A285280097C0FFFFE7802056F1BDE0
:109A1000A285280097C0FFFFE7804066F9B5894717
:109A2000E3F587EC97000000E780A0E49305E4FFEE
:109A3000C205C1811305A1009790FFFFE78040791F
:109A40006DB5A285280097C0FFFFE780E06571BD76
:109A5000A285280097C0FFFFE780A07079B597C066
:109A6000FFFFE780207951B5C16717C5FF1F035578
:109A70002520F9176307F500B7E7040003A3C7170C
:109A800002838280854717C7FF1F2301F71E014508
:109A900017F3FFFF6700235B1783FFFFE702836174
:109AA0002A8408452E89B28919C900C1971500007A
:109AB0009385A586610597300100E7808001814488
:109AC0007D5A97100000E780E03963C7A404814401
:109AD00097100000E780003A63C8A40497C7FF1FEF
:109AE0009387C7199C43DC47B307F940918723024A
:109AF000F400638309048327C900B307F440958702
:109B0000A302F4001C4C89C79C4799C32285829705
:109B10001783FFFF6700435D5C44139714008504BF
:109B2000BA972390470171BF1C481397140085040E
:109B3000BA972390070069BF832789000547B307B9
:109B4000F4409587A302F40083570400638EE70274
:109B50008DC309476384E7040D47E395E7FA9787C8
:109B600001009387E72F1CCC97870100938747302C
:109B700011A897870100938727F61CCC97870100CF
:109B8000938787F65CC8BDBF978701009387C7E1BD
:109B90001CCC97870100938727E2EDB797870100D8
:109BA0009387C7301CCC9787010093872731D9BF93
:109BB00095E51783FFFFE70283510046184483476A
:109BC000940075839D8B6317F70097100000E78062
:109BD00060B448C41783FFFF6700A35182801783D6
:109BE000FFFFE702234D13893500C164420941118B
:109BF000AA890144F11413590901054A2EC6971088
:109C00000000E7802026B2456348A40001454101D9
:109C10001783FFFF6700434D83A709001317140044
:109C2000BA9783D707006388B7006394970063747B
:109C30002A010504E1B70545D9BF1783FFFFE702F5
:109C40008346AA892E89328BB6843A8ABE8A97A027
:109C50000000E78020FB71C9268597200000E7807F
:109C600020098D4763E7A7007D551783FFFF670035
:109C7000034783DB440097100000E780A0242A8478
:109C800097100000E78040259307740031443305A6
:109C9000850263CDA70297100000E780A0229710ED
:109CA0000000E78020222A8497100000E780C0226D
:109CB0009307740031443305850263C3A7049710EA
:109CC0000000E78020209307450029A89710000096
:109CD000E7808020330585021307F0179307C0172C
:109CE000E35FA7FA2D55E3C277F963040B02D6862A
:109CF0005286A6854A8597200100E78020BAB5B72D
:109D000097100000E780401D330585029307C5FFCB
:109D1000D1BF832749001385C90083D52700970049
:109D20000000E78000EC61F581B769553DBF97C73A
:109D3000FF1F2397A7F497C7FF1F938727F490432C
:109D400081470C463307F500420741836393B70010
:109D500082805446139847008507C2962390E600F8
:109D6000D5B797C7FF1F938767F19C4303C587004B
:109D7000828017C5FF1F0355A5F082801783FFFF60
:109D8000E702E334C1671387D7FF630BE502636A19
:109D9000A700F1176300F50201451783FFFF670075
:109DA00043351387E7FF6302E502FD171D8D133569
:109DB0001500E5B797500000E780C0267D15C5BFA8
:109DC00097500000E78040FBD5BF97500000E78028
:109DD00060F9EDB71783FFFFE702632F4111AA84F3
:109DE00001442EC697100000E780C008B2456348C2
:109DF000A400014541011783FFFF6700832F9C48A2
:109E0000131514003E9583570500E385B7FE05043E
:109E1000C9BF03485500814693F7F60F63E5070174
:109E200081473E858280584593975600BA9703D75D
:109E300027006316B70003D70700E304C7FE8506B3
:109E4000E1BF8346450001479377F70F63E4D700EE
:109E5000814711A81C45131657000507B29703D672
:109E60000700E313B6FE3E8582801783FFFFE702FB
:109E7000632493170501C18797CAFF1F938A0AE0DD
:109E8000635BF00883A70A00C0479C4703570400A0
:109E9000198D420541816368F500014422851783CD
:109EA000FFFF6700632412052A94CDBFDC4713949B
:109EB0004900014A3E94834744006341FA02014A43
:109EC000834754006349FA028509C20993D90901FD
:109ED00083A70A009847E3EBE9FCC1B71C441319B8
:109EE0005A00A6853E994A8597000000E780C0EE9B
:109EF00005E1050AC9B75C4413195A00A6853E99C5
:109F00004A8597000000E78020ED19E1050A4DBF62
:109F1000E30C09FA61B7AA8481495DBF1783FFFF8B
:109F2000E702E31A1C452A8481E79307C5001CC594
:109F30001C44231204001CC09307F00F63EDB7000C
:109F400093F5F50F228597200000E78020E2178324
:109F5000FFFF6700031A93940501C167C18063F98D
:109F6000F500A685228597200000E78040E5C5B76B
:109F7000C18193F5F50F228597200000E78000DF6F
:109F8000A685228597200000E78040E0C9B797C7E3
:109F9000FF1F9387A7CE884382801C4599C797C728
:109FA000FF1F23ADA7CC014582807D55828097C7D6
:109FB000FF1F9387A7CC98438347450048479207E4
:109FC0003E9582801783FFFFE702631061710045B1
:109FD0001C183EC6B70780013EC81C183ECA8357EE
:109FE000440002CE02D002CC231EF100834784003D
:109FF0002A8902D22301F1023C083ED402D69700FE
:10A000000000E78000FB835705002316F1029750FC
:10A010000000E78060C42307A1025C400355640090
:10A02000F18313F717008347F10252055181F99B21
:10A03000D98FA307F10297100100E780807539CD11
:10A04000AA840355050097A00000E78080BC83D751
:10A0500004002AD26800231CF10083D72400231DAA
:10A06000F1001C4803D647008C4397200000E7808E
:10A0700000CD8347B400CA86178601001306468CBC
:10A080008117A305F4006C00481097200100E780B9
:10A09000E0805D611783FFFF6700A3052155D5BFF1
:10A0A0001C45B1CF03C5A700894613576500630B54
:10A0B000D7028D46630ED70285466300D702130789
:10A0C00040063305E50203C7B700418B15CB83C7B4
:10A0D000B700BD8B3355F54082801375F503130728
:10A0E000803EC5B709671375F50313070771D1BF24
:10A0F000372709001375F5031307077CD9B7014506
:10A1000082801783FFFFE70283FC03A98500630CAD
:10A1100009048347B900AE8493F7070E85C303454E
:10A120009900930520030D810505B305B502884408
:10A13000610597300100E780E0A935A02E859700E2
:10A140000000E78020F62A8419CD97000000E78000
:10A15000605C8325C900B307B54063FA87002E947D
:10A16000B305A440E9F51783FFFF670083F8854531
:10A170007DBF1783FFFFE70283F52A8403D505001F
:10A18000011132C636C43AC22EC002CA02CC02CE77
:10A1900097A00000E780E0A782452ACA22852ECC3E
:10A1A00097000000E780E0E003570500231EE10070
:10A1B00097500000E78040AAA24632469247230FFC
:10A1C000A10036874C08B286228501469700000020
:10A1D000E780E0A605611783FFFF670083F117831F
:10A1E000FFFFE702C3EE61711C183EC6B70780018E
:10A1F0003EC81C183ECA3C0800453ED4AA8402CC86
:10A2000002CE02D002D202D697000000E78060DAC8
:10A210008357050035592316F10297500000E78057
:10A22000A0A32307A10209C48357440081EB21594D
:10A230004A855D611783FFFF6700A3EB0355640048
:10A240005205518197100100E780A0542A8965D1F9
:10A250008347B40093F7070E99C71305840197301D
:10A260000100E780609983574400231EF100834773
:10A2700084002301F1025C4003550900D98313F7E0
:10A28000070883471102231CA10093F7F707D98F12
:10A29000A300F10283572900231DF1005C40F183E4
:10A2A00013F717008347F102F99BD98FA307F10237
:10A2B00097A00000E780E0952AD235D98347940023
:10A2C0006800139757008347B400FD8BD98FA3050F
:10A2D000F4001C4803D647008C4397200000E78019
:10A2E00000A6A68717770100130787657400054647
:10A2F0004C10268597000000E78060942A890DD9CC
:10A300008347B400A685FD8BA305F40097000000E9
:10A31000E78060DF31BF1783FFFFE70243DB832461
:10A3200085FE2A844111268597000000E78080D7AA
:10A33000834734FF93F7070E8DCB2AC626859700F7
:10A340000000E78060C809CD834734FFB245FD8B2C
:10A35000A309F4FE91C5228597300100E78080872C
:10A3600041011783FFFF6700C3D87DD98327C4FF4E
:10A370002685829775F5834734FF93F7070E91C7BB
:10A38000228597300100E7802087032584FE97000F
:10A390000000E78000E5E9B71783FFFFE70223D05D
:10A3A0009C4141112A8903C7070089472E8493568F
:10A3B00067006380F6040D466388C6049307F007C0
:10A3C0006304F7022E8597200000E780C0A7AA84C7
:10A3D0008149C16B130C490097C7FF1F9387078AF8
:10A3E0009C43984763E4E90441011783FFFF67003A
:10A3F000C3CE03D745008547E3F8E7FE2E859720B7
:10A400000000E780A0A9E1B703D74500E3FEE7FC21
:10A410002E8597200000E78000A3AA84228597203C
:10A420000000E78060A4C204C98C5DB7DC47035517
:10A43000A900139A49003E9A93170501C187635DED
:10A44000F00083570A006397A70263E7740383272A
:10A45000CA00034D5A002DA0A1672167A98F1307D9
:10A46000F7EFE374F7FE6397090097000000E780B9
:10A47000209161FD85098DB783278A00034D4A002D
:10A48000835DA90003576900216A138BC7003AC690
:10A49000814A33CA4D01631E5D0197B7FF1F938741
:10A4A000677E9C43E1DBA286628681452685829792
:10A4B000D1B7A1679387F7EF930C4BFF63F2470384
:10A4C000B2455A8597F0FFFFE780A0710DC10327C1
:10A4D0008B00104709CE10436382C4023107D5BFF9
:10A4E000EE85668597000000E780008F71F99386FE
:10A4F0001A0093FAF60F130B0B0271BF8356440038
:10A500005C43E3E9F6F622853AC697100000E7803F
:10A51000807DA1679387D7042A8A035D4400324770
:10A5200063E897008347D90093E707F8A306F9008B
:10A530001C4766852286E2858297C1670844FD171D
:10A54000337AFA00529508C02312A40125B797B7B1
:10A55000FF1F9387A7729843814715C3144781470C
:10A5600063FFD500939745004C47BE9519C903C7B3
:10A57000550081476375E600DC451606B2973E85B7
:10A58000828003C745008147E37BE6FE16069C45B3
:10A59000F5B71783FFFFE702E3B1AA892E8A81444A
:10A5A00097BAFF1F938A8A6D83A70A00984763E6CC
:10A5B000E4001783FFFF670023B3DC4713944400D4
:10A5C00001493E9413BB140083474400634BF900D8
:10A5D000014913BB140083475400634FF9008504FD
:10A5E000E1B70844931759005287DA860146A285DD
:10A5F0003E9582990509C9BF48449317590052876F
:10A60000DA860546A2853E9582990509E9B7178342
:10A61000FFFFE702C3AB814517F5FFFF13050548B0
:10A6200097B7FF1F239E076497000000E780A0F6FE
:10A630001783FFFF6700E3AB97B7FF1F938707649C
:10A640009C4395C31783FFFFE70263A8814517F575
:10A65000FFFF1305A54497000000E780C0F31783B0
:10A66000FFFF670003A982801783FFFFE70283A42F
:10A6700037E404008327841241112315E100AE89D9
:10A680003289368A3A8681460147ED45AA84829707
:10A690002AC621C90356A100D28597400100E78050
:10A6A000C0248327C413CE8526858297058905C9D2
:10A6B0008327440D2314210101462C00268582970F
:10A6C0002A8401C9B7E7040083A7C712ED45280013
:10A6D0008297228541011783FFFF6700E3A0494469
:10A6E000D5B76554FDB75C41FD175CC18280178307
:10A6F000FFFFE702C39DB7E70400FC5F8297954721
:10A700003305F50281450D811783FFFF6700639EC6
:10A710001783FFFFE702A39BB7E70400FC5F829764
:10A7200095473305F5020D811783FFFF6700639C92
:10A730001783FFFFE702A399B7E7040083A7870BFE
:10A740000355050082971783FFFF6700839A1783DD
:10A75000FFFFE702C397035505003287AE861796C1
:10A76000FF1F035606D497B5FF1F9385E551970049
:10A770000000E780A0EF1783FFFF67008397178330
:10A78000FFFFE702C394B7E7040083A7C7178297C8
:10A790001783FFFF6700E3951783FFFFE70223930B
:10A7A000B7E7040083A7871397B5FF1F9385C54DAF
:10A7B000829701451783FFFF6700A3931783FFFF6D
:10A7C000E702E390B7E7040083A7C71F8145179509
:10A7D000FF1F035505C982971783FFFF6700639129
:10A7E0001783FFFFE702A38EB7E7040083A7871351
:10A7F00097B5FF1F9385454A829701451783FFFF51
:10A800006700238F1783FFFFE702638CB7E704001D
:10A8100083A7C71F81451795FF1F035585CA8297D8
:10A820001783FFFF6700E38C1783FFFFE702238A8C
:10A830002E8597800000E780E0AF97800000E780DA
:10A84000E0EC1783FFFF6700C38A1783FFFFE7026F
:10A85000038897800000E780E0F61783FFFF67001A
:10A8600043895C49E1175CC95CC583572501A10791
:10A870002319F50083570501A1072318F5008280ED
:10A88000F1473305F50297B7FF1F9387E7429C43D3
:10A890003E9582808D476315F60803D746008547AD
:10A8A00063F0E7081783FFFFE7026382368536848B
:10A8B0002E8997100000E780005929C9835744006A
:10A8C00093140501C18063E397042285971000006B
:10A8D000E7806057FD14231294009307A0026300E1
:10A8E000F5029307B0026307F50293079002631F16
:10A8F000F500228597000100E780C08501A8014688
:10A90000CA85228597A00000E78060B01773FFFF1B
:10A910006700237E228597100000E780C003FDB703
:10A92000828097B6FF1F938666399C42014599CF76
:10A930009843D44217B6FF1F2322E6386396D70008
:10A9400097B6FF1F23AEE6361385C7FE82801773C6
:10A95000FFFFE702C37797000000E780A04B714438
:10A9600033058502914597900000E78020E911E5C5
:10A9700065551773FFFF6700C37797B7FF1F23ABBA
:10A98000A73297000000E780E04833058502914533
:10A9900097900000E78080E661DD97B7FF1F23AD49
:10A9A000A73097000000E780E04697B7FF1F239D80
:10A9B000A72E97000000E780E04597B7FF1F23967A
:10A9C000A72E977701009387E7FC17B7FF1F232176
:10A9D000F72E97070000938707E917B7FF1F232774
:10A9E000F72C014579B71773FFFFE702436EAA857D
:10A9F00017B5FF1F1305452B97100000E780C05BBC
:10AA00001773FFFF6700E36E1773FFFFE702236C06
:10AA100097000000E78060FD97100000E780405B32
:10AA200097B7FF1F938787299C4391CF1387C7FE52
:10AA300019CB83D5C7FF17B5FF1F1305A52897208E
:10AA40000100E78020191773FFFF6700836A1773FF
:10AA5000FFFFE702C36797000000E780C0EC09CD65
:10AA6000834785002A8493F7070499EB0355E50093
:10AA700097000000E78080F91773FFFF67006367A6
:10AA80008347C5009304450117B9FF1F1309092324
:10AA900085E3832709005CC997B7FF1F23A097228E
:10AAA00083274900F1FB97B7FF1F23AB9720E9B736
:10AAB000FD172306F500610597800000E780C0D6EA
:10AAC0008307840063CB07048347840093E707F878
:10AAD0002304F400B7E704009C5F82974205A9476E
:10AAE00041813375F5028347840093F707FCC98FD2
:10AAF0002304F4008347D4003E951C402318A4008F
:10AB000089CF984319CB8347C400504081458507BE
:10AB10003305F502420541810297832709005CC88D
:10AB200097B7FF1F23AC97188327490089E797B78A
:10AB3000FF1F23A797188347C4009DDF8355040197
:10AB400017B5FF1F1305051897200100E78080083F
:10AB500025B71773FFFFE702835797B7FF1F938748
:10AB6000A73B9C4701448583858B85E3AE84B285F2
:10AB70003A8697100000E780804B2A8419C5971009
:10AB80000000E780C041829408CC22851773FFFF44
:10AB9000670023561773FFFFE702C35141112E8947
:10ABA00032C6AA8997000000E780C03132471306F9
:10ABB0000502CA86970500009385C5CC17B5FF1F0F
:10ABC0001305850E97000000E780E0F82A8425C968
:10ABD0009304C50097000000E780E0411946AA856C
:10ABE000268597100000E7808015854526859710FB
:10ABF0000000E780601117750100130565D74E95B9
:10AC000083450500268597100000E78020165C48E4
:10AC100031468145A1075CC85CC483572401E11714
:10AC20002319F40083570401E1172318F4001C4C86
:10AC30003E859770FFFFE780804CA30425012285A5
:10AC400041011773FFFF6700234A1773FFFFE702F5
:10AC500003484111AA842EC632C497100000E78031
:10AC60006036004DB2452246834784000CC050C078
:10AC700093F7F70393E707042304F4002318040071
:10AC8000268597100000E780803183479400A9460D
:10AC90002317A40013D7370005073307D7029D8B6E
:10ACA00085072306F400A306E40083C70401D848FF
:10ACB0008507230FF7FE17B7FF1F13072700584319
:10ACC000232A04009307440129E317B7FF1F232910
:10ACD000F7FE17B7FF1F2323F7FE17B4FF1F130458
:10ACE00064FE228597200100E78000E11C44858BEB
:10ACF0005D8D19E58145228597200100E78080ED73
:10AD000041011773FFFF6700C33E1CC317B7FF1F46
:10AD10002328F7FAD9B71773FFFFE702433B9705DC
:10AD20000000938565B7014597000000E78000B0FB
:10AD300001451773FFFF6700C33B1773FFFFE7026F
:10AD4000033997000000E78080B01773FFFF6700AA
:10AD5000433A8347C500A5E31773FFFFE702233794
:10AD60002A840355E50097000000E78000C821C150
:10AD70008347840093F7F7FB2304F4001C4091C73A
:10AD8000DC4381C74C400145829797000000E78073
:10AD900080B917B5FF1F1305E5F297200100E78082
:10ADA000A0E50355E40097000000E78020C6177374
:10ADB000FFFF6700033482801773FFFFE702233130
:10ADC00097B7FF1F938787EF97050000938565C8A6
:10ADD00017B5FF1F130505EF23A0070023A20700E7
:10ADE00097200100E780E0CE1773FFFF6700633014
:10ADF0001C4D91CFDC4381CF1773FFFFE702232D5A
:10AE00008345070082971773FFFF6700832E8280B8
:10AE100097B7FF1F938747ED9C4303C507008280C8
:10AE200097B7FF1F938747EC9C4303C517008280A9
:10AE300097B7FF1F938747EB9C4303C5270082808A
:10AE400097B7FF1F938747EA9C4303C5470082805B
:10AE500097B7FF1F938747E99C4303C5370082805C
:10AE600097B7FF1F938747E89C4303C5570082802D
:10AE700097B7FF1F938747E79C4303C5670082800E
:10AE800097B7FF1F938747E69C4303C577008280EF
:10AE900097B7FF1F938747E59C4303C587008280D0
:10AEA00097B7FF1F938747E49C4303C597008280B1
:10AEB00097B7FF1F938747E39C4303C5A700828092
:10AEC00097B7FF1F938747E29C4303C5B70011E183
:10AED0001D45828097B7FF1F938707E19C4303C5F9
:10AEE000C700828097B7FF1F938707E09C4303C585
:10AEF000D700828097B7FF1F938707DF9C4303C566
:10AF0000E700828097B7FF1F938707DE9C4303D536
:10AF10000701828097B7FF1F938707DD9C4303C516
:10AF20002701828097B7FF1F938707DC9C4303D5D7
:10AF30004701828097B7FF1F938707DB9C4303D5A8
:10AF40006701828097B7FF1F938707DA9C4303D579
:10AF50008701828097B7FF1F938707D99C4303C55A
:10AF6000A701828097B7FF1F938707D89C4303C52B
:10AF7000B701828097B7FF1F938707D79C4303C50C
:10AF8000C701828097B7FF1F938707D69C4303C5ED
:10AF9000D701828097B7FF1F938707D59C438857B7
:10AFA000828097B7FF1F938727D49C4303D5C7029E
:10AFB000828097B7FF1F938727D39C4303D5E7026F
:10AFC00019E11305800C828097B7FF1F9387C7D1C3
:10AFD0009C4303C50703828097B7FF1F9387C7D0A1
:10AFE0009C43C85B828097B7FF1F938767CF8843D6
:10AFF000828097B7FF1F9387E7CE8843828019E14D
:10B000007D558280F5DE984265DFFDD917B7FF1FB9
:10B01000130787F01847AA877155058B631D07240E
:10B0200003C507001547E37DA7FC03C737001305D9
:10B03000F0057D171377F70FE364E5FC03C35700B2
:10B04000E30003FC83C86700E38C08FA03C77700BA
:10B05000494579171377F70FE364E5FA03C7A700AB
:10B0600011481305F7FF1375F50FE36BA8F803CE2E
:10B0700097000D481305FEFF1375F50FE362A8F85E
:10B0800003C8B7006309080065181378F80F1305A3
:10B09000600DE36705F703C5C70079487915137597
:10B0A000F50FE36FA8F403C8D7000D457D1813789A
:10B0B000F80FE36705F503D80701930E4017511801
:10B0C000420813580801E3ED0EF303C8E7007D18AA
:10B0D0001378F80FE36605F303C827017D1813788A
:10B0E000F80FE36F05F103C88700C54E7518137894
:10B0F000F80FE3E70EF103D86701856E938EBEE08B
:10B100006D18420813580801E3EC0EEF03D847010D
:10B110006D18420813580801E3E40EEF03D88701C5
:10B120007918420813580801E36C05ED03C8A7011C
:10B130007D181378F80FE36505ED03C5B7011D48C9
:10B140007D151375F50FE36DA8EA03C5D7017148A6
:10B1500079151375F50FE365A8EA03D5E701130820
:10B16000E00F7D1542054181E36CA8E803C50702A5
:10B17000494879151375F50FE364A8E8C85301C968
:10B1800037C834005915130858BFE36BA8E603A865
:10B19000870237C53400130555BF5918E36205E728
:10B1A00017B5FF1F2320C5B403C6050117B5FF1F40
:10B1B000232CF5B20545E375C5E403D82501D04934
:10B1C00033760603E31E06E203C61501E30A06E230
:10B1D00017B6FF1F2326B6B083C527000146638735
:10B1E000A50003C61700F1453306B60283C707035F
:10B1F0009305C00272971A071307C70516031A971B
:10B2000096084697B387B70241553E973297420753
:10B2100041836362E8061773FFFFE70243EB36855D
:10B2200097800000E780A06897000100E780204831
:10B230002A8497A00000E780805A2A9497F00000A3
:10B24000E78060262A9497900000E780A0812A94E6
:10B2500097F0FFFFE780E06F2A9497400000E780B7
:10B2600060932A9497700000E780A09C2295177342
:10B27000FFFF670003E882801773FFFFE70223E503
:10B280004111A307A10097A00000E780A0C5930586
:10B29000F100170500001305E5B597F0FFFFE78003
:10B2A000802F014541011773FFFF670083E4177387
:10B2B000FFFFE70243DF17B4FF1F1304E4C50328B1
:10B2C000840079599368180097B4FF1F23AA14C506
:10B2D0001378180063100802BA84BE89368B328A4C
:10B2E0002E89AA8A97F0FFFFE780E0A77D152695B3
:10B2F00019E531594A851773FFFF670043DE97F060
:10B30000FFFFE78040A67D152695A167E353F5FE74
:10B3100097B7FF1F938707F798433E8C814B01CB6C
:10B32000014597F00000E7802044933B15004A85D3
:10B33000DA865686D28597900000E780C04D2A892C
:10B3400011CD1C44F99B17B7FF1F232BF7BC832794
:10B350000C00CDD3E3800BFA829769BF268597B79F
:10B36000FF1F23AD07BA97F0FFFFE780809C41469F
:10B37000CE8517B5FF1F1305A5C397300100E780E1
:10B38000C05697D00000E78040990325040B97D062
:10B390000000E780009D054597D00000E78000A4ED
:10B3A000054597000000E78060EDA9B797B7FF1F3C
:10B3B000938787B69C47858BEDC71773FFFFE7021E
:10B3C00003D117B5FF1F1305E5BC97B7FF1F23A5D2
:10B3D00007B497B7FF1F23A307B497B7FF1F23A195
:10B3E00007B497200100E780208197500000E78094
:10B3F000E0F597100100E780A04C97100100E7806E
:10B40000A05297B7FF1F9387A7AF9C4391C70545ED
:10B4100097800000E780402097B7FF1F9387079829
:10B420009C4399C741657D1597700000E78040A255
:10B4300097F00000E780E03D97D00000E780808F24
:10B4400097B7FF1F938707C29C4313971701635653
:10B45000070097F00000E78000AD97B7FF1F23A912
:10B4600007B497B7FF1F23A707B497B7FF1F23A5FC
:10B4700007B497B7FF1F23A307B497000000E78026
:10B48000008C97000000E780007297F0FFFFE780D4
:10B49000401897F00000E78040D61773FFFF670061
:10B4A00043C5828097B7FF1F938707A78843828091
:10B4B0001773FFFFE702A3C197800000E780607564
:10B4C00097800000E780C0771773FFFF670063C2B3
:10B4D0001773FFFFE70203BE2A84930414020111CD
:10B4E0002E85B289A685214636C63A899730010055
:10B4F000E780403D0DE9B24638082686CE85130523
:10B50000940497500000E780604121462C084A854A
:10B5100097300100E780003B133515000561177374
:10B52000FFFF670063BC0145D5BF1773FFFFE7024C
:10B5300003BA9305450617A5FF1F1305257B971032
:10B540000100E78020691773FFFF670083BA177354
:10B55000FFFFE702C3B741112EC697F0FFFFE78058
:10B56000601BB24588C141011773FFFF670063B8D4
:10B570001773FFFFE70203B4AA842E8497800000AC
:10B58000E780006CAA898545228597000000E78046
:10B59000E07D83C7E4011389940899E313890403C8
:10B5A000CE85228597000000E780407C21469305E8
:10B5B0001902228597000000E780607897B7FF1F87
:10B5C000938787958C43228597100000E780C0827F
:10B5D000214693858402228597000000E78020762B
:10B5E0001773FFFF670043B01773FFFFE702A3ABBA
:10B5F000397197F00000E780E0B49305400661E9F7
:10B6000097800000E78000606302051497A7FF1F82
:10B6100083C7876F13B7170097A6FF1F2386E66EB1
:10B62000014499CFC16417B9FF1F1309E98E93092B
:10B63000400EFD1497000000E780C0866342A40A14
:10B6400097F0FFFFE780000D4169B7290900096AFB
:10B65000FD7A2A8B81447D199389F97B130A0A713B
:10B66000938A8AC797000000E780C08363D7A40449
:10B670001304400EB387840217B7FF1F1307C7894F
:10B680000324070B3E948357C4016382270B1840A1
:10B690003307EB4063EAE900834744008507B3873B
:10B6A0004703D6976365F70801468145094597F03A
:10B6B000FFFFE780604EAA8B29E597400000E780F6
:10B6C000808385476317F50689659385057117A5FE
:10B6D000FF1F1305A56197100100E780A04F95A0FB
:10B6E000B30734030327090BBA9703D7C7016308CD
:10B6F000970003C75700A38207002382E7000504D1
:10B7000015BF9305C500228597000000E78080E6FD
:10B710005E852286976501009385C52697F0FFFF19
:10B72000E780E0525E8597100000E780608A85041C
:10B7300015BF97A7FF1F9387277E9C478D83858B17
:10B74000C1F721611773FFFF6700639901468545C3
:10B75000094502D002D202D402D697F0FFFFE7805B
:10B76000A043AA8479DD97F00000E780E09C13896C
:10B77000C4002A8481454A8597000000E780005F65
:10B780000C4041464A8597000000E780405B8329D2
:10B7900044006385090C4E8502D802DA02DC02DE21
:10B7A00097300100E78060402ACE141005462C082F
:10B7B00008184ECC97500000E780E00A1375F50F8B
:10B7C00051ED8355840093E525004A8597000000DC
:10B7D000E780E05E11460C104A8597000000E78084
:10B7E00000560146976501009385451A268597F016
:10B7F000FFFFE780C045268597000000E780407D79
:10B800005C40A1D3014685450D4597F0FFFFE780D9
:10B81000A038AA841DD548401389C4009730010080
:10B82000E780A0382AC64A8597000000E780404C90
:10B830003246636FC5004C404A8597000000E780A0
:10B84000005001468145268597F0FFFFE7802040A4
:10B85000268597000000E780A077E5B58355840032
:10B86000ADB71773FFFFE702838697A7FF1F938784
:10B87000A76A9C471DC193E7870017A5FF1F130503
:10B88000E54617A7FF1F232DF76897100100E780F3
:10B8900040321773FFFF6700C385DD9B17A7FF1FAB
:10B8A0002320F76897300000E780E0647DF117A55A
:10B8B000FF1F1305A54397100100E780E033D1BFB8
:10B8C0001763FFFFE702237E4169AA892E8AB28AA5
:10B8D000368BBA8B814417ACFF1F130CEC63930CAF
:10B8E000400E7D1997F0FFFFE780C05B63C4A400A2
:10B8F00001443DA03384940383270C0B3E9483576B
:10B90000C401638627055A87D6865286CE851305DD
:10B91000040397000000E780E0BB01C923800B000F
:10B9200022851763FFFF6700837B8347F40185C38C
:10B930005A87D6865286CE85130594089700000054
:10B94000E78040B909C585472380FB00D1BF850446
:10B9500051BF835745006380071E1763FFFFE7024F
:10B96000637501112A8497000000E780C04D09C962
:10B9700085476309F50605611763FFFF6700C37616
:10B9800097E00000E780007C7DF58357440049473D
:10B99000ED9BE392E7FEC145228597000000E7801A
:10B9A0004033AA84228597000000E780204F035788
:10B9B000440002CE91472A89631AF7002285970036
:10B9C0000000E780A0513C082ACC3ECE97E0000062
:10B9D000E78080765C55C5D374084A86A685054500
:10B9E000829751BF03574400D147E3F6E7F8032A93
:10B9F0000400C169014997AAFF1F938AEA51130BFA
:10BA0000400EFD1997F0FFFFE780C049634FA90E74
:10BA10002285032A040097000000E780C042A14568
:10BA20002A89228597000000E780A02AAA8422851F
:10BA300097000000E780804A14402A86AA89780887
:10BA40002685CA8597000000E780C0E7AA8405D54F
:10BA500003C7F40189476315F7008347C10181DFFC
:10BA60005546D2851385640097300100E780E0E7F2
:10BA7000014597800000E780C01901C583D7C40144
:10BA8000A5E797A7FF1F938727499C479355190060
:10BA9000858913D73700058B01CF8983858B6399FF
:10BAA000B70001452EC697000000E780C0DBB24515
:10BAB0004E8597800000E780601F0346C1012A84FD
:10BAC00093751900268597900000E780E03935C10D
:10BAD000268597800000E780E018268511C0014583
:10BAE00097800000E780004C97300000E780A0407E
:10BAF0008547E312F5E883C754001307F00FE38C82
:10BB0000E7E68507A382F400BDB5B304690383A704
:10BB10000A0BBE9483D7C401638B37015546D28587
:10BB20001385640097300100E780C0D955DD050911
:10BB3000D1BD5DD86DB782801763FFFFE7028357E1
:10BB400097800000E780000C05C1C164014417A97B
:10BB5000FF1F1309693C9309400EFD1497F0FFFF86
:10BB6000E7804034634EA40017A5FF1F1305051896
:10BB700097100100E780E0031763FFFF6700C356DB
:10BB8000330534038327090B3E958357C50163882A
:10BB900097002312050097800000E780A00C0504A1
:10BBA00075BF97A7FF1F938727379C478D83858B8A
:10BBB0008DE31763FFFFE702835117A5FF1F1305EE
:10BBC000E51297100100E78020031763FFFF67006D
:10BBD000435282801763FFFFE702634F970500001F
:10BBE0009385C5A017A5FF1F1305451097100100E9
:10BBF000E78020EE1763FFFF6700A34F1763FFFF87
:10BC0000E702E34C8841B7E70400BC5B0505420549
:10BC10004181829709C585472300F5000505176313
:10BC2000FFFF6700034D83C7F5FF2E858507A38FB0
:10BC3000F5FE828083C7F5FFFD1793F7F70FA38FFB
:10BC4000F5FE99EF1763FFFFE7026348B7E70400CB
:10BC5000BC571385F5FF82971763FFFF67006349A1
:10BC600082801C41035745008D8FBA951CC1231259
:10BC7000B5003E85828093D78500A2051441DD8DF5
:10BC8000835745001387E6FF18C189072312F50083
:10BC900013D685004111238FB6FEA38FC6FE410146
:10BCA000828018419307F7FF1CC183574500850721
:10BCB0002312F500A30FB7FE8280835745008D8FB6
:10BCC0002312F5001C41BE950CC12E858280AA87E7
:10BCD00003D7470008410D8FAA952392E7008CC334
:10BCE0008280184108453305A7408280835745006C
:10BCF000035765001D8F1C4108453385A740330558
:10BD0000A74082801763FFFFE702633C41112EC604
:10BD10002A8497000000E780A0FDB2456373B50058
:10BD200001A0835744000840BE952312B4003E95FD
:10BD300041011763FFFF6700C33B1763FFFFE70283
:10BD4000033941112E84B28532C697000000E78086
:10BD5000A0FB3246A28597300100E78000B941017F
:10BD60001763FFFF6700E3381763FFFFE70223361F
:10BD70002E84854597000000E78000F923008500A8
:10BD80001763FFFF6700E3361763FFFFE702233403
:10BD900041112317B100894597000000E780C0F6E4
:10BDA0008347E1002300F5008347F100A300F5007D
:10BDB00041011763FFFF6700C3331763FFFFE7020B
:10BDC000033193D78500A2054111DD8D2317B10002
:10BDD000894597000000E78020F38347E1002300B6
:10BDE000F5008347F100A300F50041011763FFFF51
:10BDF000670023301763FFFFE702632D1397850168
:10BE000093D78501C166938606F0D98F13D7850035
:10BE1000758FD98FA2053707FF00F98D4111DD8D90
:10BE20002EC6914597000000E78000EE6C00114699
:10BE300097300100E78060AB41011763FFFF6700A7
:10BE4000432B1763FFFFE70283281C41854503C48A
:10BE5000070097000000E78080E622851763FFFF58
:10BE6000670023291763FFFFE70263261C41411186
:10BE7000894503C7070083C717002307E100A3070D
:10BE8000F10097000000E78080E30355E1004101E5
:10BE90001763FFFF6700E3251763FFFFE702232314
:10BEA0001C414111894503C7070083C717002307B9
:10BEB000E100A307F10097000000E78040E083570E
:10BEC000E100410113D58700A2075D8D4205418144
:10BED0001763FFFF6700E3211763FFFFE702231FDC
:10BEE0000C4141112A841146680097300100E78017
:10BEF000C09F9145228597000000E78040DCB24753
:10BF0000C166938606F01397870113D58701598D73
:10BF100013D78700758F598DA2073707FF00F98F58
:10BF20005D8D41011763FFFF6700A31C1C45BE9593
:10BF30000CC18280AE87944391E6584101EF0CC159
:10BF40005CC1828003C7570013671700A382E70014
:10BF5000B687D5B70CC3EDB7AA87084119CD1841EC
:10BF6000D44398C36313D500D8C32A870346570028
:10BF70009376160081E6232007008280944381CACD
:10BF80008C4203A847008CC363930601CCC3799A03
:10BF900014C3A302C7003687D1BF1C45DC471D8DE3
:10BFA000B777DBB6938777DB09853305F502420562
:10BFB00041818280F147B385F50248452E95828004
:10BFC0008347450085072302F50082801763FFFF42
:10BFD000E702E30F2A8409E41763FFFF6700631198
:10BFE00083474400F5DBFD1793F7F70F2302F400B6
:10BFF000E5F71C4403D7270005072391E700DC433E
:10C0000099C3228582974C4889CD83475400898BF8
:10C0100099E71C4422859C479C439C478297232A8E
:10C0200004000040232004007DB71763FFFFE702F0
:10C03000030A8357250041112EC681EB0144228556
:10C0400041011763FFFF6700C30A035705008147DB
:10C05000F146E305F7FEB385D702404585072E94E8
:10C060008345440008C4F5F5B247AA8481E7232A32
:10C07000040009A81C456C0022859C439C438297C0
:10C0800048C84DDD85472312F400B2472320040041
:10C09000231804002319F4005C485CC483D72400EF
:10C0A000FD172391F40061BF1763FFFFE70223022E
:10C0B00097A7FF1F938787C588432326050023245E
:10C0C0000500410597100100E78000B31763FFFFEB
:10C0D000670023021763FFFFE70263FF17A4FF1F38
:10C0E0001304C4C21C40411199CF9C472300B500E2
:10C0F0002AC65CC197000000E78040FB1C40DC437F
:10C1000099C33245829741011763FFFF670063FEC1
:10C110000347450029E3584DAA877D551DCF176376
:10C12000FFFFE702C3FA1CC3DC4797A6FF1F23AF3C
:10C13000E6BCF156130507012390D70097050000D0
:10C140009385050297100100E780A09801451763C9
:10C15000FFFF670003FA7D55828082801763FFFF2F
:10C16000E702E3F601116146814528009760FFFF71
:10C17000E780E0F897A7FF1F938747B99C43280003
:10C180009305F00FDC473EC697000000E780C0F43F
:10C1900005611763FFFF6700C3F597A7FF1F93872C
:10C1A000E7B69C43D847A1679387C702631EF70A87
:10C1B000397106DE22DC26DA80004AD84ED652D407
:10C1C00056D23285B28497000000E780C0C7AA89A2
:10C1D000268597000000E78020C92318A4FC268547
:10C1E00097000000E78040C82319A4FC268597002B
:10C1F0000000E78060C783D744000A8A231AA4FCA2
:10C20000858393F7F70F230EF4FC8607BD0793F79A
:10C21000073F3301F1408A8A01498347C4FD6367C0
:10C22000F902CE85130584FC232C54FD97000000F1
:10C23000E78080EA5281130104FCF2506254D25428
:10C240004259B259225A925A21618280268597001A
:10C250000000E78060C193171900D6970509239065
:10C26000A7001379F90F55BF828097A7FF1F938707
:10C27000E7A99C43D847A1679387A702631AF70AE7
:10C28000397106DE22DC26DA80004AD84ED652D436
:10C2900056D23285B28497000000E780C0BAAA89DE
:10C2A000268597000000E78020BCFD572318A4FCDA
:10C2B00026852319F4FC97000000E780E0BA83D7B5
:10C2C00044000A8A231AA4FC858393F7F70F230EF0
:10C2D000F4FC8607BD0793F7073F3301F1408A8AD4
:10C2E00001498347C4FD6367F902CE85130584FCC9
:10C2F000232C54FD97000000E78000DE52811301DB
:10C3000004FCF2506254D2544259B259225A925A01
:10C3100021618280268597000000E780E0B49317B2
:10C320001900D69705092390A7001379F90F55BF77
:10C33000828097A7FF1F9387679D9C43D847A1677B
:10C3400089076310F70A397106DE22DC26DA8000DD
:10C350004AD84ED652D456D2328532899700000040
:10C36000E78060AEAA894A8597000000E780C0AFE9
:10C37000835749000A8A2318A4FC858393F7F70F93
:10C38000230CF4FC8607BD0793F7073F3301F14008
:10C390008A8A8144834784FD63E7F402CE851305CE
:10C3A00084FC232A54FD97000000E780E0D25281EC
:10C3B000130104FCF2506254D2544259B259225A29
:10C3C000925A216182804A8597000000E780C0A9C7
:10C3D00093971400D69785042390A70093F4F40F45
:10C3E00055BF828097A7FF1F938747929C43D847EA
:10C3F000A1679387E704631EF70A397106DE22DC22
:10C4000026DA80004AD84ED652D456D23285B2842B
:10C4100097000000E78020A3AA89268597000000E6
:10C42000E78080A42318A4FC268597000000E780FD
:10C43000A0A3231AA4FC268597000000E780C0A2D1
:10C4400083D744000A8A2319A4FC858393F7F70F46
:10C45000230EF4FC8607BD0793F7073F3301F14035
:10C460008A8A01498347C4FD6367F902CE851305B3
:10C4700084FC232C54FD97000000E780E0C5528126
:10C48000130104FCF2506254D2544259B259225A58
:10C49000925A21618280268597000000E780C09C27
:10C4A00093171900D69705092390A7001379F90F60
:10C4B00055BF828097A7FF1F938747859C43D84726
:10C4C000A1679387C704631AF70A397106DE22DC75
:10C4D00026DA80004AD84ED652D456D23285B2845B
:10C4E00097000000E7802096AA8926859700000023
:10C4F000E7808097FD572318A4FC2685231AF4FCB7
:10C5000097000000E780409683D744000A8A2319E9
:10C51000A4FC858393F7F70F230EF4FC8607BD0771
:10C5200093F7073F3301F1408A8A01498347C4FDED
:10C530006367F902CE85130584FC232C54FD970014
:10C540000000E78060B95281130104FCF25062548C
:10C55000D2544259B259225A925A21618280268578
:10C5600097000000E780409093171900D6970509BF
:10C570002390A7001379F90F55BF82809797FF1F6B
:10C580009387C7789C43D847A167DD076317F704F3
:10C590001763FFFFE702A3B37971328532849700F6
:10C5A0000000E780408A2AC6228597000000E780C5
:10C5B000A08B2311A102228597000000E780A088AC
:10C5C000B2452300A102280897000000E780C0B010
:10C5D00045611763FFFF6700C3B182809797FF1F14
:10C5E0009387C7729C43D847A167938787046317D3
:10C5F000F7041763FFFFE70283AD79713285328458
:10C6000097000000E78020842AC62285970000005A
:10C61000E78080852311A102228597000000E78032
:10C620008082B2452300A102280897000000E7801D
:10C63000A0AA45611763FFFF6700A3AB82809797AD
:10C64000FF1F9387A76C9C43D847A1679387A704D4
:10C650006312F7021763FFFFE70263A701112800C7
:10C66000814597000000E78020A705611763FFFF61
:10C67000670023A882809797FF1F938727699C43B1
:10C68000D847A167938757026319F7021763FFFF23
:10C69000E702E3A30111328597F0FFFFE780A07A5C
:10C6A0002308A1008145280097000000E780C0A270
:10C6B00005611763FFFF6700C3A382809797FF1F81
:10C6C0009387C7649C43D847A1679387E702631B9E
:10C6D000F7041763FFFFE702839F0111328532845D
:10C6E00097F0FFFFE7804078AA84228597F0FFFF4C
:10C6F000E7808077854709E9228597F0FFFFE7808B
:10C7000080744205B337A0002800814523189100AA
:10C710003ECA97000000E780209C05611763FFFF79
:10C720006700239D82809797FF1F9387275E9C4316
:10C73000D84799476313F7081763FFFFE702239968
:10C7400079713285328497F0FFFFE780C06F2AC687
:10C75000228597F0FFFFE78020712310A102228538
:10C7600097F0FFFFE780206E2301A102228597F05A
:10C77000FFFFE780406DA301A102228597F0FFFF34
:10C78000E780606C2302A102228597F0FFFFE7801B
:10C79000806B2313A102228597F0FFFFE780A06A38
:10C7A000B2452314A102280897000000E780C09238
:10C7B00045611763FFFF6700C39382809797FF1F50
:10C7C0009387C7549C43D847A1679387C7036313D4
:10C7D000F7081763FFFFE702838F79713285328490
:10C7E00097F0FFFFE78020662AC6228597F0FFFFBB
:10C7F000E78080672310A102228597F0FFFFE78082
:10C80000A0662311A102228597F0FFFFE780A063B5
:10C810002302A102228597F0FFFFE780C062A302F6
:10C82000A102228597F0FFFFE780E0612303A102C8
:10C83000228597F0FFFFE7800061B245A303A102C4
:10C84000280897000000E780208945611763FFFFF3
:10C850006700238A82801763FFFFE7024387011185
:10C860002A8497F0FFFFE780005EAA84228597F074
:10C87000FFFFE780605F228597F0FFFFE780C05EE3
:10C88000035744008D4763F7E700228597F0FFFFC9
:10C89000E780805D228597F0FFFFE780E05C28005D
:10C8A000A68597000000E780208305611763FFFFDE
:10C8B000670023849797FF1F938747459C43D8477A
:10C8C000A167FD07631FF7001763FFFFE7022380DF
:10C8D000328597000000E78040F81763FFFF67008C
:10C8E000438182809797FF1F938747429C43D84795
:10C8F000A167E5076315F7081753FFFFE702237DDC
:10C9000079713285328497F0FFFFE780C0532AC6E1
:10C91000228597F0FFFFE7802055228597F0FFFFE3
:10C92000E78080542310A102228597F0FFFFE78063
:10C93000A053520551812311A10222852302010235
:10C9400097F0FFFFE7802050A302A102228597F015
:10C95000FFFFE780404F2303A102228597F0FFFFEE
:10C96000E780604EB245A303A102280897F0FFFFBD
:10C97000E780807645611753FFFF670083778280E9
:10C980009797FF1F938787389C43D847A167938762
:10C99000E703631FF7001753FFFFE7024373328576
:10C9A00097000000E78060EB1753FFFF6700637498
:10C9B00082809797FF1F938767359C43D847A1676D
:10C9C00093874704631EF7021753FFFFE7022370A4
:10C9D00079713285328497F0FFFFE780C0462AC61E
:10C9E000228597F0FFFFE7802048B245280897F09E
:10C9F000FFFFE780606E45611753FFFF6700636FBD
:10CA000082809797FF1F938767309C43D847A16721
:10CA1000938787026310F7041753FFFFE702236B26
:10CA200079713285328497F0FFFFE780C0412AC6D2
:10CA3000228597F0FFFFE7800041B2452300A10265
:10CA4000280897F0FFFFE780206945611753FFFF33
:10CA50006700236A82801753FFFFE70243670111D3
:10CA600097F0FFFFE780203EAA85280097F0FFFFA0
:10CA7000E780806605611753FFFF6700836797971C
:10CA8000FF1F9387A7289C43D847A167D107631F3F
:10CA9000F7001753FFFFE70283633285970000001A
:10CAA000E780A0FB1753FFFF6700A364828097977E
:10CAB000FF1F9387A7259C43D847A167C507631F1E
:10CAC000F7001753FFFFE7028360328597000000ED
:10CAD000E780A0F81753FFFF6700A3618280979754
:10CAE000FF1F9387A7229C43D847A167B907631FFD
:10CAF000F7001753FFFFE702835D328597000000C0
:10CB0000E780A0F51753FFFF6700A35E8280979729
:10CB1000FF1F9387A71F9C43D847A167AD07631FDB
:10CB2000F7001753FFFFE702835A32859700000092
:10CB3000E780A0F21753FFFF6700A35B82809797FF
:10CB4000FF1F9387A71C9C43D84789476318F702A8
:10CB50001753FFFFE702A3570111328532C897F040
:10CB6000FFFFE780402EAA85280097F0FFFFE780AF
:10CB7000A05605611753FFFF6700A3578280979760
:10CB8000FF1F9387A7189C43D847A1678D076311A0
:10CB9000F7041753FFFFE7028353011132853284F4
:10CBA00097F0FFFFE780202A13066100AA844C005B
:10CBB000228597300000E780C0232800A68597F0E3
:10CBC000FFFFE780605105611753FFFF6700635265
:10CBD00082809797FF1F9387A7139C4381CFDC43E5
:10CBE00091CB1753FFFFE702834E82971753FFFF46
:10CBF0006700235082801753FFFFE702434D79718E
:10CC00003C08AE843ED2A165B7070A002A843ED410
:10CC100048103C08DD053ED636C432C63AC297D02D
:10CC2000FFFFE780E02F12474810BA8597F0FFFF1B
:10CC3000E780C01332464810B28597F0FFFFE780C7
:10CC4000E014A2464810B68597F0FFFFE780001277
:10CC5000501001478146A685228597D0FFFFE780C7
:10CC6000805145611753FFFF6700A3481753FFFF2B
:10CC7000E702E34501117C000329C501AE843ECAE9
:10CC8000A165B70707002A843ECC48087C00C5058B
:10CC90003ECE97D0FFFFE780A0288345D900480803
:10CCA00097F0FFFFE780800C500801478146A6857A
:10CCB000228597D0FFFFE780004C05611753FFFFE7
:10CCC000670023431753FFFFE702634083C79500C4
:10CCD00093F7F707A384F50097000000E78040F979
:10CCE0001753FFFF6700E3401753FFFFE702233EA0
:10CCF00079713C08AE843ED2A165B70709002A8449
:10CD00003ED448103C08938545043ED632C636C40E
:10CD100097D0FFFFE780C020A2464810B68597F065
:10CD2000FFFFE780A00432464810B28597F0FFFF6E
:10CD3000E780C005501001478146A685228597D01F
:10CD4000FFFFE780404345611753FFFF6700633AE9
:10CD50001753FFFFE702A33783C7950041112A84C9
:10CD600093F7F707A384F50032852EC697F0FFFFEF
:10CD7000E780800F85672AC46370F5029770000012
:10CD8000E78020E92246B24509ED11478146228518
:10CD900097000000E78060E641011753FFFF67003E
:10CDA000433501478346F501DDB71753FFFFE7021F
:10CDB000633001113C003ECAB7070A003ECC3C007C
:10CDC0003ECE83C79500AA89328593F7F707A384DF
:10CDD000F5002E8497F0FFFFE78000098567637DEB
:10CDE000F504A165AA8493858504480897D0FFFFC0
:10CDF000E7800013268597700000E78080E12A898C
:10CE000029E19145480897F0FFFFE78020F6A685C5
:10CE1000480897F0FFFFE78060F7CA85480897F059
:10CE2000FFFFE780A0F4014781465008A2854E85A8
:10CE300097D0FFFFE780203405611753FFFF67009D
:10CE4000A32A8145480897F0FFFFE78020F20349B5
:10CE5000090275BF1753FFFFE702C32579711C1044
:10CE60003ECAB7070F003ECC404D1C10AA84AE89C5
:10CE70004808994532C636893ECE97D0FFFFE780F5
:10CE8000200A32464808B28597F0FFFFE78000EE9F
:10CE9000630C0902A545480897F0FFFFE780C0E64C
:10CEA0002546CA8597200100E78020A45008014745
:10CEB0008146CE85268597D0FFFFE780C02B456150
:10CEC0001753FFFF670043228355C402480897F0B9
:10CED000FFFFE780A0EB0355E402814505C58547C8
:10CEE00085456301F502C167FD179305F00F630BDC
:10CEF000F5007D1597700000E780208E93051500E2
:10CF000093F5F50F480897F0FFFFE78020E683458B
:10CF10000403480897F0FFFFE78040E583451403CA
:10CF2000480897F0FFFFE78060E483552403480832
:10CF300097F0FFFFE78080E583554403480897F0AA
:10CF4000FFFFE780A0E49DB71753FFFFE702231818
:10CF500083C795008146014693F7F707A384F50040
:10CF600097000000E78040EF1753FFFF670063184A
:10CF70001753FFFFE702A31579713E841C103ECAC8
:10CF80002E89B7070F00A1653ECCFD051C10AA84B1
:10CF9000480842C03AC23ECE36C432C697D0FFFFE0
:10CFA000E78000F832464808B28597F0FFFFE78037
:10CFB000E0DBA2464808B68597F0FFFFE78000DD7A
:10CFC00012474808BA8597F0FFFFE78020DC024847
:10CFD000630C08029145480897F0FFFFE780C0D234
:10CFE0001146A28597200100E78020905008014754
:10CFF0008146CA85268597D0FFFFE780C017456127
:10D000001753FFFF6700E30E8945480897F0FFFFBD
:10D01000E78080CF834704002300F5008347140096
:10D02000A300F500E1B71753FFFFE702A30883C78A
:10D03000950001112A8A93F7F707A384F50032853A
:10D04000AE8432C697F0FFFFE78000E232462A89BD
:10D05000328597F0FFFFE78000DF85676373F90291
:10D06000AA894A8597700000E780A0BA2A8419ED42
:10D07000114781464A86A685528597000000E780C1
:10D08000C0B705611753FFFF670003069387E9FFE9
:10D0900093F7F70F0547E366F7FE8347F50195EB36
:10D0A0008947E380F9FE8346F401528501474A86A9
:10D0B000A68597000000E78040B4A167D90748081B
:10D0C0003ECC230A010002CE97000000E780A0B00A
:10D0D0004DBF639EE7008947639EF90093071020C8
:10D0E000231FF50097700000E780C0B76DBF0947A8
:10D0F000E39BE7FA8D47E398F9FA228597700000E1
:10D10000E78080DF9797FF1F938787DF9C4399E72E
:10D110009797FF1F938787C89C4399C703D504003F
:10D1200097800000E780A0CE231F040022855DBF0A
:10D130001753FFFFE702A3F901113C003ECAB707EE
:10D140000B003ECC3C003ECE83C795002A89328539
:10D1500093F7F707A384F500AE8497F0FFFFE7800D
:10D16000A0D093170501C187635AF006A1652A84F0
:10D170009385E502480897D0FFFFE78060DAA28533
:10D18000480897F0FFFFE78060C09797FF1F9387DD
:10D19000E7C09C43A9EB01449375F40F480897F04E
:10D1A000FFFFE780A0BC9355844093F5F50F480836
:10D1B00097F0FFFFE78080BB9355044193F5F50F8F
:10D1C000480897F0FFFFE78060BA014781465008A2
:10D1D000A6854A8597D0FFFFE780E0F905611753E0
:10D1E000FFFF670003F1416585460546A2857D1571
:10D1F00097500000E78060BD59DD510597000100A0
:10D20000E780808F130440063344850271B71753BB
:10D21000FFFFE702C3EB0111B70706003EC683C755
:10D22000950021642A8993F7F707A384F500AE845B
:10D2300028009305A4040AC40AC897D0FFFFE7801A
:10D2400020CE300001478146A6854A8597D0FFFF52
:10D25000E78060F297E0FFFFE780801513049404F5
:10D26000480822CC230A010002CE97000000E78084
:10D27000809605611753FFFF6700A3E71753FFFF71
:10D28000E70243E3C1642A8901449799FF1F938908
:10D29000A9C8130A8002FD1497E0FFFFE78080C150
:10D2A0006347A40001451753FFFF6700E3E3B3079B
:10D2B000440303A7C90ABA9703D707006306970078
:10D2C00083D72700638427010504F9B70545E1BF2B
:10D2D0001753FFFFE70203DE2A8A2E8999C123A094
:10D2E000050081498144979AFF1F938AAAA2614B46
:10D2F00097E0FFFFE78040C263C7A4004E85175345
:10D30000FFFF670063DE3384640383A70A003E9453
:10D310008357040099E763040900232089008504EA
:10D32000C1BF4146D2851305440097100100E78034
:10D33000605975F5A289E5B71753FFFFE70283D758
:10D3400039717C083ED4B7070A003ED67C083ED827
:10D3500083C795002A8A328593F7F707A384F500DF
:10D360002E8932C697F0FFFFE78000B085676373B0
:10D37000F5083246AA84328597F0FFFFE780A0AC1B
:10D380008547AA8963E8A706A165938585042810C7
:10D3900097D0FFFFE780C0B8268597700000E78030
:10D3A00040872A8429ED9145281097F0FFFFE780F8
:10D3B000E09BA685281097F0FFFFE780209DCE8593
:10D3C000281097F0FFFFE780609A014781463010F0
:10D3D000CA85528597D0FFFFE780E0D9A167938780
:10D3E000770448183EDC230A010202DE97F0FFFFB3
:10D3F000E780607E21611753FFFF6700E3CE814520
:10D40000281097F0FFFFE7806096A685281097F018
:10D41000FFFFE780A0979797FF1F938767E69C43DE
:10D4200081CB22856389090097D00000E7804024E2
:10D430008345040271B797D00000E780C022CDBFBA
:10D440001753FFFFE70203C783C795004111AA895D
:10D4500093F7F707A384F5003285AE84328A97F0FC
:10D46000FFFFE78060A08567637FF5022A899760E8
:10D470000000E780007A2A84914631C58347F50190
:10D4800005476387E70291C70D476366F704AD461A
:10D490001DA89305050303250A00414697100100C6
:10D4A000E78040420DE941011753FFFF6700C3C306
:10D4B0009305950803250A00414697100100E7806F
:10D4C0006040814669F54A86A6854E859700000032
:10D4D000E780C081C9BF83250A00130594089770AF
:10D4E0000000E780A02919C1C146F1BF9797FF1F2F
:10D4F000938707A19C4399E79797FF1F9387078A14
:10D500009C4399C7228597800000E780208A69FDA7
:10D510008547A30FF400228597B00000E780608460
:10D52000228597600000E780E0734E8581464A8639
:10D53000A68597F0FFFFE780607BA167938757047C
:10D5400048003EC42302010002C697F0FFFFE780B7
:10D55000806891BF1753FFFFE702E3B483C79500CC
:10D560004111AA8993F7F707A384F50032852E8924
:10D57000B28A97F0FFFFE780208F85676374F50E0E
:10D58000AA8497600000E780C0682A840DED416B93
:10D59000014A979BFF1F938B2B98130C400E7D1B0A
:10D5A00019A833048A0383A70B0B3E948357C40145
:10D5B00063836705050A97E0FFFFE780A08EE342DB
:10D5C000AAFE95460DA08357C50163969702930561
:10D5D000050303A50A00414697100100E780802E4D
:10D5E000994611E181462686CA854E8597F0FFFF50
:10D5F000E780C06F85A883A50A0013050403977010
:10D600000000E780A017C14679FD2285231E940003
:10D6100097A00000E780E074228597600000E78013
:10D6200060649797FF1F9387A7C59C43A9C32300F6
:10D630000402228597D00000E78040F04E858146A5
:10D640002686CA8597F0FFFFE780406AA167938727
:10D65000070448003EC42302010002C697F0FFFF02
:10D66000E780605741011753FFFF670043A78947D1
:10D670002300F402E1B7397106DE22DC4AD88000CB
:10D6800052D456D25AD026DA4ED65ECE2E8A32895F
:10D690002A8B97D0FFFFE780E07D06057105419951
:10D6A0008A8A3301A140232224FC231404FC97D04E
:10D6B000FFFFE780207C83479A000605350593F736
:10D6C000F7072315A4FCA304FA004A85232624FCAB
:10D6D00097E0FFFFE780407993170501C18763401A
:10D6E000F0025681130104FCF2506254D2544259A4
:10D6F000B259225A925A025BF24B21618280AA846B
:10D700004A8597E0FFFFE7802076AA894A8597E05F
:10D71000FFFFE7806075A1659385C5022A8913051F
:10D7200044FC97C0FFFFE780A07F268597C0FFFFDE
:10D73000E780E073854511C94A86CE8597C0FFFF13
:10D74000E780606DAA8B21E98945130544FC97E0C9
:10D75000FFFFE780A061A685130544FC97E0FFFF6B
:10D76000E780C062CE85130544FC97E0FFFFE780A9
:10D77000E061CA85130544FC97E0FFFFE780006184
:10D7800001478146130644FCD2855A8597D0FFFF96
:10D79000E780609EB9B78145130544FC97E0FFFF21
:10D7A000E780C05CA685130544FC97E0FFFFE78097
:10D7B000E05DCE85130544FC97E0FFFFE780005D48
:10D7C000CA85130544FC97E0FFFFE780205C814495
:10D7D00097D0FFFFE780006AE3D4A4FA83A70B0188
:10D7E00013971400BA9783D5070099C5130544FC15
:10D7F00097E0FFFFE78080598504D9BF797106D68D
:10D8000022D44AD000184ECE52CC56CA26D25AC87C
:10D81000AE893289AA8A97D0FFFFE780A065060506
:10D82000690541990A8A3301A140232A24FC231C5B
:10D8300004FC97D0FFFFE780E06383C799000605EB
:10D840002D0593F7F707231DA4FCA384F9004A854F
:10D85000232E24FC97E0FFFFE7800061931705016A
:10D86000C187634FF0005281130104FDB25022546E
:10D8700092540259F249624AD24A424B456182802F
:10D88000AA844A8597E0FFFFE780005EA165938543
:10D89000A5022A89130544FD97C0FFFFE780406871
:10D8A000268597C0FFFFE780805C854509C9CA854A
:10D8B00097C0FFFFE78020592A8B29E1894513058E
:10D8C00044FD97E0FFFFE780604AA685130544FD0D
:10D8D00097E0FFFFE780804BCA85130544FD97E082
:10D8E000FFFFE780A04A01478146130644FDCE852D
:10D8F000568597D0FFFFE7800088B5B781451305AF
:10D9000044FD97E0FFFFE7806046A685130544FDD0
:10D9100097E0FFFFE7808047CA85130544FD97E045
:10D92000FFFFE780A046814497D0FFFFE780805447
:10D93000E3DBA4FA83270B0113971400BA9783D56E
:10D94000070099C5130544FD97E0FFFFE7800044F9
:10D950008504D9BF1743FFFFE7026377834745007C
:10D96000404DD5EFFD575DC483469400094763637E
:10D97000D70A0346B400854663EEC6088306E40072
:10D9800063CA06085C45F9562390D7009787FF1FA6
:10D9900083C7873899E3A304E4009787FF1F938721
:10D9A000E73F9C4381E78947A306F4009797FF1F51
:10D9B0009387078D9C4381E789472306F4009705E9
:10D9C000000093854506AA841305040197F0000022
:10D9D000E7802010FD57231AF40281471CDC014820
:10D9E0009787FF1F23A687329787FF1F938787326A
:10D9F000232E040304C0804397D0FFFFE780C0516B
:10DA000061463306C502814522859740FFFFE780C6
:10DA1000006F81473E851743FFFF6700836DFD5709
:10DA2000D5BF1743FFFFE702836A2A8403554502E7
:10DA300097600000E780E01D19E5231E04001743EE
:10DA4000FFFF6700036B8357E401F5DB930504FFD9
:10DA5000174501001305452D97E00000E780E0140D
:10DA6000F9BF1743FFFFE70283662E89A1654111C5
:10DA70009385E5032A8436C432C6BE843AC297C071
:10DA8000FFFFE780E04912472285BA8597E0FFFF54
:10DA9000E780C02D32462285B28597E0FFFFE78000
:10DAA000E02EA2462285B68597E0FFFFE780002E94
:10DAB000630309029145228597E0FFFFE780C024B8
:10DAC0001146A68597100100E78020E24101174327
:10DAD000FFFF670003628945228597E0FFFFE7802B
:10DAE000A02283C704002300F50083C71400A3000D
:10DAF000F500E9BF1743FFFFE702635D83C79500A9
:10DB0000444D054793F7F707A384F5001C424111E4
:10DB100083C707006367F7062E842A89B1C003C74D
:10DB2000D400630FF7021787FF1F13072727184337
:10DB300005C3A386F40097A00000E780404A83C78E
:10DB4000D40099E741657D1597400000E78040309B
:10DB500083D72403918B89C797E00000E780C01327
:10DB60004A85A28597F0FFFFE7808010A167C10773
:10DB700048003EC42302010002C697F0FFFFE78081
:10DB8000800541011743FFFF6700A3561743FFFFBE
:10DB9000E702E35303D745008D47AA8441112E8441
:10DBA00032892E8563E3E70297E0FFFFE780C02B11
:10DBB000AA8523000900268597C0FFFFE780A028DB
:10DBC00041011743FFFF6700C35297E0FFFFE78063
:10DBD000A0292AC6228597E0FFFFE780E028B2450A
:10DBE00085472A862300F900268597C0FFFFE78036
:10DBF0008022F9B7397106DE22DC26DA80004ED6A3
:10DC000052D456D24AD85AD05ECEAE89B284AA8AAD
:10DC100097D0FFFFE78000250605130525024199EF
:10DC20000A8A3301A140232224FC231404FC97D048
:10DC3000FFFFE780202383C7990006054D0593F772
:10DC4000F7072315A4FCA384F9002685232624FCCA
:10DC500097E0FFFFE780402193170501C1876340EC
:10DC6000F0025281130104FCF2506254D254425922
:10DC7000B259225A925A025BF24B21618280AA8BDE
:10DC800003AB040097C0FFFFE780601E51E583D718
:10DC9000440001498544F11793B71700A301F4FC30
:10DCA000834734FCA165C9C79385E504130544FC8B
:10DCB00097C0FFFFE780C026A685130544FC97E0C8
:10DCC000FFFFE780A00ADE85130544FC97E0FFFF15
:10DCD000E780C00B834734FC114691E30946DA859F
:10DCE000130544FC97E0FFFFE78060058144630A69
:10DCF0000900416B7D1B97D0FFFFE780A01663CC26
:10DD0000A40201478146130644FCCE85568597C080
:10DD1000FFFFE7804046B1B7A685130634FC9700A5
:10DD20000000E780E0E6933415002A8986048DBF61
:10DD30009385C504A5BF8327C90013971400BA971C
:10DD400083D5070063886501130544FC97E0FFFF56
:10DD5000E780C003850445B71743FFFFE702A334FC
:10DD600079711C103EC4B7070F003EC61C103EC898
:10DD700083C79500AA8A328593F7F707A384F50035
:10DD8000AE89328497E0FFFFE780000E931705010C
:10DD9000C187635AF0062A8A228597E0FFFFE78051
:10DDA000A00C2A895285032B040097C0FFFFE7804F
:10DDB000000C39ED8357440081440544F11793B7B3
:10DDC0001700A303F10083457100DA872287CA8612
:10DDD0005286280097000000E780E0C8014781468E
:10DDE0003000CE85568597C0FFFFE780C038A16719
:10DDF0009387D70348083ECC230A810026CE97F0AC
:10DE0000FFFFE78040DD45611743FFFF6700232DDB
:10DE1000A2851306710097000000E78060D7AA84EE
:10DE2000094455D13544E30055FB4A8597F0FFFF7F
:10DE3000E78000450D4441D9014497D0FFFFE780BA
:10DE40006002634DA400C16B0144FD1B97D0FFFF2E
:10DE5000E7804001634EA4001544B5B7DC441317B6
:10DE60001400BA9783D70700638327030504F1B72B
:10DE7000D84493171400BA9703D70700631B7701A0
:10DE800023902701268597A00000E78080DB0144CE
:10DE90001DBF050465BF1743FFFFE702A32183C72A
:10DEA000950041112A8A93F7F707A384F50032857C
:10DEB0002E89328497E0FFFFE78000FB931705016E
:10DEC000C1876353F006AA89228597E0FFFFE780A8
:10DED000A0F92311A1004E85832A040097C0FFFFFB
:10DEE000E780E0F839E58357440085440144F117A1
:10DEF00093B71700A300F100034811000357210056
:10DF0000D6875285CE862686CA8597F0FFFFE780A2
:10DF10006006A167F10748003EC42302910022C6B3
:10DF200097F0FFFFE78020CB41011743FFFF670019
:10DF3000A31BA2851306110097000000E78040C5CF
:10DF40002A84894455D98357210011678544BA979B
:10DF5000C2071167C1831307F7EFE36FF7F89787DD
:10DF6000FF1F9387E7F99C4381CB8545130521006B
:10DF700097500000E7802075835521002285814459
:10DF800097C0FFFFE78040E525D9231005002285D3
:10DF900097A00000E78040CD85B71743FFFFE70259
:10DFA000831083C7950041112A8B93F7F707A38449
:10DFB000F50032852E8A328497E0FFFFE780C0EAC1
:10DFC00093170501C1876351F006AA8A228597E05D
:10DFD000FFFFE78060E92A895685832B040097C0FC
:10DFE000FFFFE780C0E831E58357440081440544E2
:10DFF000F11793B71700A301F10003483100DE8742
:10E000005A854A87D6862286D28597F0FFFFE78019
:10E0100060F6A167ED0748003EC42302810026C6D2
:10E0200097F0FFFFE78020BB41011743FFFF670028
:10E03000030BA2851306310097000000E78040B56E
:10E04000AA8409445DD99167CA97C2071167C18341
:10E050001307F7EF0544E362F7FACA8597C0FFFF9D
:10E06000E78080D7014451F9814997D0FFFFE780CD
:10E0700060E063DBA900984893971900BA9703D72B
:10E08000070005EF2390270197D0FFFFE78080DE90
:10E090001544E384A9F6268597A00000E780C0BC5C
:10E0A0009787FF1F9387C7E59C430144B9D74A85EB
:10E0B00097500000E780C05889B785097DB717439E
:10E0C000FFFFE70223FF79713E847C083EC82E8A59
:10E0D000B7071400A1653ECAE5057C08AA890808AF
:10E0E00036C4428932C6BA8AC6843ECC97C0FFFF86
:10E0F000E78000E3CA85080897E0FFFFE78000C7D4
:10E1000032460808B28597E0FFFFE78020C8A246A4
:10E11000630A09049D45080897E0FFFFE780C0BE39
:10E120001D4681459740FFFFE78060FD63890A082F
:10E130009145080897E0FFFFE78000BD1146A685DE
:10E1400097000100E780607A100801478146D28578
:10E150004E8597C0FFFFE780000245611743FFFF30
:10E16000670083F8B685080897E0FFFFE78000C2E4
:10E170001C400808D8439355C7018589120751836D
:10E18000B205D98D97E0FFFFE78040C01C4008082A
:10E1900083C5870097E0FFFFE78040BD1C4008086B
:10E1A00083C5A70097E0FFFFE78040BC1C4008083C
:10E1B00083C5970097E0FFFFE78040BB85BF894597
:10E1C000080897E0FFFFE78020B483C7040023001E
:10E1D000F50083C71400A300F500BDB71743FFFF88
:10E1E000E70243ED83C795004111AA8993F7F7072A
:10E1F000A384F5003285AE84328497E0FFFFE78088
:10E20000A0C693170501C187635DF0042A89032A1C
:10E21000040097C0FFFFE78080C519E983574400D9
:10E220000548F11793B71700A307F100814631A8FD
:10E230001306F100A28597000000E78060951DC5D8
:10E240001C459DC783D6470001480347F10093074B
:10E250008500D2884A86A6854E8597000000E78013
:10E2600040E641011743FFFF670003E809487DBF0F
:10E270001D486DBF1743FFFFE702C3E365715C08EC
:10E280003EC4B7077B013EC65C083EC883C7950005
:10E290002A8A328593F7F707A384F500AE8997E0C1
:10E2A000FFFFE78040BA8357E100E1C789452800B6
:10E2B00097C0FFFFE780C0C68145280097E0FFFFB9
:10E2C000E780C0AA97C0FFFFE780A0CC9787FF1F19
:10E2D000938707FB9C431784FF1F0344E4A3AA848E
:10E2E0003334800099C3136424009787FF1F9387FA
:10E2F000E7AA9C4399C3136444009787FF1F938741
:10E3000027C09C4399C31364840083D5040028006C
:10E31000014997E0FFFFE78060A783D5240028002C
:10E3200097E0FFFFE78080A683D54400280097E0B0
:10E33000FFFFE780A0A597D0FFFFE780A0AE931571
:10E340000501C181280097E0FFFFE78020A4A28596
:10E35000280097E0FFFFE78060A39C446360F90218
:10E36000014781463000CE85528597C0FFFFE78088
:10E3700080E059611743FFFF670003D7DC441314A3
:10E38000490028003E9497E0FFFFE78060968347AE
:10E3900044000347540089070607BA978607E36AD3
:10E3A000F5FC835524002800814A97E0FFFFE780B1
:10E3B000E09D83454400280097E0FFFFE780009B35
:10E3C00083455400280097E0FFFFE780209A8347A9
:10E3D000440063C9FA00814A8347540063C1FA02CA
:10E3E0000509A5BF1C4413975A002800BA9783D586
:10E3F0000700850A97E0FFFFE7804099C9BF032B1C
:10E40000C40093975A0028003E9B83552B00850A31
:10E4100097E0FFFFE780809783550B00280097E087
:10E42000FFFFE780A0964DBF1743FFFFE70223CA17
:10E430005C4993E717005CC997A00000E78020B60D
:10E440001743FFFF6700E3CA1743FFFFE70223C834
:10E450002E84814597F0FFFFE780C0E705C583570D
:10E460000500FD172310F50009C48357250023106C
:10E47000F40097000000E78060FB01451743FFFFB1
:10E48000670023C731457DD823100400C5BF17435B
:10E49000FFFFE70223C283C7950041112A8A93F741
:10E4A000F707A384F50032852E89328497E0FFFFB9
:10E4B000E780809B93170501C1876356F006AA8900
:10E4C000C145228597E0FFFFE780A0802A8B4E851B
:10E4D000832A040097C0FFFFE780609931E98357E2
:10E4E0004400231101000544F11793B71700A3005E
:10E4F000F10081440348110003572100D68752855B
:10E50000CE862286CA8597F0FFFFE780A0A6A16786
:10E510009387170248003EC42302810026C697E075
:10E52000FFFFE780406B41011743FFFF6700C3BB5C
:10E5300013061100A28597F0FFFFE7806065AA84AB
:10E5400009E523110100094475B7930521005A8597
:10E5500097000000E78080EF835721002A84D9DBF1
:10E560009787FF1F9387C7999C4381CB85451305E8
:10E57000210097500000E780001583552100268573
:10E58000314497C0FFFFE78020852DD5231005007B
:10E59000268597900000E780206D0144A1BF1743B6
:10E5A000FFFFE702C3B241112E896C00AA8402C6A4
:10E5B00097F0FFFFE78000D20DC103570500050764
:10E5C0002310E50097000000E78040E681473E8584
:10E5D00041011743FFFF6700C3B13247954765DB31
:10E5E000CA85268597300000E780400DC147E3408B
:10E5F00005FE3244854741462310F4008357090045
:10E60000A685130544002311F40097000100E7805C
:10E61000C02D228545BF1743FFFFE702A3A983C78B
:10E6200095004111AA8A93F7F707A384F500328574
:10E63000AE89328497E0FFFFE780008393170501DE
:10E64000C1876356F0062A8AC145228597D0FFFF0D
:10E65000E7802068AA845285032B040097C0FFFF3F
:10E66000E780E08031E983574400231101008544AD
:10E67000F11793B71700A300F100014403481100FC
:10E6800003572100DA875685D2862686CE8597F0F5
:10E69000FFFFE780208EA1679387070248003EC4F2
:10E6A0002302910022C697E0FFFFE780C05241019C
:10E6B0001743FFFF670043A3A2851306110097F0DD
:10E6C000FFFFE780E04C2A8409E52311010089441B
:10E6D00075B726859305210097000000E78060EC60
:10E6E000AA8449FD83552100228597B0FFFFE7806A
:10E6F000A06E49F5014997C0FFFFE780A077635DF1
:10E70000A900184893171900BA9703D707000DEF0F
:10E71000035721002390E70097C0FFFFE780807533
:10E72000630625039777FF1F9387877D9C4399C7CF
:10E730000355210097500000E78080F022859790D4
:10E740000000E78060521DBF050975B795443DB7CD
:10E7500005C19307F00F630FF500C547630CF50083
:10E760009307F5FF05453315F50042054181828089
:10E770000145828041657D158280B9E91743FFFF1D
:10E78000E702E39403450603328497000000E78024
:10E7900060FC9305803EB305B502C205C18181CD01
:10E7A0000357E402854763F8E7001305040197E087
:10E7B0000000E78020428357E40241677D176385AC
:10E7C000E700FD172317F4021743FFFF670063926A
:10E7D00082801743FFFFE702038D004283C7950045
:10E7E000444D0349140093F7F707A384F5008347CA
:10E7F0000400220911673369F900A167B347F900E2
:10E8000041112A8BAE8A63ECE70E8347240013077D
:10E81000C00EB91793F7F70F6373F710034734006F
:10E82000C14763EEE70E834744001307E00793C731
:10E8300007086371F70C8349840083477400A209B9
:10E84000B3E9F900856763F7F90A034A640083476F
:10E8500054004E85220A336AFA0097500000E78080
:10E86000403B61C123962403834B3400137AFA00A2
:10E87000239A34032388740323994403938904015E
:10E88000631C090023A60402239804024E8597E026
:10E890000000E78060363DA0034924004A859700C8
:10E8A0000000E78020EB2397A402834744004E85B5
:10E8B000A388F402E38D0BFCE30B09FC97E0000056
:10E8C000E780202F97900000E78000738146014683
:10E8D000D6855A8597E0FFFFE7800058A1679387A8
:10E8E00097033EC423020100480002C697E0FFFFE1
:10E8F000E780602E41011733FFFF6700437E8544A8
:10E90000A2862686D6855A8597E0FFFFE780C05409
:10E91000A167938797033EC423029100F1B7BD44DA
:10E92000C5B79144F1BF1733FFFFE702A378011188
:10E930001C08404D3EC2B7070F003EC41C083EC62F
:10E940002A89AE8997C0FFFFE780A0DA585C1C5C7B
:10E950006346B70E6394E50063E2A70E3385A740D4
:10E96000B3B7A700B305B7401306803E81469D8D1F
:10E9700097000100E78080B793140501C180A1656D
:10E980009385C503480097B0FFFFE7806059814534
:10E99000480097D0FFFFE780603D8355040448009E
:10E9A00097D0FFFFE780803E83552404480097D02E
:10E9B000FFFFE780A03D814589CCC167FD17930526
:10E9C000F00F6388F400268597500000E780E0E0B0
:10E9D000AA85480097D0FFFFE780403903554404DB
:10E9E000814501CDC167FD179305F00F6307F50061
:10E9F00097500000E78060DEAA85480097D0FFFFAF
:10EA0000E780C03683456404480097D0FFFFE78065
:10EA1000E03583457404480097D0FFFFE780003558
:10EA2000500001478146CE854A8597B0FFFFE780B9
:10EA3000807405611733FFFF6700036B814481B762
:10EA40001733FFFFE702A36883C7950093F7F70723
:10EA5000A384F50097000000E78020ED1733FFFF47
:10EA6000670023691733FFFFE702C36483C795007C
:10EA70004111404D93F7F707A384F5002A8A3285A8
:10EA8000B284AE8997D0FFFFE780003E2A8B2685AF
:10EA900097D0FFFFE780403D2A89268597D0FFFF6A
:10EAA000E780603A93170B0163CA0702E177CA97C0
:10EAB000C207C183116763E3E70293070910C20726
:10EAC000C1831307B00F637BF70093170901C18758
:10EAD000AA8A634AF000C54763FE57014101173314
:10EAE000FFFF6700636097B0FFFFE780C028E31770
:10EAF00025FFD5B763080B026306090281446389C9
:10EB00000A02B7077F0023106405231124057CC087
:10EB1000568597000000E780E0C39304803EB3046D
:10EB2000950239A0B7077F00232004047CC08144EC
:10EB30000355240497E00000E780A0A3A1C497C078
:10EB4000FFFFE78000BB269593D7F441333795004C
:10EB5000AE97BA9708DC5CDCCE8552859700000042
:10EB6000E780A0DC99E023220404A1679387B70320
:10EB700048003EC42302010002C697E0FFFFE78081
:10EB80008005A9BF814701481CDC232E0403E9B797
:10EB90001733FFFFE702A35397C0FFFFE780C0379B
:10EBA000E1473305F502914597500000E78000C525
:10EBB000E55711C59777FF1F23AEA71481473E8500
:10EBC0001733FFFF6700E35285471777FF1F2305C1
:10EBD000F71482801733FFFFE702634F9777FF1F19
:10EBE0009387071380433DC0835704046390A706AF
:10EBF00083572404639CB7043689B28497C0FFFF0F
:10EC0000E78020AF5C5C63C3B7046395B7001C5C0E
:10EC100063EEA7028347640463F3F400A68723032B
:10EC2000F4048347740463F39700A687A303F404F2
:10EC30008357440441677D176385E70085072312E6
:10EC4000F4043C4481C7CA85268582971733FFFFA9
:10EC50006700234A9777FF1F9387870B9C430145E3
:10EC600099C303C5870082801733FFFFE70223465D
:10EC70000111B70707003EC683C79500584D0AC467
:10EC800093F7F7070AC8A384F5002A89AE8411CB4D
:10EC90001C4283C707002304F70097900000E78019
:10ECA0000034216493055402280097B0FFFFE780E9
:10ECB000202797000000E78020FAAA85280097D037
:10ECC000FFFFE780A00A300001478146A6854A85FC
:10ECD00097B0FFFFE780204A13044402480822CC83
:10ECE000230A010002CE97E0FFFFE780C0EE056136
:10ECF0001733FFFF6700E33F1733FFFFE702233DB2
:10ED000001117C003ECAB70707003ECC7C003ECE16
:10ED100083C795002E84AA8493F7F707A384F50090
:10ED2000A16593855502480897B0FFFFE780401F13
:10ED300097000000E78040F2AA85480897D0FFFFBF
:10ED4000E780C002500801478146A285268597B01A
:10ED5000FFFFE780404205611733FFFF670063391B
:10ED60009777FF1F9387C7FA9C43094599C303C54B
:10ED7000970082809777FF1F938787F99C43094507
:10ED800099C303C5D70082809777FF1F938747F801
:10ED90009C43014599C303C5A70082801733FFFF39
:10EDA000E70243310111B70708003EC683C795004B
:10EDB000404D0AC493F7F7070AC8A384F5002A89CF
:10EDC000AE8429C41442854703C7060063E0E70AFE
:10EDD00083479400094681496380C702B307F7401F
:10EDE000A304E400B339F00083C716002305F40040
:10EDF00097900000E780A01E03572403058B19C7D6
:10EE00006386090097D00000E78000E9216493053C
:10EE10008402280097B0FFFFE78080109700000071
:10EE2000E78040F4AA85280097D0FFFFE78000F430
:10EE300097000000E78080F5AA85280097D0FFFFA3
:10EE4000E780C0F2014781463000A6854A8597B029
:10EE5000FFFFE780403213047402480822CC230AE3
:10EE6000010002CE97E0FFFFE780E0D6056117338F
:10EE7000FFFF670063271733FFFFE70243250111F8
:10EE80007C003ECAB70708003ECC7C003ECE83C75C
:10EE900095002E84AA8493F7F707A384F500A16553
:10EEA00093858502480897B0FFFFE78060079700C9
:10EEB0000000E78020EBAA85480897D0FFFFE78095
:10EEC000E0EA97000000E78060ECAA85480897D048
:10EED000FFFFE780A0E9500801478146A28526850B
:10EEE00097B0FFFFE780202905611733FFFF670018
:10EEF00043209777FF1F9387A7E19C43014599C360
:10EF000003C5B70082801733FFFFE702431C0111DE
:10EF1000B70707003EC683C79500404D0AC493F764
:10EF2000F7070AC8A384F5002A89AE8405C81C42E5
:10EF3000054783C707006368F7060347B400630FFC
:10EF4000F700A305F40097900000E780400983478D
:10EF5000B400B9CF97D0FFFFE78040BE216493058E
:10EF6000B400280097B0FFFFE78080FB9700000007
:10EF7000E78060F8AA85280097D0FFFFE78000DFD0
:10EF8000014781463000A6854A8597B0FFFFE7809C
:10EF9000801E2904480822CC230A010002CE97E0F3
:10EFA000FFFFE78040C305611733FFFF670063146D
:10EFB00097D0FFFFE78020BF55B71733FFFFE70269
:10EFC000031101117C003ECAB70707003ECC7C004C
:10EFD0003ECE83C795002E84AA8493F7F707A384B7
:10EFE000F500A165AD05480897B0FFFFE78040F345
:10EFF00097000000E78020F0AA85480897D0FFFF1F
:10F00000E780C0D6500801478146A285268597B083
:10F01000FFFFE780401605611733FFFF6700630DB0
:10F020009777FF1F9387C7CE9C43094599C303C5B4
:10F03000C70082801733FFFFE702630901117C00DC
:10F04000AE843ECAA165B70707002A843ECCD1052D
:10F050007C0048083ECE97B0FFFFE78060EC970049
:10F060000000E78020FCAA85480897D0FFFFE780D2
:10F07000E0CF500801478146A685228597B0FFFF63
:10F08000E780600F05611733FFFF670083061733C2
:10F09000FFFFE702C30383C7950093F7F707A38435
:10F0A000F50097000000E78020F91733FFFF6700A5
:10F0B00043041733FFFFE702E3FF83C795000329EB
:10F0C000C501411193F7F707A384F5001C4283C9DA
:10F0D0000700854763E637079777FF1F9387471A2F
:10F0E0009C432E84AA8485CF97000000E78080F39C
:10F0F00089476306F502630409028347C9006380F8
:10F1000037032306390197900000E78040ED8357CD
:10F110002903898B89C797D00000E780E0B726854F
:10F12000A28597000000E78020F1A167CD07480085
:10F130003EC42302010002C697E0FFFFE780A0A9BA
:10F1400041011733FFFF670023FA9777FF1F93876B
:10F1500027BC9C431D4599C303C5E7008280173334
:10F16000FFFFE702C3F60111B70707003EC683C7DA
:10F170009500584D0AC493F7F7070AC8A384F50011
:10F180002A89AE8415C71C4283C70700939687015E
:10F19000E18663C4060685466381D7068346E70099
:10F1A0006388F6002307F70097900000E78020E3CC
:10F1B00021649305E400280097B0FFFFE78040D664
:10F1C00097000000E780A0F8AA85280097D0FFFFED
:10F1D000E780C0B9014781463000A6854A8597B0CF
:10F1E000FFFFE78040F93504480822CC230A0100DC
:10F1F00002CE97E0FFFFE780009E05611733FFFF17
:10F20000670023EF1733FFFFE70263EC01117C0077
:10F210003ECAB70707003ECC7C003ECE83C79500B0
:10F220002E84AA8493F7F707A384F500A165B90596
:10F23000480897B0FFFFE780A0CE97000000E78066
:10F2400000F1AA85480897D0FFFFE78020B2500858
:10F2500001478146A285268597B0FFFFE780A0F190
:10F2600005611733FFFF6700C3E81733FFFFE702AD
:10F2700063E4AA8401441779FF1F1309A9A9E1498E
:10F2800097C0FFFFE78040C96344A400014519A867
:10F2900033053403832709003E9583572500639780
:10F2A000970011051733FFFF670003E40504C9BF8A
:10F2B000032E8500630A0E121773FF1F130343C446
:10F2C00003230300631503002943639006120323FD
:10F2D0004E01631503001D43639907101733FFFFA9
:10F2E000E70263DCC689428A3E89BA8AB684328BD9
:10F2F000AE8B2A84B5E103554E0019E501431A850A
:10F300001733FFFF6700A3DDA167A98F116763FBB8
:10F31000E70097000000E78080F5814597F0FFFF48
:10F32000E780C0120844B70700E05841F98F18453C
:10F330005CC1B707001FF98F1CC55C4991C7610507
:10F3400097E00000E780408BE38A09FA22859790D6
:10F350000000E78060C65DB7328597C00000E78097
:10F3600040430D4349DD1C44116703D54700A167A5
:10F37000A98F63FBE70097000000E78040EF81451D
:10F3800097F0FFFFE780800C0323840093164B0166
:10F39000D1828347B300035663008588FD8BA305A4
:10F3A000F300FD777D8E558EFD76FD16B204F18E4D
:10F3B00083274301C58E231273012313D300230433
:10F3C000530123052301A3044301BDDF228597B028
:10F3D000FFFFE78020CDAA850844B5D1610597D00D
:10F3E0000000E780207F8DB71D431A858280173388
:10F3F000FFFFE70223CC0569AA84AE89328A014463
:10F40000FD5A7D1997C0FFFFE780C0A56347A400A0
:10F4100001451733FFFF670023CDD844931714002D
:10F42000BA9703D70700631F370323905701630779
:10F430000A00268597900000E780A0809C449DC329
:10F4400083D76700B3F72701639E3701D28801484D
:10F450008147014781460146814526859700000086
:10F46000E78040E5050479BF1733FFFFE70283C457
:10F4700079711C103EC4B7070F003EC61C103EC871
:10F4800083C79500AA8A328593F7F707A384F5000E
:10F490002E89328497D0FFFFE780009D93170501E6
:10F4A000C187635AF006AA89228597D0FFFFE780BB
:10F4B000A09B2A8A4E85032B040097B0FFFFE780AC
:10F4C000009B39ED8357440081440544F11793B7FD
:10F4D0001700A303F10083457100DA872287D286E3
:10F4E0004E86280097E0FFFFE780E05701478146FE
:10F4F0003000CA85568597B0FFFFE780C0C7A16777
:10F500009387F70348083ECC230A810026CE97D084
:10F51000FFFFE780406C45611733FFFF6700C3BC06
:10F52000A2851306710097E0FFFFE7806066AA845A
:10F53000094455D1528597E0FFFFE78060D40D4420
:10F5400059D90546D285268597000000E78060EAF4
:10F550002A8451B71733FFFFE70263B783550700CB
:10F560000346270041112A842E8532C62EC497E017
:10F57000FFFFE780E0D001C93246A245228597000F
:10F580000000E78000E741011733FFFF670063B623
:10F590001733FFFFE70223B183C795004111AA8A01
:10F5A00093F7F707A384F5003285AE89328497D0AC
:10F5B000FFFFE780608B93170501C1876357F00A4F
:10F5C000C1452A8A228597C0FFFFE78080702A8D77
:10F5D000228597D0FFFFE78020892A89228597D04E
:10F5E000FFFFE7804086930705F893F7F70F1307AF
:10F5F000E007AA8B637BF706228597D0FFFFE780A1
:10F6000080842A8C228597D0FFFFE780C083AA8C54
:10F610005285032B040097B0FFFFE780408539E94E
:10F6200083574400231101008144F11793B7170059
:10F63000A300F1000544034711008356210093877E
:10F6400084005685DA8822885286CE8597F0FFFF9F
:10F65000E78020A7A167E90748003EC42302810094
:10F6600026C697D0FFFFE780005741011733FFFF01
:10F670006700E3A613061100A28597E0FFFFE7806D
:10F680002051AA8409E52311010009446DB79305AF
:10F6900021006A8597F0FFFFE780A0F02A8441FDF2
:10F6A000835521009356C900131649018548668881
:10F6B000E2875E87858A5182268597000000E78071
:10F6C00060BF2A848DBF1733FFFFE702C39D83C746
:10F6D000950041112A8B93F7F707A384F500328533
:10F6E000AE89328497C0FFFFE78000789317050149
:10F6F000C1876352F00A2A8A228597C0FFFFE780FC
:10F70000A076AA8A228597C0FFFFE780E0752A8944
:10F71000228597C0FFFFE7800073930705F893F7F2
:10F72000F70F1307E0072A8C6377F706228597C047
:10F73000FFFFE7804071AA8C228597C0FFFFE7801A
:10F7400080702A8D5285832B040097A0FFFFE780ED
:10F75000007239E58357440085440144F11793B79B
:10F760001700A301F10003473100930784005A8575
:10F77000DE882688D6865286CE8597F0FFFFE78002
:10F7800040948D4748003EC42302910022C697D082
:10F79000FFFFE780404441011733FFFF67002394D8
:10F7A000A2851306310097E0FFFFE780603E2A84C0
:10F7B000894455D99356C9001316490185486A886A
:10F7C000E6876287858A5182D68597000000E780A8
:10F7D00060AEAA8449BF1733FFFFE702A38D2A89D1
:10F7E00081440144617A916A176BFF1F130B4B71BF
:10F7F00097B0FFFFE780006863C7A4002285173336
:10F80000FFFF6700638E8327090093991400CE974A
:10F8100003D507003307450142074183636457035B
:10F8200005C103270B0019C785453E859740000099
:10F83000E78060E9832709000504CE97239007003D
:10F8400085047DB797000000E78060A28327090048
:10F850000504CE972390070065D5814597F0FFFFFB
:10F86000E780C0BEF1BF1733FFFFE702A38483C761
:10F87000950041112A8A93F7F707A384F500328592
:10F880002E89328497C0FFFFE780005E9317050141
:10F89000C187635AF004AA89832A040097A0FFFF56
:10F8A000E780E05C31E58357440085440144F1176B
:10F8B00093B71700A301F10003483100D6875285A2
:10F8C0000147CE862686CA8597D0FFFFE780806AEB
:10F8D000A167F50748003EC42302910022C697D0D5
:10F8E000FFFFE780402F41011723FFFF6700C37F21
:10F8F000A2851306310097E0FFFFE78060292A8484
:10F9000089445DD99767FF1F9387875F9C4381CFA9
:10F91000044997B0FFFFE780E055AA852685974008
:10F920000000E78040DA1305040197000000E7803B
:10F93000C0EA228597800000E78000338144ADBF94
:10F940001723FFFFE702237683C795004111AA8A98
:10F9500093F7F707A384F5003285AE89328423112B
:10F96000010097C0FFFFE780205093170501C18772
:10F970006354F0062A8AC145228597C0FFFFE780BD
:10F980004035AA8B5285032B040097A0FFFFE78028
:10F99000004E21E98357440085440144F11793B791
:10F9A0001700A300F1000348110003572100DA8774
:10F9B0005685D2862686CE8597D0FFFFE780805B6E
:10F9C000A1679387270248003EC42302910022C604
:10F9D00097D0FFFFE780202041011723FFFF67003A
:10F9E0000370A2851306110097E0FFFFE780401A1D
:10F9F0002A8489444DD99767FF1F9387675098439E
:10FA00003E8901CF044997B0FFFFE780A046AA8551
:10FA1000268597400000E78000CB1305040197007E
:10FA20000000E78080DB97B0FFFFE780A0449544AB
:10FA30003DD9930521005E8597F0FFFFE78060B612
:10FA4000AA8435F11C480357210022852390E70042
:10FA500097800000E780402183270900A9D703553C
:10FA6000210097400000E780A0BD35BF1723FFFFAE
:10FA7000E702636383C795004111AA8A93F7F707EA
:10FA8000A384F5003285AE89328497C0FFFFE780FA
:10FA9000A03D93170501C1876351F0062A8A22858C
:10FAA00097C0FFFFE780403C2A895285032B040062
:10FAB00097A0FFFFE780A03B31E5835744008544D2
:10FAC0000144F11793B71700A301F1000348310077
:10FAD000DA8756854A87D2862686CE8597D0FFFF5D
:10FAE000E7804049A167F90748003EC4230291001E
:10FAF00022C697D0FFFFE780000E41011723FFFFCA
:10FB00006700E35DA2851306310097E0FFFFE78001
:10FB100020082A8489445DD99167CA97C207116772
:10FB2000C1831307F7EF8544E362F7FA9767FF1F76
:10FB30009387073D9843BE8B01CF044997B0FFFFE1
:10FB4000E7804033AA85268597400000E780A0B76C
:10FB50001305040197000000E78020C897B0FFFF5D
:10FB6000E780403195443DD11C4822858144239053
:10FB7000270197800000E780200F83A70B00B9D7EB
:10FB80004A8597400000E780A0AB89B71723FFFFA5
:10FB9000E702E3532A844105B28497000000E7801E
:10FBA000C0C311C5228597800000E780E00B814625
:10FBB0000146A685228597800000E780C04E1C4C38
:10FBC00089C7DC4799C3228582971723FFFF670007
:10FBD00043529767FF1F9387A7139C43014599C31F
:10FBE0001385070182809767FF1F938767128843F9
:10FBF00082801723FFFFE702834D9317C600DD8D38
:10FC0000C2054111C1812A8432C697C0FFFFE78037
:10FC1000E0173246228511829375F60F97C0FFFFD9
:10FC2000E780C01441011723FFFF6700834C1723AF
:10FC3000FFFFE702234879713C083ED2B7070C006A
:10FC40003ED43C083ED683C79500AE842A8993F7FC
:10FC5000F707A384F500A16593853504481097A0A4
:10FC6000FFFFE780E02BC165FD150144176AFF1F08
:10FC7000130A8A2A930A400EAE892E8B2EC697B09D
:10FC8000FFFFE78020224205931704014181C183D1
:10FC9000B24563E9A702C167FD176387F500481005
:10FCA00097C0FFFFE780800E501001478146A68570
:10FCB0004A8597A0FFFFE780004C45611723FFFFAF
:10FCC000670083423307540383270A0BBA9703D68E
:10FCD000C701630A3601638A3501481097000000A6
:10FCE000E78060F1DA85050451BFB285EDBF1723C7
:10FCF000FFFFE702433B79717C083EC8B70711005C
:10FD00003ECA7C083ECC83C79500AA89328593F70A
:10FD1000F707A384F5002E8997C0FFFFE780C01482
:10FD200085676378F504A165AA848905080897A00A
:10FD3000FFFFE780E01E268597400000E78060ED2A
:10FD4000133415000A04A285080897C0FFFFE78056
:10FD5000E001A685080897C0FFFFE780200325CCB7
:10FD6000014781461008CA854E8597A0FFFFE780AE
:10FD7000804045611723FFFF67006336B3075403D4
:10FD80000327CA0ABA9703D70700631C970003D654
:10FD9000270063806505080897000000E780A0E55C
:10FDA000DE8505042EC697B0FFFFE780A010420550
:10FDB000931704014181C183B245E3E1A7FCC16708
:10FDC000FD17E38FF5F8080897C0FFFFE78000FCF8
:10FDD00041BFB285F9B7C165FD150144176AFF1F20
:10FDE000130A8A13930A80022E8BAE8B65BF1723EA
:10FDF000FFFFE702C32D1841834717008346070022
:10FE0000A207D58FD207D1832390F500834727001F
:10FE1000034717008D45A207D98F91832310F60061
:10FE200097C0FFFFE780A0E91723FFFF6700632C5F
:10FE30001723FFFFE7020328C16401441769FF1F6E
:10FE40001309890D93098002FD1497B0FFFFE78025
:10FE500060066347A40001451723FFFF6700C3281E
:10FE6000330534038327C90A3E9583570500E3858C
:10FE700097FE0504D9BF1723FFFFE702A3232A8AB1
:10FE8000AE89B284B68A97400000E78080D819E531
:10FE900091473E851723FFFF670003252A894E857A
:10FEA00097C00000E780E08E2A84638E0A048D47A5
:10FEB0006DD103570500C547E31D47FD0347F90111
:10FEC0008546AD47E317D7FC8347450081CF4146C0
:10FED000A6855D0597F00000E780C09E814755D953
:10FEE000AD4745BF130965012302E500CA85268594
:10FEF00097100000E780606231C1A547E38B0AF8E4
:10FF00002302040079B705C183570500E39247F93E
:10FF10004146A685190597F00000E780A09A814721
:10FF20002DD99947BDB74E8597000000E78080F036
:10FF30002A84954739DD130955004DBF4146A685F2
:10FF400023104401231134011305190097F0000018
:10FF5000E780A099228597800000E780A0EA81478A
:10FF60000DBF1723FFFFE702831679717C003ECC9B
:10FF7000B7070A003ECE7C003ED083C79500B2840E
:10FF80002E8493F7F707A384F5001306A1002A89AE
:10FF90002C00268597000000E780A0E5A1652808D1
:10FFA0008D0597A0FFFFE780A0F790408355A10043
:10FFB00003558100854697000000E78000ECAA8485
:10FFC000AA85280897C0FFFFE78040DA0356A10002
:10FFD00083558100280897000000E780C0C13008E1
:10FFE00001478146A2854A8597A0FFFFE780A018B8
:10FFF000854748103ED42302910202D697D0FFFFD6
:020000040001F9
:10000000E78060BD45611723FFFF6700830E17235C
:10001000FFFFE702C30B79717C003ECCB7070A00F3
:100020003ECE7C003ED083C79500B2842E8493F7E9
:10003000F707A384F5001306A1002A892C00268562
:1000400097000000E780E0DAA16528088D0597A0F9
:10005000FFFFE780E0EC90408355A100035581004D
:10006000814697000000E78040E1AA84AA8528081D
:1000700097C0FFFFE78080CF0356A1008355810022
:10008000280897000000E78000B730080147814644
:10009000A2854A8597A0FFFFE780E00D4810230264
:1000A000910202D402D697D0FFFFE780C0B245612B
:1000B0001723FFFF6700E3031723FFFFE702230176
:1000C00097000000E78060DB1723FFFF67006302F3
:1000D0009767FF1F938707C4884382801723FFFF1A
:1000E000E702E3FE835725004111AE842A842307EB
:1000F000B10017F5FFFF130525466C002316F1002C
:1001000097A0FFFFE780204991C4228597800000D7
:10011000E780E0D6FD572310F40013062002814546
:10012000130554009720FFFFE78060FD410117236E
:10013000FFFF670003FC1723FFFFE702A3F77971B6
:100140007C003ECCB7070A003ECE7C003ED083C781
:100150009500AA89AE8493F7F7073285A384F5004A
:100160001306A1002C0097000000E78080C803550B
:100170008100114497400000E780A0A915C50355F0
:10018000A100014497B00000E780A06011CD0357A3
:1001900005008357810045446318F70085459700A3
:1001A0000000E780E0F30144216993053900280845
:1001B00097A0FFFFE780C0D6A285280897C0FFFF61
:1001C000E780C0BA0356A100835581002808970034
:1001D0000000E78040A2300801478146A6854E8591
:1001E00097A0FFFFE78020F948104AD4230281023C
:1001F00002D697D0FFFFE780009E45611723FFFFDF
:10020000670083EE1723FFFFE702C3EA9767FF1F2C
:10021000938707B02A8488432E8915C50357450361
:100220008357C4016311F702232605022318050230
:10023000410597D00000E780209C63060900978065
:100240000000E78060DB81449769FF1F9389C9CC78
:10025000130A800297B0FFFFE780C0C563C4A404FF
:100260009767FF1F938787B39C4399C70355C401C2
:1002700097200000E780C0BD6307090022859780B2
:100280000000E780C0A01306400E8145228597201C
:10029000FFFFE780C0E6FD57231EF4001723FFFF92
:1002A000670083E43385440383A7C90A3E95035757
:1002B00005008357C4016317F700CA859700000043
:1002C000E78000E2850479B71723FFFFE70283DEAA
:1002D00083C795004111AA8993F7F707A384F50016
:1002E0003285AE8497C0FFFFE78000B885676378EA
:1002F000F5042A8997400000E780A091014401CDD0
:1003000083D70400314463882701854597000000A6
:10031000E78080EF01444E85A2864A86A68597D065
:10032000FFFFE780A09CA1679387170448003EC4A5
:100330002302810002C697D0FFFFE780C0894101F8
:100340001723FFFF670043DA1723FFFFE70283D677
:100350009767FF1F9387C79B804329C4014597C0B8
:100360000000E780002181470148C1641CDC232E86
:100370000403232004041769FF1F1309E9B901448A
:100380009309400EFD1497B0FFFFE780A0B1634FC3
:10039000A400814517F5FFFF1305857F97A0FFFF98
:1003A000E780601F1723FFFF670003D43305340382
:1003B0008327090B3E958357C501638797008545C1
:1003C00097000000E78040E4050475BF93570501DE
:1003D00013D78700A380F50093170501C183A1837C
:1003E0002380E5002381F500A381A50082801723E7
:1003F000FFFFE702C3CD2300050083C71500A3005C
:10040000F50083C725002301F50083C73500A3014C
:10041000F50083C745002302F50083C75500A302FA
:10042000F50083C7650093059500A303050023032A
:10043000F50023040500328597000000E78040F9AD
:100440001723FFFF6700E3CA1723FFFFE70283C6F6
:100450004111E9540DCD85CD93F9C5FF2E842A892C
:10046000AA84338AA900B7EA040063189A020D88A7
:10047000854411CCB7E704009C5F82972AC6228688
:100480006C003305390197E00000E78000462685BF
:1004900041011723FFFF670023C583A78A03910447
:1004A000829793170501C183A183A38EF4FE93570E
:1004B0000501238FF4FEA183238EA4FEA38FF4FEF7
:1004C0006DB763E6D5021723FFFFE70243C0B2878B
:1004D00041113686BE8536C697E00000E780E040D1
:1004E000B246410136851723FFFF670083C081466E
:1004F00036858280838705001387F5003D05FD87DB
:1005000093F77708834607007D158606B58FA3000D
:10051000F5006307B7007D17834717009D83DDB79C
:1005200082801723FFFFE70283BAB7E7040083A79F
:10053000070932872A863A858297133515001723D3
:10054000FFFF670003BB15C181478DC11723FFFF64
:10055000E702E3B7414697E00000E78000398547AE
:100560003E851723FFFF6700C3B881473E85828021
:100570001DCD1723FFFFE70283B5414681452A843D
:100580009720FFFFE780A0B741468145130504038C
:100590009720FFFFE780A0B60147C167232204042C
:1005A00038C87CC805451723FFFF670083B40145A1
:1005B000828081473DCDB5CD1723FFFFE70223B1F0
:1005C000B2842E891306800581452A849720FFFF77
:1005D000E780E0B2CA8524C4268597000000E78042
:1005E000C0F64146814522859720FFFFE78020B174
:1005F0003044A285228597000000E780C0F2930472
:100600000401A285268597000000E780E0EEA6851C
:100610001305040297000000E78000EE2285970092
:100620000000E78020F585473E851723FFFF670020
:1006300043AC3E8582801723FFFFE702A3A7411149
:10064000E9540DCD85CD93F9C5FF2E842A89AA845E
:10065000338AA900B7EA0400639844030D888144F3
:1006600011CCB7E704009C5F82972AC622866C00F3
:100670003305390197E00000E780202726854101F6
:100680001723FFFF670043A683A78A03910482977D
:1006900093170501C183A183A38EF4FE935705012F
:1006A000238FF4FEA183238EA4FEA38FF4FE6DB7E7
:1006B00065CD1723FFFFE702E39FB28411E60545EE
:1006C0001723FFFF670043A22A842E890145EDD935
:1006D0003C487848B3E6E700E5D69386F7FFB3B722
:1006E000F6007D17032A4404BA9734C87CC8630512
:1006F0000A06C14913050A03B38949412295637D5E
:100700003601B2862E86A68597000000E780A0DB22
:100710007C40BE9464C065B7CE862E86CE85970099
:100720000000E78040DAC114D2944E9923220404D9
:10073000A2879306040103C7070003C607038507C2
:10074000318FA38FE7FEE398F6FE3044A285228521
:1007500097000000E78020DD2699C14933069940C3
:1007600063EC9900A9DCA686A6851305040397000F
:100770000000E78040D579BF8147B306F400330716
:10078000F6000347070083C5060085072D8F2380E9
:10079000E600E39437FF3044A285228597000000ED
:1007A000E78060D8C1145DBF014582800DC1172369
:1007B000FFFFE702C3911306800581459720FFFFE5
:1007C000E780E09305451723FFFF6700839201450B
:1007D0008280814749C5C1C51723FFFFE702238FE8
:1007E000FC4141462E84AA846399C70413860501FF
:1007F000A2878146C14503C7070003C507038507D4
:10080000298F3305D600034505008506298FA38F60
:10081000E7FEE392B6FE3044A285268597000000ED
:10082000E78060D0228597000000E78060F8854768
:100830003E851723FFFF6700C38B138507031D8EBB
:10084000814522959720FFFFE780608B7C4013074E
:1008500000F813060402A2972388E70251BF3E85E1
:1008600082801723FFFFE70283866D712E84B28496
:10087000AA8590102800368997000000E780A0D351
:1008800009EDD55725A050400C40280097000000E6
:10089000E78040E27DD5FD142104F5F42C004A8563
:1008A00097000000E78020F3814761DD3E855161BC
:1008B0001723FFFF6700E3831723FFFFE70223816E
:1008C00041112EC432C62C00054697000000E78077
:1008D00080F941011723FFFF6700A3811713FFFF72
:1008E000E702E37E01112A842EC602C802CA02CCA6
:1008F00002CE97E00000E780402BB2462A86A28510
:10090000080897000000E78060FB1375F50F05618C
:100910001713FFFF6700E37D1713FFFFE702237B39
:100920007971B2872A8421462308B1001305110189
:10093000BE853AC436C697E00000E78000FBB246A9
:1009400093059101368597000000E78060A8228515
:10095000141035460C0897000000E78020F62A8422
:10096000224701E921460C103A8597E00000E78014
:10097000C0F7228545611713FFFF670083771713C0
:10098000FFFFE702C3747171AE84AA850A853284C1
:1009900097000000E78060BB11C90A86A685228502
:1009A00097000000E78020B8814711E1C5473E85E8
:1009B0004D611713FFFF6700C3731713FFFFE702B3
:1009C000036E1D712A8AB289BE8435468547130598
:1009D00011012E8CB68A3A8BC28C468D2308F10009
:1009E00097E00000E78060F010100C085285231F8C
:1009F000010097000000E780C0F82A843DEDA14780
:100A00006313FD089307900591E0E5473546E285BD
:100A10001305110113990A012308F1001359090163
:100A200097E00000E78060EC1357890093978A00F5
:100A3000D98F90080C085285231FF1009700000001
:100A4000E78020F42A8415E9A1E49387FA009183D2
:100A50001379F9003EC6631309004149668B81444E
:100A6000C14B854DB247639F970C6A868C003385D6
:100A70005C0197E00000E78040E7228525611713BD
:100A8000FFFF6700836593079004C9F0A547BDBFCA
:100A9000834701050947C14B2308F100834711052E
:100AA000A58FA308F10093872400814463E1FB0430
:100AB000014714083386E6008C08B386E400BA9533
:100AC000DA9683C6060083C505000507AD8E2300B0
:100AD000D600E390E7FE4147639CE70490080C08CA
:100AE000528597000000E780C0E925D181A0B306B8
:100AF0009B00BA871008B305F60090083E9603C520
:100B000006000346060085078506298E2380C5005A
:100B1000E39277FF998F90080C085285BE94970056
:100B20000000E78000E68947014749D12A84B1B730
:100B300090083E96034606001408BE962380C60021
:100B4000850759BFB2478504638797148147180802
:100B5000B306F70098083E973386F900034707006D
:100B6000034606008507318F2380E600E39177FF77
:100B700090080C08528597000000E78080E05DF542
:100B80003546E285130511012308B10197E0000005
:100B9000E780A0D5139704014183939784002183B4
:100BA000D98F10180C085285231FF1009700000000
:100BB000E78020DD25FD814710183387F9003E9638
:100BC0000347070003460600B306FB008507318F85
:100BD0002380E600E39277FF65A81808B306F700C4
:100BE00098083E973386F90003470700034606003E
:100BF0008507318F2380E600E3E127FFCA87639EE4
:100C0000770990080C08528597000000E78060D7AC
:100C100011FD81479800B306F700900818103E9721
:100C20003E9603470700034606008507318F238061
:100C3000E600E39177FF3546E285130511012308AD
:100C4000B10197E00000E78040CA13970401418397
:100C5000939784002183D98F10180C085285231F85
:100C6000F10097000000E780C0D1E31105EC814757
:100C700010183387F9003E96034707000346060025
:100C8000B306FB008507318F2380E600E3E227FFF0
:100C9000C109410BC1BB814785B79408BE9683C685
:100CA000060018083E972300D700850789BF638098
:100CB00006321713FFFFE702833E59712A84BE896B
:100CC000B28B85473546130511022E8B468C42891F
:100CD000BA8A368A2300F10297E00000E780E0C07C
:100CE00010180C1022852317010297000000E780DE
:100CF00040C963180512A147631FFC0693079005BE
:100D000063930900E5473546DA851305110293140C
:100D10000A012300F102C18097E00000E780E0BCF7
:100D200093178A0013D78400D98F90080C1022855E
:100D30002317F10297000000E780A0C47DE16392D1
:100D400009049307FA00BD88918391E0C144C2076A
:100D5000C183DE8C814A3EC6414DB24763E2FA0E42
:100D60006286B3854B01881097E00000E78080B56C
:100D70004DC93D557DA093079004E39609F8A5471A
:100D800059B7834701050947C14C2300F102834746
:100D90001105B3C7F900A300F10293872900814927
:100DA00063E1FC04814618103306D7008C083387B2
:100DB000D900B69556970347070083C505008506F9
:100DC0002D8F2300E600E390D7FE41476390E706AE
:100DD00090080C10228597000000E78080BA35D17A
:100DE00089A0B3863A01BA871010B305F6009008BF
:100DF0003E9603C506000346060085078506298E34
:100E00002380C500E39297FF3387EC4090080C10D5
:100E10002285BA9997000000E780A0B6894701476C
:100E200041D165611713FFFF6700232B90083E96A1
:100E3000034606001410BE962380C600850779B7C6
:100E4000B247850A93990A01939D8A0093D90901B3
:100E50006391570F85473546DA8513051102230044
:100E6000F10293D9890097E00000E78000A8B3ED74
:100E70003D0190000C1022852317B103970000005C
:100E8000E78020B059FD8147A68963EA9706268648
:100E90000C084A8597E00000E78020A581471810DC
:100EA000B306F700100898083E973E9603470700E0
:100EB000034606008507318F2380E600E3E197FEB5
:100EC000639FA90590080C10228597000000E78019
:100ED00040AB21F981479810B306F7009008181825
:100EE0003E973E9603470700034606008507318F6D
:100EF0002380E600E391A7FF4109C10CB9BD1808A2
:100F00009000B306F7003E963387FC0003470700C6
:100F1000034606008507318F2380E600B5B79808A1
:100F20004E97034707001C10CE972380E7008509E2
:100F300041BF85473546DA85130511022300F102CA
:100F400093D9890097E00000E780209AB3ED3D0136
:100F500090000C1022852317B10397000000E78052
:100F600040A2E31005EC814718089000B306F70093
:100F70003E963387FC0003470700034606008507BB
:100F8000318F2380E600E391A7FF41460C084A8594
:100F900097E00000E780609581471810B306F700DE
:100FA000100898083E973E96034707000346060040
:100FB0008507318F2380E600E391A7FF90080C108E
:100FC000228597000000E780C09B1DD599BD7D5507
:100FD00082801713FFFFE702830F01112A842E85F9
:100FE00093055100328902C002C202C402C69304B2
:100FF000740097F0FFFFE780A03D1D46A68513050E
:10100000910097E00000E780408E10088A854A85AD
:1010100097000000E780E09619ED93071400180888
:1010200083C607000346070085070507B18EA38F17
:10103000D7FEE397F4FE05611713FFFF6700630B0C
:101040001713FFFFE70203072E848C414111AA8981
:10105000838715003289914463D30700A1449757D1
:10106000FF1F9387E7219C43A1C7C1CA8D47231067
:10107000F10083C725004A852301F10083C73500AD
:10108000A301F10083C745002302F10083C7550087
:10109000A302F10083C7650093059100A30301003B
:1010A0002303F1002304010097F0FFFFE7804032A3
:1010B0000C404A860A8597F0FFFFE78080330328BB
:1010C000040083564400A6881D0881470147E516A1
:1010D00042868A854E8597000000E780408E2A89E7
:1010E00019E5A685228597B0FFFFE780E0C14A8514
:1010F00041011713FFFF670023FF4A860A8597F017
:10110000FFFFE780002F6DB71713FFFFE70283FA99
:101110002E848C414111AA8983871500328991441C
:1011200063D30700A1449757FF1F938767159C431C
:10113000A1C7C1C68D472310F10083C725004A858A
:101140002301F10083C73500A301F10083C74500E7
:101150002302F10083C75500A302F10083C7650095
:1011600093059100A30301002303F1002304010070
:1011700097F0FFFFE780C0250C404A860A8597F06C
:10118000FFFFE780002783564400032804008A8578
:10119000858EC2061D08C1822312D400A68881470D
:1011A0000147E51642864E8597000000E78060B053
:1011B00041011713FFFF670023F34A860A8597F062
:1011C000FFFFE78000234DBF1713FFFFE70223F067
:1011D000B335B000011185052A891315F601336571
:1011E00015012308B1009305110136843AC632C0B7
:1011F0003EC442C297F0FFFFE780801DA24712481D
:10120000425593D68700230BF10093059101935724
:101210008800A30AD100A30BF100230C010197F071
:10122000FFFFE780E01A3247024603280400B33785
:10123000E000835644009207914411C2A1444A85BC
:10124000A68842860C0897F0FFFFE78040772A893E
:1012500019E5A685228597B0FFFFE780E0AA4A85B9
:1012600005611713FFFF6700C3E81713FFFFE702CD
:1012700063E401113EC68647B335B0008505AA89EF
:101280001315F6015D8D2308B10093051101368415
:101290003A89B28442C446C297F0FFFFE780401308
:1012A00022489248164593578800A30AF1009305F7
:1012B000910193D78800230B0101A30BF100230CAC
:1012C000110197F0FFFFE780A010324710408356CE
:1012D0004400B337E000920703280900914891C009
:1012E000A1480C084E8597000000E780809CAA84E6
:1012F00001E9835544004A8597B0FFFFE780C0A00D
:10130000268505611713FFFF670003DEAA95930783
:10131000F00F171701001307A7A46317B50013C533
:10132000F7FF1375F50F828005058346F5FFB58F2E
:10133000BA9783C70700D5B70357450014419307F1
:10134000F00F171601001306A6A136974207418336
:10135000139506014181631BE500AD8FB29703C56C
:101360000700130515F3133515008280850603C5A4
:10137000F6FFA98FB29783C70700D9BF1713FFFFE6
:10138000E702E3D4B28736842E86BA86AA853E85E4
:10139000BA8497F0FFFFE7806052634F0500228513
:1013A00097E00000E78060802A86A686A2852685D1
:1013B00097F0FFFFE78080501713FFFF670063D3AC
:1013C0001713FFFFE70203CF5D712A8BAE8A171553
:1013D0000100130565962C00B284368ABA893E89CD
:1013E00097F0FFFFE780C04F2A845DE1341041464B
:1013F000DA85280097F0FFFFE780404C2A8449E90E
:101400008547A303F100A6C2930771002408BEC458
:10141000A68685470D462C18281002DC02DED6C0B1
:10142000BEC697F0FFFFE78000442A8435E183477A
:101430007102A6860D4693F7F7072300FA00C1470D
:101440003EDE2C188947281026DCA303F10097F014
:10145000FFFFE78040412A8405ED4146A6854E8581
:1014600097D00000E78060488D47A6860D462C186F
:101470002810A303F10097F0FFFFE780C03E2A8405
:1014800001E94146A6854A8597D00000E780E045FE
:10149000228561611713FFFF670003C51713FFFF64
:1014A000E702E3C297F70000938707EF984383C7EB
:1014B000470079712A89AE84171501001305458804
:1014C0000C083AC42306F10097F0FFFFE780404183
:1014D0002A8405ED14104146CA85080897F0FFFFDD
:1014E000E780C03D2A8415E1140815462C00081039
:1014F00097F0FFFFE780803C2A8401E921462C0811
:10150000268597D00000E780403E2285456117136D
:10151000FFFF670003BE1713FFFFE70243BB97F708
:101520000000938767E79C477971AA842E8417157A
:101530000100130565810C083EC697F0FFFFE780A8
:10154000203A0DE914104146A685080897F0FFFFE0
:10155000E780C03605E1140811466C00081097F0CA
:10156000FFFFE780A03519E58347F10193F7F70303
:101570002300F40045611713FFFF670083B71713BB
:10158000FFFFE702C3B43688A14881470147E5461B
:1015900097F0FFFFE780A0421713FFFF670063B5D6
:1015A0001713FFFFE702A3B23688A148814701471E
:1015B000E54697F0FFFFE780C06F1713FFFF670056
:1015C00043B31713FFFFE70283B001112A842E856E
:1015D0000C0832C697F0FFFFE780803009ED3247F4
:1015E000970601009386C6741008C14522859700AE
:1015F0000000E780E0D805611713FFFF670063AFC5
:101600001713FFFFE702A3AC4111C1472EC032C43C
:101610008A8509463EC23EC697F0FFFFE780A024B8
:1016200041011713FFFF6700C3AC1713FFFFE70269
:1016300003AA4111AE8613061009AA850A8502C0C5
:1016400002C202C402C697F0FFFFE78020274101D3
:101650001713FFFF6700E3A91713FFFFE70223A794
:101660003287970601009386A66E2E8693050002A8
:1016700097000000E780C0D01713FFFF670063A743
:101680001713FFFFE702A3A47971C1472ACC2ED01C
:1016900032D42C080D4628003ECE3ED23ED602C49F
:1016A00002C602C802CA97F0FFFFE780C01B45616F
:1016B0001713FFFF6700E3A31713FFFFE70223A140
:1016C0000111AA842E84170501001305E5688A8597
:1016D00097F0FFFFE780C02015E514084146A68576
:1016E0000A8597F0FFFFE780601D09ED8347E10160
:1016F0000347F101A207D98FCA07C9836177D98F40
:101700002310F40005611713FFFF6700839E15CDBA
:101710001713FFFFE702A39B9747FF1F93870764F9
:1017200090439745FF1F9385A5631745FF1F13053A
:10173000E55E97D00000E78000C51745FF1F130541
:10174000E55D1713FFFF6700C39A1745FF1F1305D9
:10175000E55C82808DCD1713FFFFE7024397974723
:10176000FF1F9387A75F944301112E840A86974534
:10177000FF1F9385E55E97D00000E78040C60A858D
:101780000294014505611713FFFF670083967D559D
:1017900082801713FFFFE702839397D00000E78052
:1017A00080D19747FF1F23ABA75A17F5FFFF1305FB
:1017B000E5C997B00000E780C0741713FFFF67000A
:1017C00043931747FF1F1307A75B931715000843A1
:1017D0003E95FD572310F50082801713FFFFE702A7
:1017E000038F2A84084009E51713FFFF6700639001
:1017F0001C4158401CC06313E5005CC08347550082
:1018000023200500F99BA302F50097A0FFFFE780C6
:10181000207CC9BF1713FFFFE702C3899747FF1F4B
:101820009387075898432A8411CB8347350093F751
:10183000070289C70355050089450297130544012E
:1018400097B00000E780403B835504000355E40057
:1018500097300000E780A00C485819C597A0FFFFFB
:10186000E7800077232A0402130584039700000011
:10187000E780E0F68144B1499790FFFFE780C06DB3
:1018800063CBA402834734002320040493F727FC8E
:10189000A301F40000489790FFFFE780E06C131667
:1018A0001500814522859710FFFFE78040851713BB
:1018B000FFFF67006383B3873403032904038504B0
:1018C0003E994A8597000000E78060F123040900F3
:1018D00065B78347350093F7070299E30145828096
:1018E0008357E500E39CB7FEC167FD176316F6005A
:1018F00005458280054599A81703FFFFE702237D70
:1019000093170601C187B2842A8401496359F00202
:10191000835705009DCB01456367F60003458400AE
:101920003E953325A6001375F50F0DA01C4813171F
:101930001900BA9783D70700E38E97FA05099790A5
:10194000FFFFE7806062E343A9FE01451703FFFF45
:101950006700237A1703FFFFE702C375AE89AA84E5
:101960009790FFFFE78000562A8497D0FFFFE7801B
:10197000A02EAA86014713068401970500009385CF
:1019800085E41745FF1F1305E53F9790FFFFE780AC
:10199000801C2A8925C98C441304C50022859E0514
:1019A00093F5050897A0FFFFE780403CCC40838774
:1019B0007400E18163DD070493E50508228597A0A3
:1019C000FFFFE780A03A0D4693854400228597A04B
:1019D000FFFFE780C03683D50400228597A0FFFF74
:1019E000E780E03D83D52400228597A0FFFFE780B4
:1019F000003D03D6490083A50900228597A0FFFF7B
:101A0000E780E0334A851703FFFF6700E36D93F536
:101A1000F5076DB71703FFFFE702636B01112A8417
:101A2000328532C697A0FFFFE780E0279780FFFF4F
:101A3000E7806034835704001747FF1F1307C74D23
:101A40003246231BF100930700F8A30DF1001C4759
:101A50001843231AA1008983858BB307F740B28509
:101A600048083ECE231C0100230D01009700000012
:101A7000E78080EE05611703FFFF670083671703A8
:101A8000FFFFE7022363004101453DC49304C40006
:101A900026853289AE8997A0FFFFE780C02495454F
:101AA0002A8A2685035B040197A0FFFFE780202197
:101AB000268597A0FFFFE780603E8D45AA8A268590
:101AC00097A0FFFFE780A01F268597A0FFFFE78074
:101AD000E03C5C48420A135A0A01D2975CC42318BE
:101AE0006401814763983A0146054D8133062541DB
:101AF0009337160013F5F70F1703FFFF6700C35E58
:101B00001703FFFFE702235A89692A8BAE8B328ABB
:101B1000B68A81440144314CFD199790FFFFE7805C
:101B2000A04363CDA4009790FFFFE780E045018DBF
:101B300033B5AA001703FFFF6700635A3389840394
:101B400083270B003E9963170A00834789008504A9
:101B50003E94E1B703560A00DE854A8533F6C90094
:101B600097000000E780E0F16DD10545E1B717036C
:101B7000FFFFE702C35501112A847C000355E500ED
:101B80003ECAB70707003ECC7C003ECE972000003F
:101B9000E78020082A898545480897A0FFFFE7804D
:101BA00020399945480897A0FFFFE780E015AA84EF
:101BB0004A8597200000E780A0082380A40097476B
:101BC000FF1F938767359C434166130606F0939683
:101BD000870113D78701558F93D68700F18E558FD4
:101BE000A207B706FF00F58FD98F11462C00138589
:101BF00014003EC497D00000E78020CF5008A38295
:101C000004008945228597000000E780E0E019C9BB
:101C1000AA851305840397A0FFFFE780E0313C40CD
:101C200085073CC005611703FFFF6700834C17035E
:101C3000FFFFE702C3499790FFFFE780E0342A8463
:101C400005049790FFFFE78020333305A402F14796
:101C500091453305F50297200000E78020BA11E591
:101C600065551703FFFF6700C3489747FF1F23A170
:101C7000A7129790FFFFE78020312A8405049790F0
:101C8000FFFFE780602F3305A402894506059720F2
:101C90000000E780A0B669D59747FF1F23A2A70ED3
:101CA0009790FFFFE780402E2A8405049790FFFF5E
:101CB000E780802C3304A4029747FF1F2394870CEE
:101CC0009790FFFFE780402C2A849790FFFFE780E2
:101CD000A02A930714003385A7029747FF1F239478
:101CE000A70A970701009387E7CA1747FF1F232F0B
:101CF000F7080145BDB71703FFFFE702A33BAA841E
:101D00002E8901449749FF1F93890921130A8006F0
:101D10009790FFFFE78040266347A4000145170323
:101D2000FFFF6700633C3305440383A709024A862B
:101D3000A6853E9597000000E780E0B919E105040B
:101D4000C1BF0545E9BF1703FFFFE702C335AA8AF4
:101D50002E8BB28B368C3A8A814401448149974C50
:101D6000FF1F938C6C1B130D80069790FFFFE7807D
:101D7000A02063C9A40011E085494E851703FFFF29
:101D80006700E3353389A40383A70C025E86D685FA
:101D90003E994A8597000000E780E0B31DC1979007
:101DA000FFFFE780601E0544636D4501D2866286B1
:101DB000DA851305090397000000E780A0D411C15C
:101DC000854985045DB71703FFFFE702A32EC164B1
:101DD00041112A8901449749FF1F9389E913130A86
:101DE0008006FD1436C632C42EC29790FFFFE780EE
:101DF000A01892452246B2466348A400014541011D
:101E00001703FFFF6700432E3305440383A709022E
:101E10003E9509C683473500C18B9DC791C6834750
:101E2000350093F707028DC3630699008357E500D9
:101E3000639C27010357050001CB63E7E500834757
:101E40008500BA97E3CDF5FA050469BF1703FFFFD4
:101E5000E7024326C1642A8901449749FF1F9389F9
:101E6000A90B130A8006FD149790FFFFE780C010AE
:101E70006346A4001703FFFF6700032733054403ED
:101E800083A709023E958357E500638A97006304A0
:101E900099006396270197000000E780E09705040A
:101EA000E1B71703FFFFE702831F89692A8AAE8A19
:101EB000328BB68B8144174CFF1F130CEC05930C2F
:101EC0008006314DFD199790FFFFE780E00A63C659
:101ED000A4001703FFFF670043203389940383277F
:101EE0000C028355CA015A863E994A859700000024
:101EF000E780609E31C1814D15A03384AD038327F7
:101F0000090303D60B00D68533F6C9003E9422851B
:101F100097000000E780E0B609E9850D9790FFFF84
:101F2000E7808003E3CBADFC01A822859700000089
:101F3000E780E08A23040400850471B71703FFFFDC
:101F4000E70263164169AA8A014A174BFF1F130B68
:101F5000ABFC7D19C14B054C9790FFFFE780C0019A
:101F60006346AA001703FFFF670063179309800603
:101F7000B3073A0383290B02BE9983D7E900638E26
:101F8000270163842A01639A570103A4890301E8A6
:101F90004E8597000000E780C0BD050A75BF8357D6
:101FA0000401639977099304C400268597A0FFFF75
:101FB000E78060D385452A8D2685835C040197A040
:101FC000FFFFE780C0CF268597A0FFFFE780A0E74F
:101FD00062056185635905048D45268597A0FFFF3D
:101FE000E780E0CD8945268597A0FFFFE78020CDDB
:101FF0008945268597A0FFFFE78060CC854526852B
:1020000097A0FFFFE780E0CC83470500094793F7DF
:10201000F707639AE7009945268597A0FFFFE780B9
:1020200040CBA30285014848337D2D01231894013C
:102030006A9548C40040A1BF1703FFFFE7022309C8
:1020400037E404008327041D82979747FF1F83C747
:10205000A7D91715FF1F1305254CA300F5008327EB
:10206000441C82978327841C81461306F00F814508
:10207000014582971703FFFF6700A3071747FF1F5C
:10208000130787C618439745FF1F83C5E5D59747B4
:10209000FF1F9387E7D3834687030346970363971E
:1020A000D5009747FF1F2381C7D4828083C587014E
:1020B0000347A7036317B6009747FF1F2386E7D29E
:1020C000828003C687016317C7009747FF1F238DD0
:1020D000D7D0828083C68701130750026319D700C7
:1020E000930760021747FF1F2300F7D0828083C643
:1020F0008701130660026315D60093077002DDB7EF
:1021000083C7870155BF9747FF1F938767CCD44B81
:102110000947638DE6081703FFFFE70243FB1749F2
:10212000FF1F130929C83E8483470900918B9DCF67
:10213000B7E4040083A7041D829783A7441C1745B6
:10214000FF1F1305A5C6829783A7841C81461746E7
:10215000FF1F0346A6C781450145829721C58347D6
:102160000900ED9B1747FF1F230EF7C283470400AA
:1021700093F7F70F85CB91471747FF1F2324F7C627
:1021800097000000E78080EB97000000E78040EFB9
:10219000B7E70400BC4F414691451745FF1F034573
:1021A000A5C382971703FFFF6700A3F4828017037C
:1021B000FFFFE702C3F18D4741116306F504C547F0
:1021C0006308F50285476310F5029747FF1F238FC9
:1021D000A7C0B7E70400BC4B930500101745FF1FCD
:1021E000034585BF829741011703FFFF670063F036
:1021F00085471747FF1F230BF7BEB7E70400BC4B0B
:1022000093050020E1BF9747FF1F938767BCD44B1E
:102210001147638DE600B7E7040083A7071D829787
:10222000B7E70400BC4B930500044DBF05491747B1
:10223000FF1F232927BB83C7070032C62E8493F7CD
:10224000F70FD5D3B7E4040083A7041D7D141374DE
:10225000F40F8297E37689FCB245994703C61500CF
:10226000E3F0C7FCFC4409061745FF1F130545B8FA
:102270008297BC48930500081745FF1F0345C5B565
:10228000829779BF1703FFFFE70263E41747FF1F39
:10229000130707B44047184B1C409746FF1F23AF56
:1022A000F6B26316E4001747FF1F232BF7B213059E
:1022B00084FE9790FFFFE78000AA035564FF978094
:1022C000FFFFE780807297A0FFFFE78060D01703D1
:1022D000FFFF670003E21703FFFFE70243DF9747B3
:1022E000FF1F9387E7AED84BDC4789C797000000F4
:1022F000E78080F985471747FF1F2325F7AE9747EB
:10230000FF1F9387679E9C43930500021745FF1F9D
:10231000034585AC83C787031747FF1F2306F7AC28
:10232000B7E70400BC4B82971703FFFF670063DC2D
:102330009747FF1F23A0A7AA82801703FFFFE7028A
:1023400063D737E404007C4CA1451745FF1F0345C4
:10235000A5A882977C48A1451745FF1F0345C5A73F
:102360009744FF1F9384C4A68297DC4489EB9700AF
:102370000000E78080D91703FFFF6700E3D603D58D
:1023800067FF9780FFFFE7804066AA896DD1D84834
:1023900091476310F7027C4C91451745FF1F034599
:1023A000A5A382977C4891451745FF1F0345C5A209
:1023B000829703A9490103D409018947B7E90400B9
:1023C0001747FF1F2320F7A283A7091D21044204FA
:1023D000829783C784011715FF1F1305E513611941
:1023E0001717FF1FA30AF71283A7491C4180829782
:1023F0009747FF1F238C079E83A7C91C8146094668
:102400009375F40F4A85829711E99747FF1F83C799
:1024100027AE89C79700FF1FE780A07CB7E70400BD
:10242000BC4F2146A1451745FF1F0345E59A8297FA
:1024300099B71703FFFFE70283C993F7052001113E
:102440002E8481CF97000000E78020E91345042007
:1024500005611703FFFF6700C3C993F70510A9CFF4
:102460009744FF1F9384C496DC4897000000E780E0
:1024700020C11747FF1F13072787184383C784010D
:10248000034787036318F700DC4489C797000000FF
:10249000E78080DF85471747FF1F2325F794B7E7BD
:1024A0000400BC4B930500021745FF1F0345C5926E
:1024B00082971345041069BF93F70508BDC7974776
:1024C000FF1F83C7F792E91719469745FF1F9385AA
:1024D00045921305D10093F4F70F1749FF1F0349E5
:1024E000299197C00000E780404093970401C18381
:1024F0001747FF1F13074790231DF100231CF1000E
:102500009747FF1F9387C78C3ACE3ACAD843230612
:10251000010009CBDC439315890154080D46E18580
:10252000680082971345040825B793F72500A5C3D3
:102530009747FF1F9387C789D84B89476306F702E0
:102540009747FF1F83C7078613F7270011EF918B6B
:1025500099CFB7E70400BC4F1306000A8945174519
:10256000FF1F03456587829713452400D5B597372C
:10257000FF1F938767779C4383C787031747FF1F16
:102580002304F78697000000E78060DBF1BF93F734
:10259000050281CB97000000E78060DA1345040252
:1025A00045BD93F7850081CB97000000E780E0D21E
:1025B0001345840071BD93F7150081CB970000008F
:1025C000E780A0B41345140061B593F7450081CBB3
:1025D00097000000E78060B31345440095BD93F772
:1025E000050495C39737FF1F83C7877E91CB97005C
:1025F0000000E780A0A491471737FF1F2324F77E30
:1026000013450404B1B593F705010145E38207E4DE
:102610009737FF1F9387C77BD84B91476310F70409
:102620009737FF1F938707789C4313D7270085832D
:10263000D98F858B91E7B7E7040083A7071D8297A1
:10264000B7E70400FC4F91451735FF1F0345C578D8
:10265000829785471737FF1F2326F7781345040114
:10266000C5BB9747FF1F2385A78882801703FFFFFD
:10267000E702E3A59737FF1F23A207769737FF1FCF
:1026800023A0077685471734FF1F1304E465173727
:10269000FF1F2329F7741C4083C787031737FF1FC9
:1026A0002304F7749790FFFFE780409329C597179D
:1026B000FF1F23A7A7E61C40170500001305A5D799
:1026C00083C787031737FF1F2300F7721717FF1FF2
:1026D000A304F7E49737FF1FA38C076EB7E7040046
:1026E00083A7070882979737FF1F2387A76E1703D3
:1026F000FFFF670003A0B7C7898E938767ED1717A1
:10270000FF1F232FF7E045BF1737FF1F0347476C15
:10271000795555E79737FF1F9387876B03C71700D6
:1027200005079736FF1FA385E66A03C717008D4686
:102730003377D7029736FF1FA38CE66883C617004E
:102740001737FF1F1307475A184393F6F60FA9EEE2
:10275000834787031737FF1F2308F7688547173715
:10276000FF1F2307F7669737FF1F9387A7639C43D5
:102770000145998BA9E71703FFFFE702439537E46B
:1027800004007C48C1451735FF1F0345E564829767
:102790003C4885451735FF1F034505648297014571
:1027A0001703FFFF6700E39483C71700854663950F
:1027B000F6008347970379BF8347A70361BF8280F1
:1027C0009737FF1F83C7C760A1CF1703FFFFE7023B
:1027D000039037E404009737FF1F238B075E7C4884
:1027E00085451735FF1F0345255F82977C4C914532
:1027F0001735FF1F0345455E82977C489145173585
:10280000FF1F0345655D82973C48C1451735FF1F93
:102810000345855C829701451703FFFF6700638DC1
:10282000795582801703FFFFE702638A2A840355E4
:1028300065FF9780FFFFE780401B9737FF1F938757
:102840002759D847BE841DEF9790FFFFE780807718
:102850009C48232004009DEB9737FF1F23A2875835
:102860009737FF1F23AC8756B7E70400BC4B894559
:102870001735FF1F03454556829701451703FFFF94
:1028800067002387630A8700184375BF80C39737A3
:10289000FF1F23A78754C9BF7955CDB71703FFFF83
:1028A000E702E3829737FF1F9387C7648843232695
:1028B000050023240500510597A00000E780C033E0
:1028C0001703FFFF6700E3821703FFFFE702238080
:1028D0001734FF1F130404621C40411199CF9C4719
:1028E0002302B5002AC61CC197000000E78040FB08
:1028F0001C409C4B99C332458297410117F3FEFF60
:102900006700237F17F3FEFFE702637C4111444D0C
:10291000328532842EC69790FFFFE780C0522AC4CA
:1029200022859790FFFFE780205403A84400630CA2
:102930000800B245835744001840224683D545001D
:10294000AA8626850298410117F3FEFF6700637A85
:1029500017F3FEFFE702A377404D1DC808C0970597
:102960000000938565031305440197A00000E780EC
:1029700040169737FF1F9387E7579C43014589E728
:102980009737FF1F23A8875617F3FEFF670063766C
:102990007D55DDBF17F3FEFFE70263730111680089
:1029A0009305F00F02C602C802CA02CC02CE9700FD
:1029B0000000E780A0F1056117F3FEFF6700637375
:1029C0009737FF1F938707539C43D847A1679D07FD
:1029D0006319F70217F3FEFFE702636F01113285F7
:1029E0009790FFFFE7802046230AA10081456800F9
:1029F00097000000E78080ED056117F3FEFF670098
:102A0000436F82809737FF1F9387C74E9C43D847F9
:102A1000A167938777036319F70217F3FEFFE702B5
:102A2000036B011132859790FFFFE780C041230AB5
:102A3000A1008145680097000000E78020E905615A
:102A400017F3FEFF6700E36A82809737FF1F9387C3
:102A5000674A9C43D84795476316F70417F3FEFF70
:102A6000E702E3660111328532849790FFFFE78029
:102A7000803D230AA10022859790FFFFE780C03E9A
:102A800083574400231BA10081453ECC1C406800B5
:102A90003ECE97000000E78060E3056117F3FEFF7C
:102AA000670023658280930785FF8DC38327C5FF59
:102AB00091CFDC4B81CF17F3FEFFE7024361032583
:102AC00085FF829717F3FEFF6700A362828017F3EA
:102AD000FEFFE702C35F2A8432859790FFFFE780FD
:102AE0008036BD4763EBA70018449377F500034594
:102AF000B70041995D8DA305A70017F3FEFF67009E
:102B0000435F17F3FEFFE702835C01117C003ECABE
:102B1000B70707003ECC7C003ECE5C4DA9C72A8497
:102B200013858700AE8497A00000E780E0FCA165D4
:102B30002A899D0548089770FFFFE780603E93054E
:102B4000803EB345B902480893F5F50F9790FFFF13
:102B5000E780C021014781465008A68522859770ED
:102B6000FFFFE7804061056117F3FEFF67006358D0
:102B700017F3FEFFE702A35597000000E780A0F8D7
:102B800017F3FEFF6700E35617F3FEFFE702235437
:102B900001117C00AE843ECAA165B70707002A84F4
:102BA0003ECC48087C00938575033ECE9770FFFFAE
:102BB000E78000371C44480883C5B700BD8997905B
:102BC000FFFFE780A01A500801478146A6852285AD
:102BD0009770FFFFE780205A056117F3FEFF67003B
:102BE000435117F3FEFFE702834E2A84AE84970019
:102BF0000000E78000EEA685228597000000E780B0
